:020000040000fa
:080000000002040000000000f2
:020000040000fa
:100400002ff421000e6f24000e0188000000000070
:100410000c000700e0252e0001002000110007005d
:10042000000020000000e000020032000000020096
:10043000000000001ea50200000000000040da00dd
:100440000000fe004440a900406b21000000e000d5
:100450000300320000002000a00188004440a800f2
:100460000000060091018800800078000000eb0089
:1004700015003700e280400032a0b4009101ba00bc
:10048000e280400032a0b4009102ba00e280400055
:1004900032a0b4000002eb00472bde00f507b200eb
:1004a000602ce10004003a000059eb008301e900f0
:1004b000fdff3e00040037006128e100010032002a
:1004c0000082eb00040007001101ba000200e00006
:1004d000e8ff3a00000006003159ba008301e90044
:1004e0000c0032002159ba008301e90008003200f3
:1004f0000400e00003003a00e280400032a0b400b3
:10050000f5ff370011d9ba008301e900faff3a007c
:100510008100e800e180400032a0b4000000060045
:10052000103f040000000000f64e04000000000030
:10053000ac3f040000000000f04d0400000000008b
:100540000a41040000000000a84d04000000000063
:100550005850040000000000d84b040000000000c8
:10056000884c0400000000001c4d04000000000046
:100570005256040000000000f44304000000000094
:100580001244040000000000304404000000000099
:100590007a440400000000009444040000000000bd
:1005a000804e0400000000005643040000000000dc
:1005b000224c040000000000f04304000000000092
:1005c000c8440400000000003245040000000000a0
:1005d000cc46040000000000ec46040000000000cf
:1005e0000c470400000000002c470400000000003d
:1005f0004c470400000000006c47040000000000ad
:100600008a47040000000000aa4704000000000020
:10061000ca47040000000000ea4704000000000090
:100620000a480400000000002a48040000000000fe
:100630004a480400000000006a480400000000006e
:100640008a48040000000000aa48040000000000de
:10065000ca48040000000000ea480400000000004e
:100660000a490400000000002849040000000000be
:100670004649040000000000644904000000000036
:100680008249040000000000a049040000000000ae
:10069000b24a040000000000d04a0400000000003c
:1006a000ee4a040000000000de49040000000000e3
:1006b000fc490400000000001a4a04000000000089
:1006c000384a0400000000005a4a040000000000fc
:1006d0007c4a0400000000009e4a04000000000064
:1006e000c0490400000000005e3304000000000068
:1006f000003904000000000032390400000000004e
:100700006439040000000000963904000000000075
:10071000103a0400000000005835040000000000fa
:10072000a635040000000000f435040000000000bd
:100730004236040000000000903604000000000073
:10074000de360400000000002c370400000000002a
:100750007a37040000000000c837040000000000e1
:100760001638040000000000643804000000000097
:10077000b238040000000000363a04000000000017
:10078000583a040000000000c839040000000000ce
:10079000ee390400000000007a3a04000000000076
:1007a000cc3a0400000000004e34040000000000b9
:1007b000b63404000000000004350400000000000e
:1007c000ee3a040000000000343e04000000000087
:1007d000543e040000000000803e040000000000c1
:1007e000a63e040000000000cc3e04000000000013
:1007f000ee3e040000000000323e04000000000055
:100800009433040000000000fa33040000000000ec
:10081000e8b804000000000044b904000000000033
:10082000d4b7040000000000eeb704000000000090
:1008300042b80400000000005ab8040000000000a4
:1008400086b80400000000001cbb0400000000008b
:100850004cb904000000000086b90400000000004c
:100860008cbb040000000000123b040000000000ec
:1008700088b104000000000060b304000000000024
:1008800088b3040000000000c4b4040000000000ad
:10089000c6b4040000000000aab704000000000075
:1008a00006ae040000000000b0b304000000000029
:1008b00000ae0400000000000040da000000fe006e
:1008c0000a00fa0080017800e20f500028003e0084
:1008d000b03c8200e10f500008003200802320006d
:1008e0000000e00005003200042320002523200042
:1008f00046232000800178000400370004222000f5
:10090000252220004622200083222000144090004f
:100910000004e000040035008009eb001440900062
:100920000074a00010429800154090000028a30019
:1009300003003a00154090000024a0009042980067
:100940008001eb0007003700154090000008a3006d
:10095000fdff320063c078000000fb00000b780050
:100960008301e800828f5100f7ff3a00080037004a
:1009700030002000b0bf9f00c3bf9f00d1bf9f00c9
:10098000e2bf9f006a80570000c0da006fb997008d
:10099000020078000080fa0000000600020ab90098
:1009a000001bb9000200b800810042008100430032
:1009b000000006000001be002a0107000470a70025
:1009c00003f0a1006509b100160032000d003500ea
:1009d0006828e10006003500f0ff2f00f1ff270036
:1009e0000300e00013003b000100280000000500a8
:1009f00000004000818048008502e900fcff3a00c9
:100a000008003700f88f420002003c008000eb0035
:100a1000000005008100d1000080d3008502e800bd
:100a2000fcff3a000300e00002003b006000100001
:100a3000e080180000000600889fbe008a9fbe006c
:100a40008c1f78001c0107002301330003866c0013
:100a50006450e1002e0032006420e10033003200d7
:100a60006150e1002f0032006120e10031003200ce
:100a700085855500eb07b000090020000804200020
:100a8000050037000804440089844c000a00310046
:100a90000603430087834b000001530081815b0004
:100aa000f8ff33000203be000800a0000804440061
:100ab00089844c00f6ff3900c639dd0083017300dc
:100ac00001003200130020008904d1000884d30003
:100ad0000998a300050032000800a7000300a00049
:100ae0008904d1000884d3008b05e8008904d10073
:100af0000884d3000001eb000281d2000601070048
:100b000001f0a1000cf0a70001f0a000fb003700ed
:100b10006420e100fd0032000801be000200be00ba
:100b2000f7ff37006120e100f80032006000b800f4
:100b3000f3ff37000000200001f82700f0ff370026
:100b400003f0a200889fbe008a9fbe008c1f780021
:100b5000d9000700e00033006450e1004f0032008c
:100b60006420e1005200320003826c0007003b0069
:100b70000905d0000306d000820f54000c065d006a
:100b80000200390002003200890178000306780073
:100b90008582550004003d000003fd008103fd0037
:100ba0008502ea008b854200840f720002003b0040
:100bb00060001000e08018006011b8000005eb0034
:100bc0007a28e1000a00390006007800c75ddd00e0
:100bd000f707b200878075002d0037008281710011
:100be0000a017800610560008180d1000080d30097
:100bf0008502e900f9ff3b000604400087844800b5
:100c000002003b0060041400e0841c000988a3007b
:100c1000070032008a8171008281710061016400e5
:100c20008904d1000884d3008b05e8001700370041
:100c30000978a30013003a000b00e0001300340011
:100c40008b05e9000804440089844c000a447400c0
:100c50000978a3000d003a000b00e0000700340003
:100c60008b05e9000804440089844c0001003a0027
:100c70000b0020000978a300f7ff32000001eb0011
:100c800002003700828171000a017800a20007008b
:100c90000cf0a70001f0a000980037006420e100ec
:100ca00002003a00838f6c00980033000801be00f8
:100cb0000200be0091003700889fbe008a9fbe00e0
:100cc0008c1f78007c0007008300330003866c00d3
:100cd0006450e100240032006420e100270032006b
:100ce0006150e100220032006120e1002100320069
:100cf0008b854200eb07b1000134b800003ab80020
:100d00000804420089844a00013ab8000030b80063
:100d10008880400009014a000400330000004000c0
:100d200081804800020149008b05e900c909dd0006
:100d3000830170000100320013002000c814de009f
:100d40004814dd004709de001200b200c808de00ca
:100d5000088470007000070001f0a1000cf0a700eb
:100d600001f0a000650037006120e100670032005b
:100d70000801be000200be00f7ff37006150e1002d
:100d8000fcff3a0061003700889fbe008a9fbe00ca
:100d9000010578000100e0000400350008003c0077
:100da0000000e00020003200050037006000100065
:100db000e080180002003b0001f02c001a00370010
:100dc0000004be006011b8006b0920000982cf004a
:100dd000020039000882cf000441b000694252008d
:100de0000e00320008003b00828171006101640046
:100df0008904d1000884d3008b05e8000442e80090
:100e0000f9ff3a00050037000804440089844c00cb
:100e10008b05e9000442e900fbff3a003e000700b1
:100e20000af0a70001f0a0004f05be004f04be006d
:100e300000000600f4ff2f005d00370014002000c2
:100e40005b0037004f89de008201780073003700b5
:100e5000809feb00a80007008f87e9000000e000fa
:100e600000000600c70ade00f107b200f50fb2006d
:100e700008003200e1cf4200020032000170a00001
:100e800024000500810f70000100320004080500f5
:100e900044000500810f700002003a0014000500b4
:100ea0008502e9000000400081c04800fcff3b00d3
:100eb0000170a000240005000004be00e9ff070047
:100ec0000003be000405be000200be00e5ff0700ef
:100ed000844f7500000006000200be006450e1006f
:100ee000050036006420e100020036000968a30016
:100ef00001003a000800be000160a0004f06780023
:100f00004f05be004f04be0000000600f0ff2f009a
:100f1000f1ff2700f9ff37008100200061805500b4
:100f20000b003d000b00200061fe2f000100e100de
:100f30001d00340082817100610164008904d100c8
:100f40000884d3000000e800faff3a007100200096
:100f500061006400030070000200600009003200bc
:100f600061044400e0844c000988a50005003200bb
:100f70008b05e8006808e10002003a008904d1000e
:100f80000884d300f20f20000258e10005003d0064
:100f9000c75ddd00f907b2008980750008007800a0
:100fa000000006000bf827008b0078000000050009
:100fb000889fbe008a9fbe00841f7800beff070086
:100fc0004f00780011003300f0ff2f00838f6c007a
:100fd00006003b00040565000a00a7000800370072
:100fe00009f0a6001000200008003700820f54000e
:100ff000838f5c00030039001000200001003e00d8
:101000000000200009f0a7000000ea004f05be0024
:101010004f04be000000e00000000600889fbe00f4
:10102000830478000300e0002c00350003003c003e
:101030000082700004027100260032003643200056
:10104000c50020008383cf000a0039000541b100ac
:101050008283cf00070039000541b1008183cf00b2
:10106000040039000541b1008083cf000100390040
:101070000541b10085c353006022b8001200320060
:101080000a003b0084827200610260008301d1008b
:101090000281d3008180d3000080d3000603e800e2
:1010a0008743e800f7ff3a000700370000004000e0
:1010b0008180480002014900838149000603e9005c
:1010c0008743e900f9ff3a003400070009f0a70060
:1010d00003f0a0004f04be000000060060001000f6
:1010e000e080180060011900e0811900d3ff3b0087
:1010f000033e2c00f7ff3700889fbe008a9fbe008a
:101100008c9fbe000404be000605be00809fbe008a
:10111000829fbe004d000700040678000800be0054
:101120000a01be0049000700840678004f03be0094
:101130004f02be008d4f76007fb097001300330042
:10114000f0ff2f008b8f6b0006003b000d06660042
:101150000c00a7000a00370007f0a60010002000ce
:101160000a003700880f5200898f5a008a0f5b00ef
:101170008b8f5b00030039001000200001003e004f
:101180000000200007f0a7000000ea004f06be00a4
:101190004f05be004f04be000000060018002000ee
:1011a00057002000080453000d003d0006002000f9
:1011b00097fc2f000740e1001e003400848272007b
:1011c000610260008301d1000281d3008180d300dd
:1011d0000080d3000804e800f8ff3a004700200030
:1011e0006104600005047400040464000d00320012
:1011f00061004000e080480060014900e081490052
:1012000003b8a500070032000603e8006538e100d6
:1012100004003a008301d1000281d3008180d30011
:101220000080d300f87f20000830e1000300350083
:10123000080378006000b8006011b8004433dd0096
:10124000f300b200830173000000060005ff2700d1
:1012500005826100070032000428e100010032002d
:10126000240005000600070001003a0044000500c4
:101270000408050002000700f9ff3a001400050009
:101280006f82610081027000850271008502720028
:1012900000000600881f7800000478005001be009e
:1012a0004000be000400400085804800060149005f
:1012b00087814900009cbe000294be000400e1004a
:1012c0000588e1000690e1000798e1000200310086
:1012d000680044001008e8004f0478000000060091
:1012e000f4874700889fbe008a9fbe008c9fbe0087
:1012f0008e1f78000205be000004be00d4b79f0018
:10130000e5b79f00f6b79f0087bf9f000000eb0086
:10131000c0b79f00b0b79f00a0b79f0090b79f00d5
:1013200080b79f000d042000bfb097004fb097001a
:10133000000140000000e0000f003d004f08de000b
:1013400000007100c0b79f009e00070001003d0033
:1013500012002000a100070001003d001200200043
:10136000a6000700b1000700b60007000f0040000c
:10137000c8ff0700220037004f08de00000671009a
:10138000ccb79f008f00070001003d001200200035
:101390009200070001003d001200200097000700a6
:1013a000a20007000fb297009fb297002fb39700db
:1013b000bfb39700a90007000000520081805a00c7
:1013c00002015b0083815b0080b79f0091b79f00a3
:1013d000a2b79f00b3b79f000007eb009f00070074
:1013e0000020e10001a8e10002b0e10003b8e10043
:1013f000010031001e0020000e005600c0b79f0003
:101400004fb297000400e0000700350010002000f4
:10141000010020006011b800080470008984700089
:101420000a0571008b8571008d06e900beff3a0048
:101430000400e00003003d00820007000f004000b0
:1014400094ff07004fa897000000e00004003a0056
:101450000fb497009fb497002fb59700bfb59700c2
:10146000940007004f0778004f06be004f05be00ee
:101470004f04be004f01b10000000600881f780035
:1014800018002000881f780095ff07008f87e9006b
:101490004f04780000000600801feb0090ff07005b
:1014a0008f87e90000000600889fbe008a9fbe006b
:1014b0008c1f78006e00070007003d0073000700d6
:1014c000e00f5b00e08f5b0007003d00320007008b
:1014d0000006eb00040037003400070002003d0066
:1014e0002a0007001c00200072000700e3ff07002d
:1014f0000203be000002be000c00e000010032004a
:10150000220007000400be000601be004f0678005e
:101510004f05be004f04be0000000600889fbe00bd
:101520008a9fbe008c1f78005100070005003d0017
:1015300056000700e00f5b00e08f5b0006003d00f7
:10154000040037001900070003003d006000b800e8
:101550006011b8001000070056000700ceff07001a
:101560000203be000002be000c00e00001003200d9
:10157000060007000400be000601be004f0678000a
:101580004f05be004f04be00000006006000b8001a
:101590006011b80000003700040250008582580036
:1015a0000603590087835900000006000006eb007f
:1015b000e00f5200e08f5a00e00f5b00e08f5b000d
:1015c000000006000180400090b79f000001eb0082
:1015d0008fb097000100e0000000060002007000dc
:1015e00090b79f000180400080b79f000001eb0092
:1015f000ffa897000100e000000006000200700054
:1016000080b79f00018040006faa9700cf20de00c6
:1016100001007000f0af9f000402420025000700a7
:101620004f18de000002720000000600e4af9f00c9
:101630000804440089844c000a054d008b854d0048
:10164000000006003fb29700cfb297005fb397004b
:10165000efb3970000fe2f00000006003fb0970098
:10166000cfb097005fb19700efb197000000060080
:101670000205be000004be00e00f5000e08f5800dd
:10168000e00f5900e08f5900000006006000b8002c
:101690006011b80008045000898458000a055900f8
:1016a0008b8559001c002000e00f5200e08f5a008b
:1016b000000006000800be000a01be00000006008f
:1016c0002800fa00889fbe008a9fbe008c9fbe0043
:1016d00003866b00d00107000028a30064003a00d5
:1016e0000128a30067003a000008a30062003a0046
:1016f0000108a30065003a001e009000be0890009b
:1017000081064000ed3fb100f4805700ee019000eb
:10171000111ab8008e099000311bb8009e09900084
:10172000311cb800511db800f48557004600070071
:10173000fe0190003a0007008b85e8003e0007009c
:101740008e09900040000700ee0190003400070071
:101750008b85e800380007008e09900040000700e4
:101760009e0990001b18b800890440000a854800b3
:10177000fe019000340007008b85e8003800070068
:10178000ee019000300007008e0990001b18b80091
:10179000890440000a8548000a98a30008003a001e
:1017a0000402420085824a0006034b0087834b00f7
:1017b00008044c0089844c000a054d008d06e900a0
:1017c00084827200850273004c3add00850272004b
:1017d0000100320015002000443ade001400b2007f
:1017e0004538de00cb45dd000b007000c540de0053
:1017f000cb4ddd008b8070004549de00cb55dd0010
:101800000b017100c551de000d03780063fe070077
:1018100003f0a1000cf0a70003f0a0009201370034
:101820001b18b8008502400006834800e0834b0087
:1018300060044c00070037001b18b8000603400086
:1018400087834800faff37001b18b8008703400061
:1018500008844800e0844c0060054d00000006004c
:101860001b18b8000804400089844800faff3700bc
:101870000108a30079013a005800be005801be00db
:10188000e3ff37000008a30074013a000904780060
:10189000f9ff37008103780072fd07000001be00e8
:1018a0006000b8000478a30013003a006220e10051
:1018b00015003e000d0039008301d1000281d300e4
:1018c0008180d3008301d1000281d3008180d300c5
:1018d0008301d1000281d3008180d3000538b0009c
:1018e000c42add00f300b2008381720007f0a70074
:1018f00003f0a00000000600f3ff2700f2ff2f0016
:101900006110b900fbff370003ff2700f7ff370026
:101910008f1fd100f8fd07008f87e9000000e0006d
:1019200000000600801feb00f3fd07008f87e90031
:101930000000e000000006001400fa00889fbe00ce
:101940008a9fbe008c9fbe000005be000206be003e
:10195000680047000c90be000a90be0047010700d7
:101960006400e1001a00320016003e006100e10050
:101970001a0032006e049000fe0490000e0b9000de
:101980009e0b90006011b8009e0590000b38b100ce
:10199000d501200082817100610164008703d100bc
:1019a0000683d3008984d3000884d3008502e9002c
:1019b000f8ff3a0058fd07000df0a70001f0a00065
:1019c00029013700f1ff2700f0ff2f002601370023
:1019d00001f8270000002000f7ff37006000b80082
:1019e000f5ff37004c0107000509780000000600ec
:1019f0002800fa00889fbe008a9fbe008c9fbe0010
:101a000007067800878669000c003b000304780015
:101a10008704780008f0a10009f0a100840f5000ad
:101a2000858f5800860f5900890f5c000300330032
:101a30000cf0a20001003a000cf0a100f600070033
:101a40006400e1005f003200780147006408e100b3
:101a5000610032006c014700748557003200be00ff
:101a60001201be003a04be001a05be001e0390001b
:101a7000be0a90008503530006003d000004fd00ef
:101a80008104fd000205fd008305fd008703ea00d7
:101a9000050378000df8a300040032006004140070
:101aa000e0841c0060051d00e0851d006022b80078
:101ab0007d0320000d38e1008006eb000b003900ab
:101ac0004433dd00f300b2008301730039003700b6
:101ad000848272000d027800e10664008b85d100db
:101ae0000a85d3008984d3000884d3008703e900e2
:101af000f7ff3b0008004000898048000a014900c8
:101b00008b81490004003b0060001000e080180059
:101b100060011900e08119000358a3000900320098
:101b20008d82720084827200610260008301d100a4
:101b30000281d3008180d3000080d3000603e80037
:101b40001b0037000348a30017003a000600e0001e
:101b5000170034000603e9000d00a3000000480050
:101b60008180480002014900838149000348a300a5
:101b70000f003a000600e000090034000603e90007
:101b80000000400081804800020149008381490033
:101b900001003a000003eb000348a300f5ff320008
:101ba0006022b80002003700848272006182660001
:101bb0007afd070003f0a1000cf0a70003f0a000dd
:101bc000a9003700640147006408e10002003a0000
:101bd0000df8a300a1003a003200be001201be00c1
:101be000a10037001400fa00889fbe008a9fbe0043
:101bf0008c9fbe000004be000205be0068004700c6
:101c00000a90be000890be009c0007000070a7006c
:101c10000bf0a1000bf8a30020003a009e099000f1
:101c20000e099000fe0090006e0090009e02900051
:101c300034432000848252008b0032000a003c00b2
:101c4000b4fc2f000428e100140034008301d1000b
:101c50000281d3008180d3000080d3008502e80098
:101c6000faff3a0080003700b40020000428e100a9
:101c700007003c000000400081804800020149004c
:101c8000838149008502e900faff3a0076003700b7
:101c90000300280002002000010037006011b80096
:101ca0006000b800700037002800fa00889fbe006e
:101cb0008a9fbe008c9fbe0003866b005600070003
:101cc0006400e100440032006408e1004a00320090
:101cd0006100e100460032006108e1004900320085
:101ce000ec0647006000b8003d02be003d03be00a8
:101cf000f48657006011b8003d04be003d05be00eb
:101d00007d0320000b0037000000a0008d06e900d5
:101d1000130032000402420085824a0006034b0091
:101d200087834b0000004000818048000201490089
:101d3000838149000802520089825a000a035b002d
:101d40008b835b00f0ff3b000802420089824a005f
:101d50000a034b008b834b008d06e900edff3a0030
:101d60008482720086827200f707b2008782720056
:101d700001003200150020001e0490003e0b900070
:101d800006035400e63fb0000368a30007003200da
:101d90000000a7000500a0008301d1000281d3004c
:101da0008180d3000080d3000603e8008301d100c6
:101db0000281d3008180d3000080d3000002eb00b9
:101dc0000482d200f5fc070003f0a1000cf0a7008c
:101dd00003f0a00024003700640247006408e1001b
:101de0001e0032003400be003401be00f6ff370092
:101df0006108e100190032006011b8006000b8000d
:101e0000f1ff370003ff270002002000fbff37002f
:101e100007f0a200f6fe3700680447000294be00f7
:101e20000094be00fc0447008694be008494be006b
:101e30000900780011000700080078000f00070073
:101e400099007800814f70000b003b000800be0035
:101e50003e0007004f00b10003003700f3ff2700ea
:101e6000f2ff2f006110b9004f06be004f05be0003
:101e70004f04be000080fa000000060080007800d9
:101e80005002be005003be004439de00f700b2002d
:101e9000f37f200003016100090032000218e10015
:101ea00016003a008501720083017300838173007c
:101eb0000008200015003a00400020001300370001
:101ec00085017200830173008381730005003a006d
:101ed00004a8be0006a8be00100020000b003700ba
:101ee0000201e9000402420085824a0006034b0019
:101ef00087834b000748a300f9ff32000740a0008a
:101f000004a8be0006a8be002000200080009800a3
:101f100092009800000006000003be00d1fb0700fd
:101f20006220e100020032000600be00050005004c
:101f3000e507b100f107b20004f0230084807000cf
:101f400007f0a70001f0a00024000500e482400093
:101f50001078a30007003200640240001178a3004b
:101f60003400be001401be00040032000330a7009c
:101f7000000006003500be001501be000330a000c1
:101f8000000006000c00fa00889fbe0000047800e4
:101f9000cfb09700f0ff2700d0bf9f008004eb0078
:101fa00099bf9f0088bf9f00a8bf9f00200c200002
:101fb000b0bf9f007881570070805700dd00070098
:101fc0000fb89700094878000fb897000804500030
:101fd000080078004f04be000080fa0000000600f0
:101fe0000001780000c2b300010037000201e800e0
:101ff0009240780080cf5000fcff3200e9cf5000c3
:10200000faff3200d0c2b30080cf500003003a0084
:102010000201e80014c0b300050037000042eb00e5
:10202000b0c2b30080cf500001003a000201e800c6
:102030008000eb0005fd2f00040037006a08b9009e
:1020400000804100850040000201e8009201fb0091
:1020500005804100e90f5000f8ff36000404e0005d
:10206000010032008100ea00010078000000060053
:10207000810178000002eb000b003700e44078009b
:102080000104e000030032000402e80093cf500096
:10209000040032008180fb001380fb0000805000b0
:1020a000000006008301e800820f5200f3ff3a00af
:1020b000000005000003780080027800020278002a
:1020c0008001eb00080037000402e90063c07800db
:1020d000805a78008301e8000004e00002003a0022
:1020e0008000eb0006003700828f5100f6ff3a00b7
:1020f000fbff37000040eb0080f07a008100e80031
:10210000848f5000fbff3a000600780000000600b4
:10211000889fbe008a9fbe008000780000c2b30086
:102120000100370089007800810478003944780084
:10213000804f5400fbff3200e94f5400f9ff32009a
:10214000d0c2b300804f540004003a001944780014
:102150008184e8001ac0b300060037000045eb0098
:10216000b0c2b300804f540002003a001944780016
:102170008184e8006022b8000a003700a200200035
:10218000030020000400be0004fa07000b414400d5
:102190000281fb000300200000024100818249000f
:1021a000394478000880fb000bfd2f000b00400035
:1021b000e90f5000f1ff36000a04e000020032008f
:1021c00060021200e0821a000400be004f05be004b
:1021d0004f04be0000000600889fbe008a1f7800e2
:1021e000804078000004e00021003d008040ea00cb
:1021f000d0c6b30080cf5000090034008104fb003a
:1022000042062000110009008204d8000001780075
:10221000010078004311dd002a9421001f003700df
:102220000100fb002394210039003700a2002000a8
:10223000110009000200d8000001780001007800b8
:102240004311dd00030141004300dd0003004000b5
:102250003002be002003be0042209000d220900039
:10226000f22190006221900015fd07002e0037003a
:10227000d0c6b30080cf5000230034008104fb009f
:1022800042062000110009008204d80000017800f5
:10229000010078004311dd002a9f21000a0141005e
:1022a000a8002000110009000800d8004300dd004c
:1022b0000a00400040229000d0229000602390004d
:1022c000f02390000288900092889000b2899000dc
:1022d00022899000fafc0700801f78000102780034
:1022e000110009008804d8000102fd004f007800a9
:1022f0000402fb004322dd000a0242005403be0038
:102300004402be00d8ff37000100fb00239f2100dc
:10231000eacf5000c5ff3c004300dd000300400051
:102320005001be004000be004f0578004f04be00c3
:10233000000006008f03b000889fbe008a9fbe0089
:102340008c9fbe008e1f7800e0b79f00f1b79f0002
:1023500082bf9f000000eb00a0b79f00e60437009b
:102360008001eb0050c2b30080cf50000900320062
:102370000100fb00efb09700ec040700e10f400004
:10238000dd043200afb097008100e800a1b79f00e4
:10239000d90437007fb1970092407800d0c2b300d3
:1023a00080cf50000c00320007003c006d40500010
:1023b00080cf50000d0032006b40400080cf5000b5
:1023c00019003a000e00370000c3b30080cf500060
:1023d00015003a000f0037000330a0007fb29700cd
:1023e0000402e800f4b79f00eaff37000300a000f2
:1023f000ffb297008502e800f5b79f00e5ff3700c0
:102400000310a0007fb697000c06e800fcb79f0001
:10241000e0ff37000320a0007fb097000000e80035
:10242000f0b79f00dbff37000318a3000100320064
:102430000300a1000338a300010032000320a10023
:102440000100fb0002fd2f0002004000e90f5000d8
:1024500010003e008000eb00c1b79f000202780030
:102460004fb197006a10b900ffb297001501fb0049
:102470000001410004014100c2b79f005500fb006c
:10248000f5b79f0004004000e90f50000d003e002a
:10249000f3ff37000006eb00ccb79f00a0c2b300eb
:1024a00080cf500007003a000fb89700c0007800b6
:1024b00080bf9f00c1b79f007fb197000201e80075
:1024c000f2b79f00e0c2b3007fb29700944f1000b4
:1024d00021003a00830678000de0a0008400e800a7
:1024e00064405000914f100004003200f1b79f008b
:1024f0008002eb00b5b79f00100037000fbe9700b9
:102500004c0078008cbf9f00b0b79f00ffb09700d1
:102510008180e800f1b79f00130037003fb29700b9
:102520006a20b9000000410003004000b0b79f00de
:10253000ffb297008502e800f5b79f007fb69700cd
:102540001c01fb0003fd2f0003004100e90f5000b8
:10255000f2ff360004003700830678000dc0a000ab
:102560000000eb00b0b79f007fb19700b240780049
:10257000f2b79f00c17f9f00c0c6b30080cf50005c
:102580002700320014003c006840500080cf50000b
:102590009d00320009003c006c40500080cf50008c
:1025a000290032006b40400080cf500072003200a2
:1025b0000104e000560432008e00370060c6b3000c
:1025c00080cf50001c0032006340400080cf50009c
:1025d00088003a008c00370030c7b30080cf50002d
:1025e0001c00320007003c006440500080cf5000c7
:1025f000130032000040e80080cf50007d003a0018
:102600001100370050c7b30080cf50007d0032006a
:102610006340400080cf500076003a000b00370046
:10262000000028000d48a30001003a00000120002e
:1026300080867600ccff37000da0a0007200370026
:102640000d60a000700037000d50a0000d70a000bc
:102650006d0037008fb997004300780083bf9f005b
:10266000000478000000e00001003a000874240033
:102670008004eb00010037008104e8008900780045
:10268000088044001004e000fbff3a003fb29700ce
:102690000400e00003003200890f52000100310005
:1026a000840478000007eb00cfb29700898f5200b6
:1026b00001003600098752004368de00e106600031
:1026c00019003a000d06780009003700efb09700b6
:1026d0000002200015040700e10f40000300320053
:1026e0002fb097000000e800a0b79f000c06e8009c
:1026f0008e0f5600f5ff3a000087eb000a00370006
:10270000880078003100fb0001047800efb09700ea
:1027100006040700e10f400003003200afb097004d
:102720008100e800a1b79f000900e900800478005b
:10273000e10f4000f2ff3a000006eb000d00e00060
:102740000a003a00ec033700efb0970000022000c7
:10275000f6030700e10f4000030032002fb197009d
:102760000201e800a2b79f000c06e8008e0f560099
:10277000f5ff3a00e00337008fb997004300780077
:1027800083bf9f00cf80de000101780082017800c6
:102790000205be000004be000203be000002be002f
:1027a0004822de00482edd0004027600c47f9f0030
:1027b0000d48a3000a0032000404e00008003200c3
:1027c000e14f420006003200d1fb2f00018047009c
:1027d00004487800184098002900200002003700c3
:1027e000d07f9f0019002000d2fb2f0002844700f9
:1027f000a6ff3700c3fb2f00038447001900200009
:10280000a2ff37000d0cb3000070200000826600ac
:10281000270232000dc8a30002003200640020002d
:10282000b4b79f000d48a300050032000fba97000f
:102830004401be004400be0084bf9f000400370076
:102840008fba97004500be0085bf9f0011fc0700ae
:10285000e0af9f00f1af9f0082b79f0093b79f004a
:102860006022b8006033b8006fa89700ffa89700f7
:102870000fb197009fb1970025fc07000000e00012
:102880000a003d006fa89700ffa897000fb19700be
:102890009fb1970003f0a200e0af9f00f1af9f004f
:1028a00082b79f0093b79f003d00b3000000eb008c
:1028b00080a79f006022b8006033b8006fa897001f
:1028c000ffa897000fb197009fb1970015fc070074
:1028d0000000e000340032006fa89700ffa89700c6
:1028e0000fb197009fb1970013fc070003fc2f0066
:1028f000038147003bfc07000fa097000000e900a0
:102900006300b900a2002000110009000200d800f5
:102910008000fd0081a79f000100e00002003d0053
:102920000100e90080a79f000fa497000840ea007b
:1029300029fe07006faa9700ffaa97000fb3970020
:102940009fb397005efb0700a0af9f00b1af9f0051
:10295000c2af9f00d3af9f006022b80006002000e6
:1029600007ff2300eafb07000000e00002003d0033
:102970000800e9000b0037006022b80006002000c4
:10298000470224002fa89700bfa897004fa99700df
:10299000dfa997002ef907000000e00002003500d3
:1029a0000800e80080a79f003fb29700f80f520090
:1029b00057003c00d0c6b300804f520029003600bb
:1029c0000485fb0042062000110009000285d800a2
:1029d00000017800010478004311dd002b942100f0
:1029e0000b0141006022b8000600200007fe230012
:1029f0000288900092889000b2899000228990000d
:102a00002ffb0700a9002000809fbe0011000900d5
:102a10000984d800000478004f00be004344dd0064
:102a20000b04440048229000d822900068239000b4
:102a3000f823900022fb0700801f78000102780035
:102a4000110009000985d8000102fd004f0078003f
:102a50004322dd000b0242005403be004402be00cc
:102a60001f0037000480fb0029942100ea4f520028
:102a700014003600a2002000110009000280d800d6
:102a800000017800010478004311dd0009014100d4
:102a90006022b8000600200007fe230042209000bc
:102aa000d2209000f22190006221900004fb0700e8
:102ab0004344dd00090444003802be002803be0080
:102ac000070037004300dd00090040006022b80025
:102ad0000600200007fe23005001be004000be009b
:102ae000f7fa07000002be000203be006fa89700bd
:102af000ffa897000fb197009fb19700bcfb07009c
:102b0000e0af9f00f1af9f0082b79f0093b79f0097
:102b10000fa49700e90f540015003c006022b80094
:102b20006033b8006fa89700ffa897000fb1970017
:102b30009fb197007bfb07000000e00032003200ed
:102b40006fa89700ffa897000fb197009fb197005b
:102b500024fc0700e00f5000e08f5800e00f590000
:102b6000e08f590028003a00e10f5400260034009d
:102b70000400200005002e00b6e02200170124000a
:102b80002fa89700bfa897004fa99700dfa997002b
:102b90005ffb07000000e00002003d0073005400ee
:102ba000010037007200540080a79f000fc09700fb
:102bb00089fd0700a0af9f00b1af9f00c2af9f008b
:102bc000d3af9f000002be000203be006fa89700b3
:102bd000ffa897000fb197009fb1970032fc070044
:102be00000fc07000205be000004be006000b80043
:102bf0006011b800a0a79f00b1a79f00c2a79f00c7
:102c0000d3a79f002e0037006fa89700ffa897005a
:102c10000fb197009fb19700f2fb07000205be00bd
:102c20000004be00e00f5000e08f5800e00f590094
:102c3000e08f590002003500f8f807001300370054
:102c400010002000010020006011b80008006000a2
:102c5000898060000a0161008b8161008b03d100d3
:102c60000a83d3008982d3000882d3000000720057
:102c7000818072000201730083817300e7f807000e
:102c80000002be000203be0059fb07000002be00a6
:102c90000203be006fa89700ffa897000fb197002e
:102ca0009fb197005afc0700a0a79f00b1a79f0003
:102cb000c2a79f00d3a79f000000eb0080a79f0042
:102cc00014c0b30025aa21000b0037000400fb004c
:102cd0004300dd00050040005001be004000be0082
:102ce0000040e10001c8e10002d0e10003d8e100aa
:102cf000030039000442e800f44f5200f3ff3a00a9
:102d0000c47f9f000400fb00bfb09700008040001c
:102d10008fa09700010040004fb1970000075100bd
:102d2000bfb197000300e000010032000e07e90088
:102d300063806600010032000e07e9000d28a30041
:102d400026003200e18066000d18a3000c0032005e
:102d5000d00220000100e00001003a000080e900fc
:102d6000efb0970071020700e10f40001800320039
:102d70002fb297000402e800a4b79f0014003700a8
:102d80000100e00012003200efb0970000022000c6
:102d900066020700e10f40000d003200afb297005d
:102da0008502e800a5b79f0009003700efb0970043
:102db000000320005d020700e10f40000300320025
:102dc0002fb697000c06e800acb79f000e07e9008d
:102dd0000e00e000f5ff3c003d0037000d38a30079
:102de0000a0032000b003700efb09700000220000d
:102df0004e020700e10f4000030032002fb09700a1
:102e00000000e800a0b79f000e07e9000e00e000f8
:102e1000f5ff3c00e18066000d18a3000c003200b5
:102e2000d00220000100e00001003a000080e9002b
:102e3000efb097003d020700e10f40002400320090
:102e4000afb097008100e800a1b79f0020003700d5
:102e50000100e0001e003200efb0970000022000e9
:102e600032020700e10f4000190032002fb1970035
:102e70000201e800a2b79f00150037000000fb0028
:102e80004300dd0021aa2100010040003002be0005
:102e90002003be000800be000a01be0077f907004b
:102ea000a4002000050020006033b8007af9070074
:102eb0000003b000efb097001c020700e10f4000d4
:102ec00003003200afb197008301e800a3b79f0071
:102ed0004f7a97000440e900c07f9f00e14f400017
:102ee000e6ff3a000b003700efb097000003200028
:102ef0000e020700e10f400003003200afb297005e
:102f00008502e800a5b79f000fa097000000e90028
:102f100080a79f000fa097000000e000f2ff3c0098
:102f20003fb6970020c1b300f20f560001003c00ed
:102f30006fe09700c07f9f00cf7897000100fb00f3
:102f40003fb1970000005100e0a79f000104e0009e
:102f500008003200efb09700e0022000f301070004
:102f6000e10f400003003200afb197008301e80099
:102f7000a3b79f004f78970097fc07000002be00a0
:102f80000203be002fa09700bfa097004fa197009b
:102f9000dfa19700caf9070012fb07001e003700e7
:102fa0000000fb004300dd002caa21000c004000c3
:102fb0003002be002003be000800be000a01be00b1
:102fc0002ef90700a4002000050020006033b8009f
:102fd00031f907000003b000efb09700d3010700fc
:102fe000e10f4000030032002fb297000402e80016
:102ff000a4b79f00cf7a97000500fb004300dd00d7
:103000000c0040003002be002003be000800be00dd
:103010000a01be0020f907000205be000004be0040
:103020004f7e97000c40e900c07f9f00e14f4000b9
:10303000dbff3a000006eb0009003700efb0970015
:1030400000032000b9010700e10f40000300320037
:103050002fb097000000e800a0b79f000c06e80022
:10306000efa09700810f5600f4ff3a000d38a3003f
:10307000a10132000e00e0009f0134000006eb00c9
:10308000efb0970000022000a8010700e10f400008
:10309000030032002fb197000201e800a2b79f00a1
:1030a0000c06e8008e0f560093013200f4ff370043
:1030b0000d007800000cb20028003a000d00e0007e
:1030c00005003d008fb997004305be004304be00d4
:1030d00083bf9f00140037000d48a3000b0032008f
:1030e0000fba97004400be0084bf9f004f89de00e6
:1030f000cf91de000002be00020378008203780058
:103100000605be000404be00070037008fba970012
:103110004500780085bf9f0000047800cfc4de0022
:10312000090578008a057800e00f5400e08f5c0004
:10313000e00f5d00e08f5d0020003d003d00b3002a
:103140006000b8006011b80008045000898458007d
:103150000a0559008b855900180037000d00e00062
:1031600005003d000fbe97004c05be004c04be009c
:103170008cbf9f00110037000d48a30008003200eb
:103180008fba97004500be0085bf9f0004017800fc
:10319000840178000205be000004be00070037006d
:1031a0000fbe97004c0078008cbf9f000004780091
:1031b000090020000a0020000b0020003fb097000b
:1031c0000000e00007003a00e00f5400e08f5c00d0
:1031d000e00f5d00e08f5d0002003a00110020006a
:1031e000b1b79f000d0778000e0cb200000420005c
:1031f000800f57002f00320003003c000e00e0005b
:10320000070032003f00370000082000800f570001
:1032100014003200000c2000800f570039003a00e3
:1032200014c0b30025aa21000b0037000400fb00e6
:103230004300dd00050040005001be004000be001c
:103240000040e10001c8e10002d0e10003d8e10044
:103250002b0039000442e800f44f5200f3ff3a001b
:103260002700370000012000010020006011b80095
:1032700014c0b3000040e10001c8e10002d0e10049
:1032800003d8e1001e003900450020000000d000f6
:103290008180d2000281d2008381d2008502e900c0
:1032a000faff3a000442e800f04f5200f1ff3a0002
:1032b0001300370080002000010020006011b800da
:1032c00014c0b3000040e10001c8e10002d0e100f9
:1032d00003d8e1000a0039003c0020000000d000c3
:1032e0008180d2000281d2008381d2000c06e900e5
:1032f000faff3a000442e800f54f5200f1ff3a00ad
:10330000c47f9f00cf7897000100fb003fb197007a
:10331000820f500002003d00c27f9f000400370072
:10332000bfb19700808f510001003d00b0b79f00f2
:103330004fb297000400e000040032006380660092
:10334000020032000402e900c4b79f000de8a300a8
:103350000b003200cfb297003fb697008c8f52001f
:1033600003003c000000eb00c0b79f0004003700e2
:10337000cfb097003fb1970082805000c1b79f0047
:10338000cf7997000300fb000002eb0094a79f0099
:10339000cfb29700808f52000200340000805200ac
:1033a00090a79f000d28a30037003200e18066003f
:1033b0000d18a3000c003200d00220000100e00034
:1033c00001003a000080e900efb09700d700070045
:1033d000e10f40000e0032002fb697000c06e80007
:1033e000acb79f000a0037000100e000080032007f
:1033f000efb0970000022000cc000700e10f400072
:10340000030032002fb097000000e800a0b79f0033
:103410009fa097000100e0000f0032000006eb00c3
:10342000efb0970000032000c0000700e10f40004c
:10343000030032002fb197000201e800a2b79f00fd
:103440000c06e8009fa19700830f5600f4ff3a0096
:103450000002eb0094a79f00bfb29700c328dd00d5
:10346000a0a921008080400091af9f004228dd008c
:103470006400500080af9f006328b900f0a79f0050
:1034800063065000820037001fa697000c00e00082
:1034900011003200688066000f003a0000067800d4
:1034a000efb0970000022000a0000700e10f4000ed
:1034b000030032002fb097000000e800a0b79f0083
:1034c0000c06e8009fa09700810f5600f4ff3a0019
:1034d0000001eb0092a79f00e18066000d18a30099
:1034e0000c003200d00220000100e00001003a0090
:1034f0000080e900efb097008c000700e10f40006a
:10350000d5ff3200afb197008301e800a3b79f0059
:10351000d1ff37000100e000cfff3200efb097008d
:103520000002200081000700e10f4000caff3200c6
:103530002fb297000402e800a4b79f00c6ff37002f
:1035400000042000800f57003000320003003c00d0
:103550000e00e000070032003d00370000082000a8
:10356000800f570011003200000c2000800f570020
:1035700037003a001fa897003002be002003be00ab
:103580000800be000a01be00bcf70700a40020002e
:10359000050020006033b800bff7070004c3b30084
:1035a00004424000c47f9f00290037007574240046
:1035b000d5b79f000d58a30002003a008075240083
:1035c000d0b79f0014002000050020006033b80031
:1035d0008fa897008100e900050033000402d000a5
:1035e0008582d2000683d2008783d200f9ff37009c
:1035f0000800be000a01be00a0f707006f006000cf
:103600005fb197006240780010003700140020007e
:10361000050020006033b8008c0178008301e900c8
:10362000050033000402d0008582d2000683d20058
:103630008783d200f9ff37000800be000a01be00f0
:103640008ef70700674060000043b000c07f9f0016
:103650004f7a97000400fb00efb09700330007009b
:10366000e10f400003003200afb297008502e8008e
:10367000a5b79f001fa897006800500090af9f005b
:103680008fa89700e480500081af9f00630656002a
:10369000d0ff2f003fb197000090b900ffa1970025
:1036a0000080410063005000800f5600a4ff3a00e4
:1036b0000d38a300100032001fa297000400e000a4
:1036c0000d0034000006eb00efb097000002200070
:1036d00016000700e10f400003003200afb2970070
:1036e0008502e800a5b79f000c06e8001fa0970020
:1036f000800f5600f4ff3a007fb19700b240780087
:10370000f2b79f00c17f9f000104e00014fb3a0064
:103710002fb097004f0778004f06be004f05be0040
:103720004f04be008f03b10000000600889fbe005a
:103730000001780001047800b10090000118a30096
:103740003d0032000198a30003003a0018009000e9
:103750000000e00038003a000190a0003104980019
:1037600082047800f90fb200180090000000e00019
:1037700002003a0028009000000c7800ea8f540004
:1037800006003a00380090000078a30003003a00d9
:1037900088007800d0002000e4ff07009800900027
:1037a00058009000808f50000b0032000100e800ac
:1037b000100498001800780009587800000c780070
:1037c00011c0b3004079240001487800ea8f54000a
:1037d00006003200190037008800780009407800a0
:1037e00019000700800478001400370038009000aa
:1037f0000088a3001100320018019000a80090007a
:10380000480090002ef4070098009000810f5000af
:1038100004003200380090000003b3003004980028
:103820008084eb000000eb0010049800280090005a
:10383000000c7800010037008084eb00090078005c
:103840004f04be00000006000200fa00889fbe0080
:10385000a0ff9f0001047800b1009000810478006f
:103860000904b200020032000000fb0036003700fd
:103870000118a30005003a000103b30031049800c9
:10388000190498000080eb002f00370058009000ca
:103890000000e00006003a004800900012002000fe
:1038a000e680570006f4070019049800240037004a
:1038b000280090000000e00008003a000079240091
:1038c00020049800000c780020002000500498008c
:1038d000100498000130a0003104980018019000f5
:1038e000a800900048009000f5f307002800900021
:1038f000000c78000080eb0010049800180078009d
:10390000aff8970001587800000c78002ff8970066
:10391000ea4f50000a003a00380090000088a300e7
:103920000700320018019000a800900048009000a5
:10393000e3f3070019049800a8009000010c780038
:10394000aff897000100fb004f04be000080fa00b2
:04395000000006006d
:020000040000fa
:0200000401f009
:04000c00fbff0000f6
:020000040000fa
:0200000401f009
:04001000bdff000030
:020000040000fa
:0200000401f009
:040014007fff00006a
:020000040000fa
:0200000401f009
:040018007fff000066
:020000040000fa
:0200000401f009
:04001c00deff000003
:020000040000fa
:100008005c0400009ae7000000e8000066e80000d1
:10001800cce8000032e900005c0400005c04000049
:10002800c4d700005c0400005c04000096d2000005
:100038009cd900005c0400005c04000010d400009f
:100048005c0400005c0400005c040000bcd40000f8
:100058005c0400005c040000ead800005c040000b6
:100068005c0400005c0400005c04000082d800000e
:100078005c0400005c0400005c0400005c040000f8
:10008800a0d900005c0400005c0400005c040000cf
:100098005c0400005c040000d6d500005c0400008d
:1000a8005c0400005c0400005c04000014d4000040
:1000b800a4d900005c0400005c0400005c0400009b
:1000c8005c0400005c0400005c0400005c040000a8
:1000d8005c0400005c0400005c0400005c04000098
:1000e8005c0400005c0400005c0400005c04000088
:1000f8005c040000b4d900007ed800005c04000055
:100108005c04000086d800005c0400005c04000069
:100118005c0400005c0400005c040000dcd6000005
:1001280050d70000a8d90000aed900005c04000038
:100138005c0400005c0400005c0400005c04000037
:100148005c0400005c0400005c0400005c04000027
:100158005c0400005c0400005c0400005c04000017
:100168005c0400005c0400005c0400005c04000007
:100178005c0400005c0400005c0400005c040000f7
:100188005c0400005c0400005c0400005c040000e7
:100198005c0400005c0400005c0400005c040000d7
:1001a8005c0400005c0400005c0400005c040000c7
:1001b8005c0400005c0400005c0400005c040000b7
:1001c8005c0400005c0400005c0400005c040000a7
:1001d8005c0400005c0400005c0400005c04000097
:1001e8005c0400005c0400005c0400005c04000087
:0801f8005c0400005c0400003f
:020000040000fa
:100208005c04000098e90000fee9000064ea0000d0
:10021800caea000030eb00005c0400005c04000047
:10022800c4d700005c0400005c04000096d2000003
:100238009cd900005c0400005c04000010d400009d
:100248005c0400005c0400005c040000bcd40000f6
:100258005c0400005c040000ead800005c040000b4
:100268005c0400005c0400005c04000082d800000c
:100278005c0400005c0400005c0400005c040000f6
:10028800a0d900005c0400005c0400005c040000cd
:100298005c0400005c040000d6d500005c0400008b
:1002a8005c0400005c0400005c04000014d400003e
:1002b800a4d900005c0400005c0400005c04000099
:1002c8005c0400005c0400005c0400005c040000a6
:1002d8005c0400005c0400005c0400005c04000096
:1002e8005c0400005c0400005c0400005c04000086
:1002f8005c040000b4d900007ed800005c04000053
:100308005c04000086d800005c0400005c04000067
:100318005c0400005c0400005c040000dcd6000003
:1003280050d70000a8d90000aed900005c04000036
:100338005c0400005c0400005c0400005c04000035
:100348005c0400005c0400005c0400005c04000025
:100358005c0400005c0400005c0400005c04000015
:100368005c0400005c0400005c0400005c04000005
:100378005c0400005c0400005c0400005c040000f5
:100388005c0400005c0400005c0400005c040000e5
:100398005c0400005c0400005c0400005c040000d5
:1003a8005c0400005c0400005c0400005c040000c5
:1003b8005c0400005c0400005c0400005c040000b5
:1003c8005c0400005c0400005c0400005c040000a5
:1003d8005c0400005c0400005c0400005c04000095
:1003e8005c0400005c0400005c0400005c04000085
:0803f8005c0400005c0400003d
:020000040000fa
:10395400414300004b000000414300004c000000c4
:10396400435200004e000000435300005400000086
:103974004342000052000000435200005200000085
:103984004352000053000000434300004100000084
:103994004352000054000000434300005200000062
:1039a400434200005400000043470000540000005c
:1039b400434200005a000000434c00005200000043
:1039c400435400004c000000435400005200000027
:1039d4004354000042000000434f00005400000024
:1039e400434c000046000000534900004e00000014
:1039f400534f0000540000005343000041000000f6
:103a040053460000520000005353000048000000d9
:103a1400535300004d000000535300004c000000bd
:103a240053530000530000005352000053000000a1
:103a3400534b00004e000000535000004b000000a8
:103a4400535000004d000000535000004c00000093
:103a54005350000053000000534900004b00000085
:103a6400534900004d000000534900004c00000081
:103a74005349000053000000534400004b00000071
:103a8400534400004d000000534400004c0000006b
:103a94005344000053000000535300004b00000047
:103aa400534300004b000000535400005400000036
:103ab4005353000049000000534d0000440000002f
:103ac4005353000043000000534100004400000031
:103ad400535000004e000000534300004800000013
:103ae40053440000590000005347000053000000f5
:103af40053470000540000005343000054000000ea
:103b04005353000054000000534c000042000000d6
:103b140053540000440000005346000053000000ca
:103b240052460000520000005253000048000000ba
:103b3400525300004d000000525300004c0000009e
:103b44005253000053000000525200005300000082
:103b5400525000004b000000525000004d00000085
:103b6400525000004c00000052500000530000006e
:103b7400524900004b000000524900004d00000073
:103b8400524900004c00000052490000530000005c
:103b9400524400004b000000524400004d0000005d
:103ba400524400004c000000524400005300000046
:103bb400525300004b000000524300004b00000031
:103bc4005254000054000000525300004900000009
:103bd400524d000044000000525300004300000016
:103be400524c000042000000524400005900000002
:103bf40052470000530000005241000044000000fe
:103c0400525000004e0000005243000048000000e3
:103c140052420000560000005246000047000000d7
:103c240052520000470000005244000043000000cc
:103c340052470000540000005245000049000000b3
:103c4400525400004700000052410000530000009d
:103c54005256000053000000525300005700000069
:103c6400524300005400000052530000540000006e
:103c7400525400004400000052430000460000007b
:103c8400022500003034000064520000434c000060
:103c94002530000034640000303000003030000073
:103ca400000d00002048000049470000203d0000ae
:103cb4002000000025640000000d0000204d0000dd
:103cc40049440000203d0000200000000d200000b9
:103cd4004c4f0000572000003d200000000d000064
:103ce4002053000054500000203d0000200000003c
:103cf4000d200000524f0000542000003d20000021
:103d0400000d0000000d0000205000004944000098
:103d14002e4b0000703d0000200000002534000000
:103d2400642c000025340000642c000025340000bd
:103d3400642c000025340000642c00005b25000086
:103d4400346400005d0000000d20000050490000b4
:103d5400442e00004b6900003d200000000d0000cf
:103d640020500000494400002e4b0000643d000038
:103d7400200000000d20000041470000565f0000b5
:103d84005350000045450000443d00002000000061
:103d940025630000000d000020730000657400001e
:103da4005f53000050450000454400003d200000e2
:103db400000d000020530000544f0000502000006c
:103dc400434e0000535400003d200000000d00004d
:103dd40020530000544f000050200000494e0000c2
:103de400545600003d200000000d0000204d00004e
:103df4004c540000206400004d56000020200000b8
:103e04003d200000000d0000205000004944000047
:103e140020430000545200004c2000003d200000cc
:103e2400000d0000204c00004f570000204200000d
:103e340041540000542000003d200000000d00000b
:103e4400205200004f54000020530000434f000054
:103e5400504500003d200000000d000020440000fb
:103e640049520000203d000020000000464f0000a1
:103e7400525700004152000044200000004200005c
:103e8400414300004b570000415200004400000031
:103e94000d20000042520000414e00004348000043
:103ea400202000003d200000004c0000454600009a
:103eb400540000005249000047480000540000002c
:103ec4005354000052410000494700004854000088
:103ed400000d00000d0d0000000d0000203e00004c
:103ee4003e2000004147000056200000464c0000e0
:103ef4004147000020530000544100005455000085
:103f0400532000003c3c0000200d0000000d000088
:103f140020650000727200006f7200005f430000b1
:103f2400525300005f520000462000002020000091
:103f340020200000203d000020000000310000008f
:103f4400300000000d20000065720000726f000058
:103f5400725f000043480000475f000052460000c3
:103f64002020000020200000202000003d20000030
:103f7400000d000020650000727200006f720000e6
:103f84005f470000415400005f52000046200000db
:103f94002020000020200000203d00002000000020
:103fa4000d20000065720000726f0000725f000057
:103fb400425500005a5a00004552000020200000db
:103fc40020200000202000003d200000000d000003
:103fd40020650000727200006f7200005f4c0000e8
:103fe40044430000454d000047200000202000000d
:103ff40020200000203d0000200000000d200000d3
:1040040065720000726f0000725f00004c44000093
:10401400434f0000435200002020000020200000f5
:10402400202000003d200000000d0000206500005d
:10403400727200006f7200005f4c00004443000085
:10404400544f0000562000002020000020200000d3
:10405400203d0000200000000d20000065720000db
:10406400726f0000725f0000535900005354000047
:10407400454d0000202000002020000020200000ea
:104084003d200000000d0000206500007272000059
:104094006f7200005f47000041540000454f00006c
:1040a400555400002020000020200000203d000086
:1040b400200000000d20000065720000726f0000f7
:1040c400725f00005452000041430000452000008c
:1040d4002020000020200000202000003d200000bf
:1040e400000d000020650000727200006f72000075
:1040f4005f430000484700005f5000005320000069
:104104002020000020200000203d000020000000ae
:104114000d20000065720000726f0000725f0000e5
:1041240043480000415200004745000020200000a1
:1041340020200000202000003d200000000d000091
:1041440020650000727200006f7200005f4f000073
:104154004352000020200000202000002020000006
:1041640020200000203d0000200000000d20000061
:1041740065720000726f0000725f0000454d000020
:104184004720000020200000202000002020000004
:10419400202000003d200000000d000020660000eb
:1041a4006c610000675f0000525500004e20000063
:1041b40020200000202000002020000020200000fb
:1041c400203d0000200000000d200000666c00006f
:1041d400616700005f530000544f0000502000004e
:1041e40020200000202000002020000020200000cb
:1041f4003d200000000d0000206600006c610000fe
:10420400675f0000736c00006f7700005354000078
:104214004f5000002020000020200000203d00001e
:10422400200000000d200000666c000061670000a3
:104234005f430000524f000053530000544f0000ee
:104244005020000020200000202000003d2000001d
:10425400000d0000206600006c610000675f000034
:10426400435200004f530000535f0000494e0000ca
:104274002020000020200000203d0000200000003d
:104284000d200000666c0000616700005f500000b4
:1042940042530000535400004f50000020200000ff
:1042a40020200000202000003d200000000d000020
:1042b400206600006c610000675f00004f42000050
:1042c40053540000414300004c45000020200000ee
:1042d40020200000203d0000200000000d200000f0
:1042e400666c0000616700005f7200006566000094
:1042f4007573000065500000425300002020000048
:10430400202000003d200000000d00002066000079
:104314006c610000675f00005245000053540000c8
:104324004152000054200000202000002020000002
:10433400203d0000200000000d200000666c0000fd
:10434400616700005f6300006e7400005245000066
:10435400535400004152000054200000202000006b
:104364003d200000000d0000206600006c6100008c
:10437400675f0000434800004152000047490000c5
:104384004e4700002020000020200000203d0000b7
:10439400200000000d200000636e0000745f000028
:1043a40043480000415200004745000054490000c2
:1043b4004d45000020200000202000003d2000008a
:1043c400000d0000206600006c610000675f0000c3
:1043d4004d410000524b0000535400004f50000068
:1043e4002020000020200000203d000020000000cc
:1043f4000d200000666c0000616700005f6400002f
:104404007269000076540000555200004e200000ee
:1044140020200000202000003d200000000d0000ae
:10442400206600006c610000675f00004d410000e1
:10443400524b000054550000524e00002020000052
:1044440020200000203d0000200000000225000084
:104454003034000064530000415300002c25000058
:1044640030340000582c000025300000345800007f
:104474002c25000030340000582c000025300000aa
:10448400345800002c25000030340000580000008f
:104494000d20000042410000545400004552000029
:1044a40059200000564f00004c2000003d20000021
:1044b40000250000362e000031660000000d0000cb
:1044c40020460000524f00004e54000020470000d8
:1044d4004453000056200000203d0000200000004e
:1044e400253600002e320000660000000d2000007a
:1044f400465200004f4e000054200000412f00009f
:1045040044200000202000003d2000000025000081
:1045140036640000000d000020460000524f0000e9
:104524004e54000020430000545600002020000098
:10453400203d0000200000000d2000004652000035
:104544004f4e000054200000474100005445000035
:10455400202000003d20000000200000205b00001f
:10456400204f00004e5d0000002000005b4f000063
:10457400464600005d0000000d200000524500008a
:104584004152000020200000474400005356000020
:10459400202000003d200000000d000020520000fb
:1045a4004541000052200000204100002f4400003b
:1045b40020200000203d0000200000000d2000000d
:1045c40052450000415200002020000043540000e6
:1045d40056200000202000003d200000000d0000b7
:1045e40020520000454100005220000020470000f6
:1045f4004154000045200000203d00002000000040
:1046040002250000303400006453000042560000cc
:104614002530000034640000000200002530000052
:104624003464000053460000472500003034000085
:1046340064000000022500003034000064530000d0
:1046440052470000253000003464000000020000de
:104654002530000034640000535300005725000047
:1046640030340000580000000d20000044490000d0
:10467400505f000053570000313d0000000d000062
:1046840020440000495000005f53000057320000ee
:104694003d0000000d20000044490000505f000070
:1046a40053570000333d0000000d0000204400007b
:1046b400495000005f530000573400003d000000e3
:1046c4000d20000044490000505f000053570000d3
:1046d400353d0000000d000020440000495000005a
:1046e4005f530000573600003d0000000d2000001d
:1046f40044490000505f000053570000373d00005c
:10470400000d000020440000495000005f530000e9
:10471400573800003d0000000d20000045580000ff
:1047240054450000524e0000414c00002049000056
:104734004e500000555400000d0000000d200000f4
:104744005b440000494f0000315d0000000d000093
:1047540020440000494e0000503100002e63000048
:1047640068310000200000005b3100005d000000a3
:104774005b3000005d0000000d2000004449000093
:104784004e500000312e000063680000322000000b
:10479400000d000020440000494e0000503100008c
:1047a4002e63000068330000200000000d2000008c
:1047b400444900004e500000312e000063680000a0
:1047c40034200000000d000020440000494e000089
:1047d400503100002e630000683500002000000006
:1047e4000d200000444900004e500000312e00000e
:1047f4006368000036200000000d00002044000023
:10480400494e0000503100002e630000683700005c
:10481400200000000d200000444900004e5000001c
:10482400312e00006368000038200000000d0000f5
:1048340020440000494e0000503100002e63000067
:1048440068390000200000000d20000044490000e9
:104854004e500000312e000063680000313000002b
:10486400000d000020440000494e000050310000bb
:104874002e63000068310000310000000d200000ac
:10488400444900004e500000312e000063680000cf
:1048940031320000000d0000205b0000444900009c
:1048a4004f3200005d0000000d200000444900006c
:1048b4004e500000322e00006368000031200000da
:1048c400000d000020440000494e0000503200005a
:1048d4002e63000068320000200000000d2000005c
:1048e400444900004e500000322e0000636800006e
:1048f40033200000000d000020440000494e000059
:10490400503200002e6300006834000020000000d4
:104914000d200000444900004e500000322e0000db
:104924006368000035200000000d000020440000f2
:10493400494e0000503200002e630000683600002b
:10494400200000000d200000444900004e500000eb
:10495400322e00006368000037200000000d0000c4
:1049640020440000494e0000503200002e63000035
:1049740068380000200000000d20000044490000b9
:104984004e500000322e0000636800003920000001
:10499400000d000020440000494e00005032000089
:1049a4002e63000068310000300000000d2000007c
:1049b400444900004e500000322e0000636800009d
:1049c40031310000000d000020440000494e000079
:1049d400503200002e6300006831000032000000f5
:1049e40002250000303400006453000045490000f3
:1049f400253000003458000000020000253000007b
:104a040034640000544100004725000030360000a3
:104a14006c640000000200004343000041250000d4
:104a240030340000642500003034000064000000cd
:104a34000d200000494e00003d25000030340000e8
:104a4400580000000d2000004f550000543d0000a8
:104a540025300000325800000002000043430000eb
:104a6400412500003034000064250000303200008d
:104a740058000000022500003034000064410000aa
:104a8400434b0000253000003464000000020000a5
:104a940025300000346400004e4100004b25000026
:104aa400303400006400000025300000346400004d
:104ab400000200002530000034640000414300007f
:104ac4004725000030340000642500003034000025
:104ad400580000004e6f00006e6500002d45000078
:104ae4007869000073740000656e0000636500005f
:104af400204300006f6d00006d6100006e640000d3
:104b04002e2e00002e210000004900006e760000c9
:104b1400616c000069640000204f000070740000a4
:104b2400696f00006e200000566100006c75000083
:104b3400652e00002e2e00002100000043520000cc
:104b44004e000000435300005400000043420000a4
:104b5400520000004343000052000000434c000098
:104b640053000000434c0000410000004342000099
:104b7400540000004347000054000000434200007a
:104b84005a000000434800004d000000435200005a
:104b940054000000435400004c0000004354000043
:104ba400520000004354000042000000435400003f
:104bb40047000000434c0000520000004343000043
:104bc400440000004343000047000000434300004a
:104bd400410000004352000053000000434f000016
:104be40054000000434c0000460000005246000000
:104bf40052000000525300004800000052530000cd
:104c04004d000000525300004c00000052530000bd
:104c140053000000525200005300000052500000a4
:104c24004b000000525000004d00000052500000a4
:104c34004c00000052500000530000005249000094
:104c44004b000000524900004d0000005249000092
:104c54004c00000052490000530000005244000080
:104c64004b000000524400004d000000524400007c
:104c74004c00000052440000530000005253000056
:104c84004b000000524300004b000000525400004f
:104c9400540000005253000049000000524d00002f
:104ca4004400000052530000430000005241000041
:104cb40044000000525000004e0000005243000027
:104cc40048000000524c0000420000005244000022
:104cd40059000000524700005300000052470000f2
:104ce40054000000524300005400000052530000de
:104cf40054000000525400004400000052560000ca
:104d040053000000534600005200000053530000bb
:104d140048000000535300004d00000053530000ae
:104d24004c00000053530000530000005352000095
:104d340053000000535000004b000000535000008b
:104d44004d000000535000004c0000005350000080
:104d540053000000534900004b0000005349000079
:104d64004d000000534900004c000000534900006e
:104d740053000000534400004b0000005344000063
:104d84004d000000534400004c0000005344000058
:104d940053000000535300004b0000005343000035
:104da4004b00000053540000540000005353000013
:104db40049000000534d000044000000535300001c
:104dc4004300000053410000440000005350000021
:104dd4004e0000005343000048000000534c000004
:104de40042000000534400005900000053470000f3
:104df40053000000534700005400000053430000d8
:104e040054000000535300005400000053540000a9
:104e140044000000534d00004900000053460000c8
:104e240053000000415400004d5900002558000073
:104e34000d000000415400004944000025300000ea
:104e4400345800000d0000004154000043480000a5
:104e540025300000345800000d00000043520000cb
:104e64004f530000532d000049440000204e000021
:104e74004f4e0000452e00002e2e000021000000a1
:104e84000225000030340000644300004352000057
:104e94002530000034640000256300002530000044
:104ea400326400002530000031640000000200007c
:104eb4002530000034640000434c0000412500000c
:104ec4003034000064300000303000003000000056
:104ed4005345000043540000204e00004f200000c2
:104ee40045520000524f0000522e00002e2e0000aa
:104ef400210000000225000030340000644300005b
:104f04004c530000253000003464000025300000bc
:104f14003464000000430000524f0000535300006b
:104f24002d4900004420000045520000524f00006b
:104f3400522e00002e2e0000210000000225000049
:104f44003034000064410000475400002530000064
:104f54003464000030250000633000002563000045
:104f640000020000253000003464000041420000cb
:104f74005a2500003034000064300000256300002e
:104f840030250000630000000225000030340000da
:104f940064430000484d00002530000034640000e4
:104fa40025630000303000003030000000020000b3
:104fb40025300000346400005355000042250000f1
:104fc40030340000643000003030000025630000fd
:104fd400000200002530000034640000524d00003f
:104fe40056250000303400006430000030300000ea
:104ff4002563000000020000253000003464000036
:1050040043420000542500003034000064250000b1
:105014006325000030340000640000000225000015
:105024003034000064520000434100002530000089
:105034003464000030300000303000000002000012
:105044002530000034640000434300004125000083
:105054003034000064250000303400006400000097
:1050640025300000366c000064000000024100009e
:10507400434b000043540000474100004403000038
:1050840000440000494f0000256300003a3000004e
:105094005825000030320000580d00000055000073
:1050a40050000000444e0000004f00004e0000007d
:1050b4004f46000046000000524500005300000027
:1050c40053540000500000005245000051000000fd
:1050d4000d2000004c490000465400005f550000bc
:1050e400505f0000535400004f5000002d0000009a
:1050f4005b3100005d0000005b3000005d000000db
:105104000d2000004c490000465400005f4400009c
:105114004e5f0000535400004f5000002d0000006b
:105124000d2000004c490000465400005f5500006b
:10513400504c0000494d0000495400002d0000006f
:105144000d2000004c490000465400005f4400005c
:105154004e4c0000494d0000495400002d00000051
:105164000d2000004c490000465400005f4500003b
:10517400525200005f550000502000002d00000036
:105184000d2000004c490000465400005f4500001b
:10519400525200005f4400004e2000002d00000029
:1051a4000d2000004c490000465400005f450000fb
:1051b4004d47000020200000202000002d000000aa
:1051c4000d2000004c490000465400005f4f0000d1
:1051d4004352000020200000202000002d00000089
:1051e4000d2000004c490000465400005f540000ac
:1051f4004f56000020200000202000002d00000059
:105204000d2000004c490000465400005f5200008d
:10521400554e000020200000202000002d0000003a
:105224000d2000004c490000465400005f4500007a
:105234004e4400005f550000502000002d00000087
:105244000d2000004c490000465400005f4500005a
:105254004e4400005f4400004e2000002d0000007a
:105264000225000030340000645300004652000060
:1052740025300000345800000002000025300000f2
:10528400346400005353000048250000303400000b
:105294006400000002250000303400006453000064
:1052a400534d00002530000034640000000200006b
:1052b4002530000034640000535300004c250000e6
:1052c4003034000064000000022500003034000087
:1052d4006453000053530000253000003464000080
:1052e4000002000025300000346400005352000026
:1052f4005325000030340000640000000225000043
:105304003034000064530000504b0000253000008e
:105314003464000000020000253000003464000002
:10532400535000004d25000030340000640000009c
:10533400022500003034000064530000504c00008b
:105344002530000034640000000200002530000015
:105354003464000053500000532500003034000032
:105364006400000002250000303400006453000093
:10537400494b0000253000003464000000020000a6
:105384002530000034640000534900004d2500001e
:1053940030340000640000000225000030340000b6
:1053a40064530000494c00002530000034640000c0
:1053b400000200002530000034640000534900005e
:1053c4005325000030340000640000000225000072
:1053d4003034000064530000444b000025300000ca
:1053e4003464000000020000253000003464000032
:1053f400534400004d2500003034000064000000d8
:10540400022500003034000064530000444c0000c6
:105414002530000034640000000200002530000044
:10542400346400005344000053250000303400006d
:1054340064000000022500003034000064530000c2
:10544400534b0000253000003464000000020000cb
:105454002530000034640000534300004b25000055
:1054640030340000640000000225000030340000e5
:1054740064530000545400002530000034640000dc
:105484000002000025300000346400005353000083
:1054940049250000303400006400000002250000ab
:1054a40030340000645300004d44000025300000f7
:1054b4003464000000020000253000003464000061
:1054c4005353000043250000303400006400000002
:1054d40002250000303400006453000056530000dd
:1054e4002530000034640000000200002530000074
:1054f40034640000534c00004225000030340000a6
:1055040064000000022500003034000064530000f1
:1055140044590000253000003464000000020000fb
:105524002530000034640000534700005325000078
:105534003034000064000000022500003034000014
:105544006453000047540000253000003464000018
:1055540000020000253000003464000053430000c2
:1055640054250000303400006400000002250000cf
:105574003034000064530000535400002530000010
:105584003464000000020000253000003464000090
:10559400535400004425000030340000640000002f
:1055a4000225000030340000645300004144000030
:1055b40025300000346400000002000025300000a3
:1055c40034640000535000004e25000030340000c5
:1055d400580000000225000030340000645300002d
:1055e4004348000025300000345800000025000026
:1055f40030340000640000004d54000025300000e9
:10560400366c000064000000434800004152000072
:1056140047450000522000006164000064720000ed
:10562400657300007320000065720000726f000053
:10563400722e00002e2e0000210000000241000006
:10564400434b0000004e00006f6e0000652d00000b
:105654004578000069730000746500006e63000003
:1056640065200000436f00006d6d0000616e000056
:10567400642e00002e2e000021000000496e000060
:10568400766100006c690000642000004f70000027
:10569400746900006f6e000020560000616c000009
:1056a400756500002e2e00002e210000004c000025
:1056b4005400000052540000004d0000530000004c
:1056c4004653000000420000530000003030000048
:1056d400004600004c00000046520000004200005a
:1056e4004c00000042520000004800005500000039
:1056f40048440000000000002d530000454c000009
:105704005f4c000046540000002d0000534500008b
:105714004c5f000052490000540000002d5300006b
:10572400454c00005f530000545200000044000048
:10573400494f0000312000006469000073430000f9
:105744004f4e00004e45000043540000004400004a
:10575400494f0000322000006469000073430000d8
:105764004f4e00004e45000043540000004c000022
:10577400494600005420000064690000734300009f
:105784004f4e00004e4500004354000000520000fc
:10579400464900004420000064690000734300008f
:1057a4004f4e00004e45000043540000004d0000e1
:1057b40036450000204d00002f440000204e00001c
:1057c400470000004c4f00005720000042410000f9
:1057d4005454000045520000590000004652000095
:1057e4004f4e0000545f0000504200005320000060
:1057f40045520000524f0000520000005245000084
:10580400415200005f50000042530000202000007d
:1058140045520000524f0000520000004c45000069
:10582400465400005f55000053540000202000003f
:1058340045520000524f000052000000524900003f
:1058440047480000545f00005553000054200000f6
:1058540045520000524f00005200000073650000e2
:10586400745f0000535000004545000044200000d0
:105874005b4800005d00000073650000745f000079
:105884005350000045450000442000005b4d0000db
:105894005d00000073650000745f00005350000059
:1058a40045450000442000005b4c00005d00000002
:1058b40073650000745f000053500000454500000c
:1058c400442000005b5300005d0000002420000021
:1058d4005b450000525200005d2000004e4f000066
:1058e4002047000041540000454f0000555400007b
:1058f4002e2e00002e21000000240000205b00005a
:1059040045520000525d0000204500004d45000056
:1059140052470000454e0000435900002e2e00005f
:105924002e210000000d00000d2000003e3e00006e
:1059340020410000475600005f5600003335000048
:10594400305f00004c460000203100002e30000083
:105954002e3100002832000030320000352f0000c4
:10596400303100002f31000030290000000d00000c
:105974000d20000041470000562000004144000073
:10598400445200003d5b00002530000032640000fa
:105994005d2000000d00000024200000726500005e
:1059a400735f000042410000434b00005f5400005d
:1059b400555200004e2e00002e2e00002100000043
:1059c40052450000533d0000256400000020000003
:1059d40042410000543d000000250000362e000026
:1059e400326600002c2000002530000034640000e2
:1059f4000064000072690000766900006e670000b0
:105a0400205300004c4f0000572000005354000066
:105a14004f5000002e2e00002e2e0000210000000a
:105a24007365000061720000636800005f7200002b
:105a3400616900006c200000544900004d450000dd
:105a4400204f000056450000522e00002e21000079
:105a5400000d000020470000445300003d250000d5
:105a64003037000064200000004500004d45000070
:105a740052470000454e0000435900002e2e0000fe
:105a8400210000004f56000045520000435500001d
:105a940052520000454e0000542e00002e210000fa
:105aa400007200006f740000617400006520000043
:105ab400534c00004f5700005f530000544f000048
:105ac400502e00002e2e00002e2100000047000062
:105ad40041540000455f00004f460000462e000080
:105ae4002e210000005300004541000052430000f5
:105af4004820000052410000494c00002e2e0000b6
:105b04002e210000005b000041470000565f0000aa
:105b140062610000636b00005f5400005552000096
:105b24004e5d0000200d00000041000047560000bb
:105b340020520000452d0000535400004152000043
:105b44005420000045520000524f0000522e000025
:105b54002e2e0000210000002420000041470000f8
:105b640056200000525500004e2e00002e2e00003c
:105b740021000000242000004147000056200000be
:105b8400535400004f5000002e2e00002e21000020
:105b94000024000020410000475600005f6c000014
:105ba40065660000745f000054550000524e00000a
:105bb4000024000020410000475600005f720000ee
:105bc40069670000687400005f54000055520000cb
:105bd4004e00000024200000414700005620000031
:105be4004d410000524b00002d540000555200005e
:105bf4004e2000004f4b00002e2e00002e2e0000e1
:105c0400210000002420000041470000562000002d
:105c14004d410000524b00002d540000555200002d
:105c24004e200000535400004f5000002e2e000060
:105c34002e2e000021000000242000004147000017
:105c4400562000004d410000524b00002d5400002e
:105c5400555200004e20000045520000524f0000f3
:105c6400522e00002e2e00002e210000005b0000aa
:105c740041470000565f00006c6500006674000038
:105c84005f540000555200004e5d0000200d0000de
:105c9400002400002041000047560000204c000072
:105ca40045460000542d000054550000524e00009b
:105cb400204f00004b2e00002e2e00002e2100004d
:105cc400002400002041000047560000204c000042
:105cd40045460000542d000054550000524e00006b
:105ce40020530000544f0000502e00002e2e0000c0
:105cf4002e2100000024000020410000475600002f
:105d0400204c000045460000542d0000545500006e
:105d1400524e000020450000525200004f52000035
:105d24002e2e00002e2e0000210000005b410000fa
:105d3400475600005f720000696700006874000045
:105d44005f540000555200004e5d0000200d00001d
:105d540000240000204100004756000020520000ab
:105d640049470000485400002d54000055520000db
:105d74004e2000004f4b00002e2e00002e2e00005f
:105d840021000000242000004147000056200000ac
:105d94005249000047480000542d000054550000ab
:105da400524e000020530000544f0000502e0000bb
:105db4002e2e00002e2100000024000020410000af
:105dc4004756000020520000494700004854000094
:105dd4002d540000555200004e2000004552000092
:105de400524f0000522e00002e2e00002e210000e3
:105df400000000000d0d00000d2000005b500000ad
:105e04004f5700002d4f00004e5d0000207300002e
:105e1400657400005f5200004c5900005f430000ad
:105e24004841000052470000450000000d200000da
:105e34004241000054560000203d000020000000b4
:105e44005b250000372e0000326600005d5b000019
:105e540025350000645d0000002e00002e2e000099
:105e64002e2e00005b4f00004b5d0000002e000052
:105e74002e2e00002e2e00005b4e0000475d000019
:105e840000200000415400005f4300004d44000026
:105e94002e2e00002e2e00006f6b0000004100002b
:105ea4005443000048250000580d00000020000065
:105eb40043480000202e00002e2e00002e2e00004d
:105ec4002e2e00006f6b00000041000054490000ba
:105ed40044250000580d0000002000004944000043
:105ee400202e00002e2e00002e2e00002e2e00004c
:105ef4006f6b000000410000544d00005925000064
:105f0400580d0000002000004d590000205b0000e7
:105f140041440000445200005d2e00006f6b0000fd
:105f240000200000444c0000205b0000305d0000b5
:105f34002e2e00002e2e00006f6b000000200000ab
:105f440041540000575200002e2e00002e2e000057
:105f54002e2e00006f6b0000004c00006f610000eb
:105f6400642000004465000066610000756c000058
:105f740074200000566100006c750000650000008c
:105f84000d0000000d2000006641000044430000a5
:105f9400203d0000200000005b250000362e00009c
:105fa400316600005d0000000d200000664700001f
:105fb40044530000203d0000200000005b25000049
:105fc400362e0000326600005d0000000d20000047
:105fd4007241000044430000203d00002000000006
:105fe4000d2000007247000044530000203d0000d3
:105ff400200000000d200000524600002d49000042
:1060040044200000202000003d0000002063000028
:106014006f6e00006e65000063740000656400002c
:106024000020000064690000735f0000636f0000db
:106034006e6e00006563000074650000640000007b
:106044000d20000045450000505200004f4d000057
:10605400202000003d00000020320000354c0000ec
:1060640043310000363000005f4f00004b21000038
:1060740000200000323500004c430000313600009f
:10608400305f00004e470000210000000d2000009a
:1060940045580000545f0000444900004f3100009f
:1060a4003d0000000d20000045580000545f000032
:1060b400444900004f3200003d000000242000004d
:1060c40041470000562000004c4f0000572d0000af
:1060d40042410000545400002e2e00002e2e0000d9
:1060e4002e2100000d000000242000004652000074
:1060f4004f4e00005420000047440000532000008d
:1061040045520000524f0000522e00002e21000084
:106114000d00000024200000524500004152000000
:106124002047000044530000204500005252000064
:106134004f5200002e2e00002e2100000d00000002
:10614400242000004d360000652000004d2f000083
:106154004420000045520000524f0000522e00001f
:106164002e2e00002e2100000d000000242000002f
:1061740052460000494400002044000049530000f6
:10618400434f00004e4e000045430000542e0000d3
:106194002e2100000d0000002420000045450000d1
:1061a400505200004f4d00002045000052520000a4
:1061b4004f5200002e2e00002e2e00002e21000033
:1061c4000d00000024200000444900004f3100006d
:1061d4002044000049530000434f00004e4e00008d
:1061e40045430000542e00002e2100000d00000045
:1061f40024200000444900004f32000020440000e5
:1062040049530000434f00004e4e00004543000038
:10621400542e00002e2100000d0000002420000058
:106224004c4900004654000020440000495300003b
:10623400434f00004e4e000045430000542e000022
:106244002e2100000d00000020660000726f000087
:106254006e740000200000002072000065610000e0
:106264007220000000470000445300005b2500003a
:10627400362e0000316600005d2c0000434500000e
:106284004e5b0000253600002e310000665d0000e4
:10629400002000004f2000000d00000020580000e6
:1062a400200d000000200000444900004f31000090
:1062b4003d5b000025300000345800003a25000002
:1062c40030320000585d00000d0000002044000042
:1062d400494f0000323d00005b25000030340000cf
:1062e400583a000025300000325800005d0d0000cf
:1062f400002000004c490000465400003d5b0000b3
:1063040025300000345800003a25000030320000e7
:10631400585d00000d000000636c0000725f000017
:106324006c690000667400005f4300004f4e00007b
:10633400545200004f4c00002e2e00002e2100006d
:10634400006900006e690000745f00006c69000061
:10635400667400005f4300004f4e0000545200007a
:106364004f4c00002e2e00002e2100000073000070
:10637400746f0000705f00006c69000066740000b8
:106384005f4300004f4e0000545200004f4c000089
:106394002e2e00002e21000000450000584500006c
:1063a4005f4c000049460000545f00005550000057
:1063b400282900002e2e00002e210000004c000091
:1063c40049460000542000005550000020540000ad
:1063d400494d0000454f000056450000522e000074
:1063e4002e2e0000210000004c49000046540000fd
:1063f400204f000056450000524300005552000053
:10640400524500004e5400002e2e00002e210000a4
:10641400004c00004946000054200000454d000097
:1064240045520000474500004e430000592e00002d
:106434002e2e00002e2e00002100000045580000e2
:10644400455f00004c490000465400005f440000d2
:106454004f5700004e280000292e00002e2e000069
:10646400210000004c490000465400002044000074
:106474004e200000544900004d4500004f560000d6
:10648400455200002e2e00002e21000000000000c6
:106494002530000034580000000d00000d200000dd
:1064a40041470000565b000025320000645d000097
:1064b400200000002b2b00002b00000041540000a2
:1064c400575200002c4300004e0d00000002000053
:1064d400534c0000443000003030000025630000bd
:1064e40000740000726100006e7300006d690000aa
:1064f400742000007265000073650000740d0000d4
:1065040000020000535200005230000030300000fe
:1065140030000000025300005453000025300000f6
:10652400336400002530000034580000253000009a
:1065340034580000253000003458000000250000c5
:106544006325000063250000632500006325000027
:106554003032000058250000303300006400000091
:106564000d2000005f460000414c00005441000033
:10657400204900006e74000065720000727500000e
:10658400707400002e2e00002e2e00002e2100001c
:10659400000d0000205f0000464100004c54000044
:1065a40042200000496e0000746500007272000011
:1065b40075700000742e00002e2e00002e2e000098
:1065c40021000000494e0000542000004d4100000d
:1065d400524b00002d530000544f0000502e000079
:1065e4002e2e00002e2e000021000000494e000037
:1065f400542000004d410000524b00002d54000077
:10660400555200004e2e00002e2e00002e2e0000ab
:106614002100000002540000414700002530000022
:10662400366c0000640000004e4f0000573a000032
:106634004d410000524b00005b250000366c000009
:10664400643a0000253600006c6400005d00000020
:1066540072650000735f00004d410000524b000062
:10666400535400004f5000002e2e00002e21000035
:1066740000720000657300005f4d0000415200008d
:106684004b540000555200004e2e00002e2e0000e8
:106694002100000072650000735f00006d7200004d
:1066a4006b4400004952000043480000472e00009c
:0866b4002e210000000000008f
:020000040000fa
:1066bc00889fbe0000047800ea48070080447800f8
:1066cc000884e80008007800e6480700c848dd00a8
:1066dc000080fb00008070000080ea006a34b60085
:1066ec006a14e20003003200100020004f04be00c8
:1066fc00000006005c94a8005cb4a9005cd4a9005e
:10670c005cf4a9005a54a800ab54070010002000f8
:10671c004f04be0000000600f6ff3700889fbe0045
:10672c00000478000000e800ce48070080447800a0
:10673c0063004400cb480700d7180700090032005b
:10674c0050c3b30080cf50001e00320090c3b30082
:10675c0080cf500012003200100020004f04be0009
:10676c00000006000280ea006a34b6006a14e200f7
:10677c00f9ff3a00cb82a8005c94a8005cb4a90095
:10678c005cd4a9005cf4a9005a54a8008a540700f0
:10679c00100020004f04be0000000600f1ff37007f
:1067ac000280ea006634b60031a38000200e20007f
:1067bc000e300700100020004f04be000000060041
:1067cc00e8ff37000280ea006834b60041a380007d
:1067dc00000e200005300700100020004f04be0002
:1067ec0000000600dfff3700889fbe000004780021
:1067fc000000e8009b4807008044780063004400d8
:10680c0098480700a41807000900320050c3b300d1
:10681c0080cf50001500320090c3b30080cf5000e1
:10682c0009003200100020004f04be0000000600da
:10683c00020078006a34b700100020004f04be003c
:10684c0000000600faff3700020078006634b7003b
:10685c0031a38000200e2000e42f07001000200040
:10686c004f04be0000000600f1ff37000200780064
:10687c006834b70041a38000000e2000db2f070016
:10688c00100020004f04be0000000600e8ff370097
:10689c001e00fa0090407800a1e79f009040900005
:1068ac00b1e79f00a0409000c1e79f0030409000ee
:1068bc00d0e79f000040eb00e0e79f007e80570090
:1068cc00c4ed07002919070020062000808f500016
:1068dc000d003e00e0a48000800f51000400320047
:1068ec00e2a48800e1a480000000eb00bf2f0700a9
:1068fc007018070022d82000624078001300200096
:10690c00e14f500003003200030078000080fa00d1
:10691c0000000600cae2a80040062000c09e8800c5
:10692c00e0a48000801f780041712a00811f78004c
:10693c00e0fd2f000f0040008fed0700e0fd2f0061
:10694c000f0040006648070013002000e487570042
:10695c00030078000080fa0000000600edff37000d
:10696c001000fa00889fbe000004780010407800e8
:10697c0064460700cc04dd00184090006146070017
:10698c004800dd0080844400284090005d460700ec
:10699c004d1807005b4607000080fb000084440094
:1069ac00881f7800c0712a00801f780078805700fb
:1069bc0071ed07007880570049480700e4875700bd
:1069cc000004e00004003a00100020004f04be0058
:1069dc000080fa000000060008a4880088007800f7
:1069ec0020062000812f0700100020004f04be005d
:1069fc000080fa0000000600f7ff37001000fa00d4
:106a0c00889fbe0000047800104078003d460700c7
:106a1c00cc04dd00184090003a4607004800dd0029
:106a2c008084440028409000364607002618070052
:106a3c00344607000080fb00008444006c005400c6
:106a4c00eb0f500004003600100020004f04be0075
:106a5c000080fa0000000600881f780060722a008f
:106a6c00801f78007880570043ed0700788057002e
:106a7c001b480700e48757000004e000f2ff3200d7
:106a8c0018a488008800780000062000572f070003
:106a9c00100020004f04be000080fa000000060029
:106aac00edff37000a00fa00881f78000b1807006a
:106abc006c80570047ed07001318070004003600e0
:106acc00010078004f0478000080fa0000000600f6
:106adc008800780060032000442f07006140b90053
:106aec00a6e807000800e0000b00350002002000bb
:106afc00a3472400cde7070020a1880031a188001e
:106b0c0011002000010078004f0478000080fa008a
:106b1c0000000600eeff370002002000037824007e
:106b2c0005e8070002002000a3472400bfe7070088
:106b3c0020a1880031a1880011002000f1ff37004e
:106b4c000a00fa00881f7800e41707006c805700d1
:106b5c0020ed0700ec170700040036000100780058
:106b6c004f0478000080fa000000060088007800ce
:106b7c00c00320001d2f07006140b9007fe807000b
:106b8c000800e0000b00350002002000a3472400a1
:106b9c00a6e7070080a1880091a1880011002000c1
:106bac00010078004f0478000080fa000000060015
:106bbc00eeff37000200200003782400dee7070018
:106bcc0002002000a347240098e7070080a188005a
:106bdc0091a1880011002000f1ff37000a00fa0093
:106bec00881f7800bd1707006c805700f9ec070070
:106bfc00c517070004003600010078004f04780028
:106c0c000080fa00000006008800780020042000b4
:106c1c00f62e07006140b90058e807000800e000b4
:106c2c000b00350002002000a34724007fe707007b
:106c3c00e0a18800f1a1880011002000010078007b
:106c4c004f0478000080fa0000000600eeff3700c9
:106c5c000200200003782400b7e7070002002000a0
:106c6c00a347240071e70700e0a18800f1a1880088
:106c7c0011002000f1ff37000a00fa00881f78008d
:106c8c00961707006c805700d2ec07009e17070080
:106c9c0004003600010078004f0478000080fa00f0
:106cac00000006008800780080042000cf2e07002a
:106cbc006140b90031e807000800e0000b00350026
:106ccc0002002000a347240058e7070040a28800d8
:106cdc0051a2880011002000010078004f047800b8
:106cec000080fa0000000600eeff370002002000d2
:106cfc000378240090e7070002002000a34724003b
:106d0c004ae7070040a2880051a288001100200029
:106d1c00f1ff37000a00fa00881f78006f17070090
:106d2c006c805700abec07007717070004003600a7
:106d3c00010078004f0478000080fa000000060083
:106d4c008800780080032000a82e07006140b9005d
:106d5c000ae807000800e0000b00350002002000e4
:106d6c00a347240031e7070040a1880051a1880007
:106d7c0011002000010078004f0478000080fa0018
:106d8c0000000600eeff370002002000037824000c
:106d9c0069e7070002002000a347240023e707004f
:106dac0040a1880051a1880011002000f1ff37009c
:106dbc000a00fa00881f7800481707006c805700fb
:106dcc0084ec07005017070004003600010078001f
:106ddc004f0478000080fa0000000600880078005c
:106dec00e0032000812e07006140b900e3e70700b3
:106dfc000800e0000b00350002002000a34724002f
:106e0c000ae70700a0a18800b1a1880011002000aa
:106e1c00010078004f0478000080fa0000000600a2
:106e2c00eeff3700020020000378240042e7070041
:106e3c0002002000a3472400fce60700a0a1880064
:106e4c00b1a1880011002000f1ff37000a00fa0000
:106e5c00881f7800211707006c8057005dec070035
:106e6c002917070004003600010078004f04780051
:106e7c000080fa0000000600880078004004200022
:106e8c005a2e07006140b900bce707000800e0007b
:106e9c000b00350002002000a3472400e3e60700a6
:106eac0000a2880011a288001100200001007800c7
:106ebc004f0478000080fa0000000600eeff370057
:106ecc0002002000037824001be7070002002000ca
:106edc00a3472400d5e6070000a2880011a2880071
:106eec0011002000f1ff37000a00fa00881f78001b
:106efc00fa1607006c80570036ec070002170700e3
:106f0c0004003600010078004f0478000080fa007d
:106f1c000000060088007800a0042000332e070033
:106f2c006140b90095e707000800e0000b00350050
:106f3c0002002000a3472400bce6070060a28800e2
:106f4c0071a2880011002000010078004f04780025
:106f5c000080fa0000000600eeff3700020020005f
:106f6c0003782400f4e6070002002000a347240065
:106f7c00aee6070060a2880071a288001100200014
:106f8c00f1ff37000a00fa00881f7800d3160700bb
:106f9c006c8057000fec0700db160700040036006e
:106fac00010078004f0478000080fa000000060011
:106fbc0088007800a00320000c2e07006140b90067
:106fcc006ee707000800e0000b003500020020000f
:106fdc00a347240095e6070060a1880071a18800f2
:106fec0011002000010078004f0478000080fa00a6
:106ffc0000000600eeff370002002000037824009a
:10700c00cde6070002002000a347240087e6070016
:10701c0060a1880071a1880011002000f1ff3700e9
:10702c000a00fa00881f7800ac1607006c80570025
:10703c00e8eb0700b41607000400360001007800e6
:10704c004f0478000080fa000000060088007800e9
:10705c0000042000e52d07006140b90047e7070058
:10706c000800e0000b00350002002000a3472400bc
:10707c006ee60700c0a18800d1a188001100200095
:10708c00010078004f0478000080fa000000060030
:10709c00eeff37000200200003782400a6e607006c
:1070ac0002002000a347240060e60700c0a188006e
:1070bc00d1a1880011002000f1ff37000a00fa006e
:1070cc00881f7800851607006c805700c1eb0700fd
:1070dc008d16070004003600010078004f0478007c
:1070ec000080fa0000000600880078006004200090
:1070fc00be2d07006140b90020e707000800e00042
:10710c000b00350002002000a347240047e60700cf
:10711c0020a2880031a28800110020000100780014
:10712c004f0478000080fa0000000600eeff3700e4
:10713c0002002000037824007fe6070002002000f4
:10714c00a347240039e6070020a2880031a288005a
:10715c0011002000f1ff37000a00fa00881f7800a8
:10716c005e1607006c8057009aeb07006616070046
:10717c0004003600010078004f0478000080fa000b
:10718c000000060088007800c0042000972d07003e
:10719c006140b900f9e607000800e0000b0035007b
:1071ac0002002000a347240020e6070080a28800ec
:1071bc0091a2880011002000010078004f04780093
:1071cc000080fa0000000600eeff370002002000ed
:1071dc000378240058e6070002002000a34724008f
:1071ec0012e6070080a2880091a2880011002000fe
:1071fc00f1ff37000600fa00881f780047160700d9
:10720c006880570073eb07004f1607000400360028
:10721c00020078004f0478000080fa00000006009d
:10722c008800780000012000702d07007f40b90015
:10723c00c0a48800c0a48000709d880080c4b300e6
:10724c00a1f3b700100020004f0478000080fa0072
:10725c0000000600f2ff37000600fa00881f7800d5
:10726c002e160700688057005aeb070036160700e9
:10727c0004003600020078004f0478000080fa0009
:10728c00000006008800780020012000572d070020
:10729c007f40b900b0a48800b0a48000709d880025
:1072ac00d0c4b300a1f3b700100020004f04780045
:1072bc000080fa0000000600f2ff37000600fa001a
:1072cc00881f7800151607006880570041eb0700ef
:1072dc001d16070004003600020078004f047800e9
:1072ec000080fa00000006008800780040012000b1
:1072fc003e2d07007f40b900a0a48800a0a4800008
:10730c00709d8800c0c4b300a1f3b700100020002a
:10731c004f0478000080fa0000000600f2ff3700ee
:10732c000600fa00881f7800fc15070068805700db
:10733c0028eb070004160700040036000200780052
:10734c004f0478000080fa000000060088007800e6
:10735c00e0042000252d07007f40b90090a4880090
:10736c0090a48000709d880030c5b300a1f3b700d5
:10737c00100020004f0478000080fa000000060086
:10738c00f2ff37000600fa00f5150700668057007b
:10739c0010eb07007916070040062000808f500084
:1073ac0003003600020078000080fa00000006009e
:1073bc0071a4880071a48000600120000b2d0700cf
:1073cc00100020000080fa0000000600f8ff3700d3
:1073dc000600fa00e215070066805700fdea070078
:1073ec00ea15070003003600030078000080fa005d
:1073fc000000060062a4880061a48000c005200083
:10740c00fa2c0700100020000080fa000000060093
:10741c00f8ff37000600fa00d11507006680570008
:10742c00ecea070055160700703e2000808f5000d4
:10743c0003003600020078000080fa00000006000d
:10744c0021a4880021a4800060022000e72c070002
:10745c00100020000080fa0000000600f8ff370042
:10746c000600fa00be15070066805700d9ea07002f
:10747c00ca15070003003600030078000080fa00ec
:10748c000000060082a4880081a48000c0022000b5
:10749c00d62c0700100020000080fa000000060027
:1074ac00f8ff37000600fa00ad150700668057009c
:1074bc00c8ea0700b915070003003600030078007e
:1074cc000080fa0000000600529e8800519e800049
:1074dc00e0022000c52c0700100020000080fa00fc
:1074ec0000000600f8ff37000600fa00881f78003d
:1074fc008a15070068805700b6ea0700a315070035
:10750c0004003600030078004f0478000080fa0075
:10751c000000060032a4880031a480004002200044
:10752c00b22c070038a480006140b90013e60700b4
:10753c000800e0000b00350002002000832c240022
:10754c003ae5070080a0880091a088001300200075
:10755c00030078004f0478000080fa000000060059
:10756c00ecff3700020020000378240072e50700ce
:10757c0002002000832c24002ce5070080a088004a
:10758c0091a0880013002000f1ff37000600fa00dc
:10759c0073150700668057008eea07007b150700fd
:1075ac0003003600030078000080fa00000006009b
:1075bc00a2a28800a1a28000a00220008b2c0700b0
:1075cc00100020000080fa0000000600f8ff3700d1
:1075dc000600fa0062150700668057007dea070076
:1075ec00e6150700c0122000808f50000300360003
:1075fc00020078000080fa0000000600f1a3880069
:10760c00e0062000792c0700100020000080fa0012
:10761c0000000600f9ff37000a00fa00889fbe0040
:10762c008a9fbe008004780000509000e34f500009
:10763c00050032000000eb004f05be004f04be00f9
:10764c000080fa000000060029409000e0ef9f0047
:10765c0039409000f0ef9f004940900080f79f0068
:10766c005940900090f79f000044eb00a8f79f0052
:10767c007280570057ea07000005780079409000a7
:10768c00e0ef9f0009489000f0ef9f001948900030
:10769c0080f79f002948900090f79f00a8f79f0063
:1076ac00728057004bea070080057800494890002b
:1076bc00e0ef9f0059489000f0ef9f006948900060
:1076cc0080f79f007948900090f79f00a8f79f00e3
:1076dc00728057003fea070000047800f070220027
:1076ec00800f5500d3ff3e00808f5500d1ff3e0028
:1076fc00800f5400cfff3e0099407800c0c4b30007
:10770c0080cf5000af00320030003400d0c4b30042
:10771c0080cf5000fd0032006640400080cf50000a
:10772c00c4ff3a008a007800800420002f2c070048
:10773c006150b90091e507000a00e00079003500be
:10774c0002002000a3472400b8e4070040a28800f0
:10775c0051a2880088007800c0042000232c070068
:10776c006140b90085e507000800e0007c003500a9
:10777c0002002000a3472400ace4070080a288008c
:10778c0091a288008b007800a0042000172c070021
:10779c006158b90079e507000b00e0007f00350067
:1077ac0002002000a3472400a0e4070060a2880088
:1077bc0071a28800100020004f05be004f04be00cf
:1077cc000080fa00000006009fff37006440500064
:1077dc0080cf500097ff3a008a00780060032000a9
:1077ec00022c07006150b90064e507000a00e000b4
:1077fc002d00350002002000a34724008be4070075
:10780c0020a1880031a1880088007800a003200006
:10781c00f62b07006140b90058e507000800e000ae
:10782c003000350002002000a34724007fe407004d
:10783c0060a1880071a188008b0078008003200073
:10784c00ea2b07006158b9004ce507000b00e0007b
:10785c000b00350002002000a347240073e407004e
:10786c0040a1880051a18800100020004f05be00e7
:10787c004f04be000080fa000000060072ff3700c3
:10788c000200200003782400abe407000200200073
:10789c00a347240065e4070040a1880051a188009b
:1078ac0010002000f1ff37000200200003782400b4
:1078bc00a1e4070002002000a34724005be40700ba
:1078cc0020a1880031a1880088007800a003200046
:1078dc00c62b07006140b90028e507000800e0004e
:1078ec00d0ff3d00020020000378240092e4070042
:1078fc0002002000a34724004ce4070060a188008c
:10790c0071a188008b00780080032000b72b070042
:10791c006158b90019e507000b00e000cdff3d00f0
:10792c00d7ff3700020020000378240082e4070010
:10793c0002002000a34724003ce4070040a288007a
:10794c0051a2880088007800c0042000a72b0700f3
:10795c006140b90009e507000800e00084ff3d0024
:10796c00020020000378240073e4070002002000ca
:10797c00a34724002de4070080a2880091a2880070
:10798c008b007800a0042000982b07006158b900e8
:10799c00fae407000b00e00081ff3d00020020002c
:1079ac000378240064e4070002002000a3472400ad
:1079bc001ee4070060a2880071a28800100020005d
:1079cc007dff37008a00780020042000872b0700f9
:1079dc006150b900e9e407000a00e000230035001b
:1079ec0002002000a347240010e40700e0a1880057
:1079fc00f1a1880088007800600420007b2b070030
:107a0c006140b900dde407000800e0002600350005
:107a1c0002002000a347240004e4070020a28800f1
:107a2c0031a288008b007800400420006f2b0700e7
:107a3c006158b900d1e407000b00e00029003500c3
:107a4c0002002000a3472400f8e3070000a28800ee
:107a5c0011a28800100020004f05be004f04be008c
:107a6c000080fa0000000600f7fe3700020020003c
:107a7c000378240030e4070002002000a347240010
:107a8c00eae30700e0a18800f1a1880088007800f3
:107a9c0060042000552b07006140b900b7e40700d3
:107aac000800e000daff3d0002002000037824000b
:107abc0021e4070002002000a3472400dbe30700b9
:107acc0020a2880031a288008b007800400420009e
:107adc00462b07006158b900a8e407000b00e00032
:107aec00d7ff3d00020020000378240012e40700b9
:107afc0002002000a3472400cce3070000a288006a
:107b0c0011a2880010002000d3ff37008a007800f3
:107b1c00c0032000352b07006150b90097e4070023
:107b2c000a00e0002d00350002002000a3472400cd
:107b3c00bee3070080a1880091a18800880078002e
:107b4c0000042000292b07006140b9008be40700da
:107b5c000800e0003000350002002000a34724009c
:107b6c00b2e30700c0a18800d1a188008b00780087
:107b7c00e00320001d2b07006158b9007fe40700cb
:107b8c000b00e0000b00350002002000a34724008e
:107b9c00a6e30700a0a18800b1a188001000200076
:107bac004f05be004f04be000080fa000000060026
:107bbc00a5fe37000200200003782400dee3070056
:107bcc0002002000a347240098e30700a0a188002e
:107bdc00b1a1880010002000f1ff37000200200046
:107bec0003782400d4e3070002002000a3472400fc
:107bfc008ee3070080a1880091a18800880078009e
:107c0c0000042000f92a07006140b9005be407007a
:107c1c000800e000d0ff3d000200200003782400a3
:107c2c00c5e3070002002000a34724007fe3070000
:107c3c00c0a18800d1a188008b007800e00320004f
:107c4c00ea2a07006158b9004ce407000b00e00079
:107c5c00cdff3d00d7ff3700100005000600fa00ed
:107c6c00bf13070066805700dae80700cf13070040
:107c7c0003003600020078000080fa0000000600c5
:107c8c00419e8800a0062000d82a07001000200082
:107c9c000080fa0000000600f9ff37000600fa0029
:107cac00af13070066805700cae807000001780090
:107cbc00c0f92f00000041008001eb00c1762000cc
:107ccc00810f500003003600030078000080fa009a
:107cdc0000000600329e880082007800c00620005a
:107cec00c22a0700100020000080fa0000000600e5
:107cfc00f8ff37000600fa0099130700668057005a
:107d0c00b4e8070019140700e0702200808f5000bf
:107d1c0003003600030078000080fa000000060023
:107d2c00b29e88008200780000072000af2a07006e
:107d3c00100020000080fa0000000600f8ff370059
:107d4c000600fa008613070066805700a1e80700ba
:107d5c008000eb00e90f50000300360001007800b2
:107d6c000080fa000000060050a48800709988007a
:107d7c0080007800200720009c2a070010002000bb
:107d8c000080fa0000000600f7ff37000600fa003a
:107d9c0073130700668057008ee8070083130700f3
:107dac0003003600020078000080fa000000060094
:107dbc0041a4880061998800400720008b2a0700a5
:107dcc00100020000080fa0000000600f8ff3700c9
:107ddc000600fa0062130700668057007de8070072
:107dec006a13070003003600030078000080fa00d5
:107dfc0000000600e2a388008200780060072000e3
:107e0c007a2a0700100020000080fa00000006000b
:107e1c00f8ff3700800078006c54a9006713070046
:107e2c00020032007094a900100005007354e200a7
:107e3c0010003d001141780021c4b300814f510066
:107e4c001a00320060c4b300804f51002a00320087
:107e5c000a1607000000e0000100320073f4a800cd
:107e6c0019c8bf000043b000414e070010000500c8
:107e7c00eeff37009140780060c4b30080cf500013
:107e8c001600320020c4b30080cf5000f0ff3a003f
:107e9c0001007800ddf3b700ddd3bf00dff3b700de
:107eac00dc02a900dc82a800e9ff3700f13d2100cb
:107ebc009140780060c4b30080cf500018003200ad
:107ecc0002007800ddf3b700ddd3bf00dff3b700ad
:107edc00dc02a900dc82a800ddff3700010078007d
:107eec00ddf3b700ddd3bf00dff3b700dc02a80081
:107efc00dc82a900d6ff3700dfd3bf00814f5000d2
:107f0c000700320002007800ddf3b700ddd3bf00bc
:107f1c00dff3b700dc02a800dc82a900ccff37003d
:107f2c006e74a80080a48000609e880071d4a800a4
:107f3c0002007800def3b70020002000709e88005d
:107f4c006c34a80010000500b8ff3700881f7800bb
:107f5c0000047800191307001d003a001a130700db
:107f6c001b003a001b13070019003a001c130700f2
:107f7c0017003a007354e200050035009840780071
:107f8c001a1307002b0032001b1307001e003200cf
:107f9c00984090001b130700100032000040e800ce
:107fac0080cf50000d0032006740500080cf500051
:107fbc000a003200c9130700284090003015070052
:107fcc00a1d3bf00a0f3b70038409000e84d0700e4
:107fdc00100020004f047800000006008000fd0017
:107fec00e0f3b7008000fd00bc13070028409000b0
:107ffc0023150700a1d3bf00a0f3b70038409000b1
:10800c00db4d0700f2ff370001007800ddf3b7000d
:10801c00ddd3bf00dff3b700dc02a900dc82a800cf
:10802c009840900020c5b30080cf5000dbff3a0091
:10803c00eaff370001007800ddf3b700ddd3bf00a5
:10804c00dff3b700dc02a800dc82a90098409000a6
:10805c0020c5b30080cf5000d0ff3a00dfff3700bf
:10806c00509d800011032000810f50001f00340030
:10807c00409d8000810f50001c00340070d4bf0064
:10808c000038a300fdff32007074a900419d8000f0
:10809c00509d8000a5130700509e8000e10f5000fa
:1080ac0004003400cc13e20006003400cc33ed00a5
:1080bc00f2ff370010002000509e8800cc13e20025
:1080cc00faff3c00d212070008003400519d8000da
:1080dc00509e8000808f500004003400d2120700a4
:1080ec0002003400d8120700e4ff3700db1207004f
:1080fc008e13370000027800dd12070017003200e3
:10810c007254a9000400e00002003a0000732a0037
:10811c0011423700831f7800821f78000100fb009a
:10812c00801f7800e0a48000801f7800841f7800f6
:10813c0020742a00801f7800c08520008ee707007d
:10814c00c0852000e24007002c35070033350700be
:10815c006d14a800ec875700000006007254a800ac
:10816c00e8ff37000000e00002003a0000732a002c
:10817c00f9413700e1a48000811f7800801f78004e
:10818c0090752a00801f7800c08520007ae70700d0
:10819c00c0852000ce400700183507001f350700aa
:1081ac006d14a800e6875700000006000000e000f0
:1081bc0013003200ea8f50000f003e00811f780040
:1081cc00e1a48000811f7800801f7800c0772a000e
:1081dc00801f7800c085200067e70700c08520005d
:1081ec00bb400700053507000c3507006d14a800cf
:1081fc00e887570000000600a0762a00d641370019
:10820c0000732a00d44137000600fa00889fbe0094
:10821c008a1f7800dc1207008044eb0089ff9f0066
:10822c006c8057006be70700000578005840900001
:10823c00c0f79f0068449000d8f79f00e9f79f00b3
:10824c006c80570063e707008c12070008003e00a3
:10825c00820078000a007800d4ff0700100020008c
:10826c004f0578004f04be000080fa0000000600a5
:10827c00d0782a00b84107000000eb004f057800c9
:10828c004f04be000080fa0000000600f8ff370023
:10829c000201fb00821f78008100fb00811f780027
:1082ac00e1a48000811f7800801f7800007a2a00ea
:1082bc00801f7800408a20002fe70700408a2000aa
:1082cc00834007006a340700713407006c94a800df
:1082dc00ea8757000000060080017800641207004e
:1082ec00280032006b120700120032000200fb0063
:1082fc00801f78000100fb00801f7800e0a4800044
:10830c00801f7800831f7800307b2a00801f780044
:10831c00408a200018e70700408a20006c400700c4
:10832c00533407005a3407006d34a800ea8757000d
:10833c00000006007214a9000200fb00801f7800e8
:10834c000100fb00801f7800e0a48000801f7800f3
:10835c00831f7800307b2a00801f7800408a200021
:10836c0005e70700408a2000594007004034070009
:10837c00473407006d34a800ea8757000000060058
:10838c00ecff37007214a8000200fb00801f78007d
:10839c000100fb00801f7800e0a48000801f7800a3
:1083ac00831f7800307b2a00801f7800408a2000d1
:1083bc00f1e60700408a2000454007002c340700f6
:1083cc00333407006d34a800ea875700000006001c
:1083dc00d8ff370000017800d04388002412070032
:1083ec00240032002b120700100032000100fb00a9
:1083fc00801f7800e0a48000801f7800821f780026
:10840c00607c2a00801f780000882000dae60700d4
:10841c00008820002e400700653407006c340700ec
:10842c006cd4a800e8875700000006007234a9003d
:10843c000100fb00801f7800e0a48000801f780002
:10844c00821f7800607c2a00801f78000088200042
:10845c00c9e60700008820001d40070054340700bf
:10846c005b3407006cd4a800e887570000000600b6
:10847c00eeff37007234a8000100fb00801f78006b
:10848c00e0a48000801f7800821f7800607c2a00a6
:10849c00801f780000882000b7e6070000882000c5
:1084ac000b40070042340700493407006cd4a80085
:1084bc00e887570000000600dcff370080017800d9
:1084cc00c0409000ea11070012003200e0a48000c6
:1084dc00f2448000834890008100fb00811f7800eb
:1084ec00801f7800821f7800b07e2a00801f7800e1
:1084fc00408a2000a0e60700e8875700408a200049
:10850c00f33f0700da330700e13307006cf4a800ef
:10851c0000000600e0a48000f24480008348900034
:10852c008100fb00811f7800801f7800821f78007b
:10853c00907d2a00801f7800408a20008ee607007c
:10854c00e8875700408a2000e13f0700c833070046
:10855c00cf3307006cf4a80000000600edff3700d5
:10856c00889fbe008a1f7800800478000144780040
:10857c0002057800d0438800800078008006200037
:10858c009a2807003a4188003141800040062000bb
:10859c009628070090c4b300804f54002b00320083
:1085ac00f0c4b300804f5400130032008a1f7800cf
:1085bc000800fb00801f7800e0a48000801f78007a
:1085cc00891f7800d07f2a00801f78000088200047
:1085dc0069e6070000882000bd3f0700f433070060
:1085ec00fb3307006cd4a800ea8757004f057800ce
:1085fc004f04be00000006007234a9008a1f7800e8
:10860c000800fb00801f7800e0a48000801f780029
:10861c00891f7800d07f2a00801f780000882000f6
:10862c0055e6070000882000a93f0700e03307004b
:10863c00e73307006cd4a800ea8757004f05780091
:10864c004f04be0000000600ebff37007234a80098
:10865c008a1f78000800fb00801f7800e0a48000cf
:10866c00801f7800891f7800d07f2a00801f780037
:10867c000088200040e6070000882000943f070097
:10868c00cb330700d23307006cd4a800ea8757001d
:10869c004f0578004f04be0000000600d6ff3700df
:1086ac000600fa00889fbe008a1f780080047800bc
:1086bc0010407800c0f79f0019409000d0f79f0041
:1086cc0029409000e0f79f0039409000f0f79f00a0
:1086dc000044eb0088ff9f006c8057003de60700cc
:1086ec000005780059409000c0f79f006940900049
:1086fc00d0f79f0079409000e0f79f000948900068
:10870c00f0f79f0088ff9f006c80570031e6070050
:10871c0000017800c0f92f0000004500313820001e
:10872c00810f500005003600100020004f05780026
:10873c004f04be000080fa0000000600c940900003
:10874c000a00780086ff0700100020004f05780013
:10875c004f04be000080fa0000000600f7ff37004f
:10876c00e1a48000811f7800801f780000812a001e
:10877c00801f7800408a2000ffe50700408a200017
:10878c00533f0700408a200059400700e6875700f6
:10879c0000000600d0438800811f7800e1a480000f
:1087ac00811f7800801f780010822a00801f7800bb
:1087bc0000882000f0e5070000882000443f0700f7
:1087cc007b330700823307006cd4a800e88757007e
:1087dc00000006000000fe00100005007354e200cb
:1087ec000c003500f51007000a003a0073d4bf00e6
:1087fc000008a30007003a00f310070005003a0038
:10880c00f410070003003a00f510070001003a00cd
:10881c006e54a800100005007354e2000c003500e3
:10882c00e61007000a003a0073d4bf000008a3004a
:10883c0007003a00e410070005003a00e5100700b5
:10884c0003003a00e610070001003a006e34a8005d
:10885c00100005001e00fa00b04090007354e200b6
:10886c001b003500d510070019003a00d610070080
:10887c0017003a00d710070015003a00d81007006f
:10888c0013003a006e14a800de100700130032002b
:10889c00c0c4b300dcf3b700011107000c003200b8
:1088ac008099800091998000809fbe0021832a00ce
:1088bc00811f7800c0fd2f000f004000aee50700bf
:1088cc00c0fd2f000f00400023400700e687570033
:1088dc00100020000080fa00000006000100780063
:1088ec00dcf3b700ecff37001400fa00748057007b
:1088fc0081832a000a00090031587800b000b100c9
:10890c00b93f0700400620006f1107008355070090
:10891c00100020000080fa00000006000040eb0070
:10892c00fdf2b7000cf3b700eef2b700fef2b700a1
:10893c000df3b700eff2b700fff2b7000ef3b7007c
:10894c00f0f2b70000f3b7000ff3b700f1f2b70085
:10895c0001f3b70010f3b700f2f2b70002f3b7005f
:10896c0011f3b700f3f2b70003f3b70012f3b7003b
:10897c00f4f2b70004f3b70013f3b700f5f2b70045
:10898c00100005001400fa00889fbe0030449000cf
:10899c0066004000334007008044780068d4bf0074
:1089ac000028a30015003a00f0ccb30000404400ae
:1089bc00e14f5000040036000000eb004f04be00f5
:1089cc000080fa000000060010c3b300804f540072
:1089dc001a00320020c3b300804f5400f6ff3a0057
:1089ec00090078005cf4b7000000eb004f04be00f7
:1089fc000080fa0000000600f3ff37000980fb003e
:108a0c00801f78000880fb00801f780030842a00cb
:108a1c00801f78007e80570057e507007e80570046
:108a2c00cd3f0700e6875700f0ccb3000040440070
:108a3c00e14f5000e0ff3e00e3ff370009007800f3
:108a4c005ef4b7000000eb004f04be000080fa009b
:108a5c0000000600dcff3700881f78000004780057
:108a6c00220020008000780010852a007de5070098
:108a7c000000e00004003a006ed4a80010002000b2
:108a8c004f047800000006002200200088007800c7
:108a9c0040852a0073e507000000e00005003a005d
:108aac006eb4a800100020004f04780000000600ef
:108abc00f5ff3700220020008800780070852a001e
:108acc0068e507000000e0000b00320032002000d7
:108adc0088007800a0852a0062e507000000e0000d
:108aec000a003a00c74b0700100020004f04780022
:108afc0000000600e4ff3700be4b0700100020000a
:108b0c004f04780000000600dfff37003200200021
:108b1c0088007800e0852a0052e507000000e0009c
:108b2c000b003200320020008800780020862a00da
:108b3c004ce507000000e0000a003a00a84b0700d3
:108b4c00100020004f04780000000600ceff370014
:108b5c00994b0700100020004f047800000006001d
:108b6c00c9ff37003200200088007800c05d2a0061
:108b7c003ce507000000e000f5ff32003200200069
:108b8c008800780060862a0036e507000000e000c7
:108b9c00baff3a00a0862a00553f070060d4bf00f8
:108bac000008a30076003200a0872a00503f07007f
:108bbc0020882a004e3f070060d4bf000018a30095
:108bcc006c003200a0872a00493f070020892a0048
:108bdc00473f070060d4bf000028a30062003200aa
:108bec00a0872a00423f0700208a2a00403f070046
:108bfc0060d4bf000038a30058003200a0872a00c0
:108c0c003b3f0700208b2a00393f070061d4bf008f
:108c1c000048a3004e003200a0872a00343f070012
:108c2c00208c2a00323f070061d4bf000058a300fb
:108c3c0044003200a0872a002d3f0700208d2a0017
:108c4c002b3f07006154e2003b003d00a0872a0047
:108c5c00273f0700208e2a00253f070061d4bf0064
:108c6c000068a30031003200a0872a00203f0700d3
:108c7c00208f2a001e3f070061d4bf000038a300dc
:108c8c0027003200a0872a00193f070020902a00f5
:108c9c00173f070061d4bf000008a3001d0032007d
:108cac00a0872a00123f070020912a00103f0700de
:108cbc0061d4bf000018a3000d003200a0872a0069
:108ccc000b3f070020922a00093f070061d4bf0028
:108cdc000028a30009003200a0872a00043f0700e7
:108cec00100020004f0478000000060066ff3700db
:108cfc00e0872a00fe3e0700f2ff3700e0872a00db
:108d0c00fb3e0700100020004f0478000000060016
:108d1c005dff3700e0872a00f53e0700e2ff3700d1
:108d2c00e0872a00f23e0700d8ff3700e0872a00d0
:108d3c00ef3e0700ceff3700e0872a00ec3e07002d
:108d4c00c4ff3700e0872a00e93e0700bbff37006d
:108d5c00e0872a00e63e0700b1ff3700e0872a00d3
:108d6c00e33e0700a7ff3700e0872a00e03e07003c
:108d7c009dff3700e0872a00dd3e070093ff370098
:108d8c00e0872a00da3e070089ff3700881f780049
:108d9c0050a3800088292100801f7800e0a4800067
:108dac00801f780020932a00801f7800080078002c
:108dbc0071e4070008007800c53d0700e6875700fe
:108dcc00100020004f04780000000600881f780077
:108ddc00c0a48000bb0f0700801f7800e0a48000b7
:108dec00801f7800f0932a00801f7800080078001c
:108dfc0061e4070008007800b53d0700e6875700de
:108e0c00100020004f04780000000600881f780036
:108e1c00b0a48000ab0f0700801f7800e0a4800096
:108e2c00801f7800c0942a00801f7800080078000a
:108e3c0051e4070008007800a53d0700e6875700bd
:108e4c00100020004f04780000000600881f7800f6
:108e5c00a0a480009b0f0700801f7800e0a4800076
:108e6c00801f780090952a00801f780008007800f9
:108e7c0041e4070008007800953d0700e68757009d
:108e8c00100020004f04780000000600881f7800b6
:108e9c0090a480008b0f0700801f7800e0a4800056
:108eac00801f780060962a00801f780008007800e8
:108ebc0031e4070008007800853d0700e68757007d
:108ecc00100020004f04780000000600881f780076
:108edc0020a48000800f0700801f7800811f78007d
:108eec0030972a00801f78000800780022e40700e1
:108efc0008007800763d0700e68757001000200038
:108f0c004f04780000000600889fbe0020a180005e
:108f1c0031a18000730f0700801f7800891f780033
:108f2c0000982a00801f78000800780012e40700df
:108f3c0008007800663d0700e68757001000200007
:108f4c004f04be0000000600889fbe0080a1800078
:108f5c0091a18000630f0700801f7800891f7800a3
:108f6c00d0982a00801f78000800780002e40700df
:108f7c0008007800563d0700e687570010002000d7
:108f8c004f04be0000000600889fbe00e0a18000d8
:108f9c00f1a18000530f0700801f7800891f780013
:108fac00a0992a00801f780008007800f2e30700df
:108fbc0008007800463d0700e687570010002000a7
:108fcc004f04be0000000600889fbe0040a2800037
:108fdc0051a28000430f0700801f7800891f780082
:108fec00709a2a00801f780008007800e2e30700de
:108ffc0008007800363d0700e68757001000200077
:10900c004f04be0000000600889fbe0040a18000f7
:10901c0051a18000330f0700801f7800891f780052
:10902c00409b2a00801f780008007800d2e30700dc
:10903c0008007800263d0700e68757001000200046
:10904c004f04be0000000600889fbe00a0a1800057
:10905c00b1a18000230f0700801f7800891f7800c2
:10906c00109c2a00801f780008007800c2e30700db
:10907c0008007800163d0700e68757001000200016
:10908c004f04be0000000600889fbe0000a28000b6
:10909c0011a28000130f0700801f7800891f780031
:1090ac00e09c2a00801f780008007800b2e30700db
:1090bc0008007800063d0700e687570010002000e6
:1090cc004f04be0000000600889fbe0060a2800016
:1090dc0071a28000030f0700801f7800891f7800a1
:1090ec00b09d2a00801f780008007800a2e30700da
:1090fc0008007800f63c0700e687570010002000b7
:10910c004f04be0000000600889fbe0060a18000d6
:10911c0071a18000f30e0700801f7800891f780072
:10912c00809e2a00801f78000800780092e30700d8
:10913c0008007800e63c0700e68757001000200086
:10914c004f04be0000000600889fbe00c0a1800036
:10915c00d1a18000e30e0700801f7800891f7800e2
:10916c00509f2a00801f78000800780082e30700d7
:10917c0008007800d63c0700e68757001000200056
:10918c004f04be0000000600889fbe0020a2800095
:10919c0031a28000d30e0700801f7800891f780051
:1091ac0020a02a00801f78000800780072e30700d6
:1091bc0008007800c63c0700e68757001000200026
:1091cc004f04be0000000600889fbe0080a28000f5
:1091dc0091a28000c30e0700801f7800891f7800c1
:1091ec00f0a02a00801f78000800780062e30700d6
:1091fc0008007800b63c0700e687570010002000f6
:10920c004f04be0000000600881f780080a4800078
:10921c00b10e0700801f7800811f7800c0a12a00c2
:10922c00801f78000800780053e3070008007800de
:10923c00a73c0700e6875700100020004f04780079
:10924c0000000600881f7800509e8000a20e0700c8
:10925c00801f7800811f780090a22a00801f780060
:10926c000800780044e3070008007800983c0700e9
:10927c00e6875700100020004f047800000006001d
:10928c00881f780070a48000930e0700801f780060
:10929c00811f780060a32a00801f780008007800e6
:1092ac0035e3070008007800893c0700e687570083
:1092bc00100020004f04780000000600881f780082
:1092cc0060a48000840e0700801f7800811f780046
:1092dc0030a42a00801f78000800780026e30700dd
:1092ec00080078007a3c0700e68757001000200041
:1092fc004f04780000000600881f780030a480001e
:10930c00750e0700801f7800811f780000a52a00c9
:10931c00801f78000800780017e307000800780029
:10932c006b3c0700e6875700100020004f047800c4
:10933c0000000600881f7800a0a280008829210068
:10934c00801f7800e0a48000801f7800d0a52a0040
:10935c00801f78000800780007e3070008007800f9
:10936c005b3c0700e6875700100020004f04780094
:10937c0000000600881f7800d0a48000560e07005d
:10938c00801f7800811f7800a0a62a00801f78001b
:10939c0008007800f8e20700080078004c3c070051
:1093ac00e6875700100020004f04780000000600ec
:1093bc00881f7800f0a38000470e0700801f7800fc
:1093cc00811f780070a72a00801f780008007800a1
:1093dc00e9e20700080078003d3c0700e6875700eb
:1093ec00100020004f04780000000600881f780051
:1093fc00409e8000380e0700801f7800811f780087
:10940c0040a82a00801f780008007800dae20700e4
:10941c00080078002e3c0700e6875700100020005b
:10942c004f04780000000600881f7800309e8000f2
:10943c00290e0700801f7800811f780010a92a00d0
:10944c00801f780008007800cbe207000800780045
:10945c001f3c0700e6875700100020004f047800df
:10946c00000006001e00fa00b09e8000e1a48000ff
:10947c00801f7800811f7800e0a92a00801f7800e7
:10948c00c0fd2f000f004000bbe20700c0fd2f0005
:10949c000f0040000e3c0700e6875700100020002c
:1094ac000080fa00000006001e00fa0050a48000a4
:1094bc00e1a48000801f7800811f7800b0aa2a00e8
:1094cc00801f7800c0fd2f000f004000aae20700ab
:1094dc00c0fd2f000f004000fd3b0700e687570042
:1094ec00100020000080fa00000006001e00fa00a8
:1094fc0040a48000e1a48000801f7800811f7800c8
:10950c0080ab2a00801f7800c0fd2f000f004000a8
:10951c0099e20700c0fd2f000f004000ec3b070054
:10952c00e6875700100020000080fa0000000600bb
:10953c00e0a38000e1a48000801f7800811f7800e8
:10954c0050ac2a00801f7800802921008ae2070095
:10955c00e687570010000500881f7800e0a4800003
:10956c00dd0d0700801f7800811f780020ad2a00d8
:10957c00801f7800080078007fe207000800780060
:10958c00d33b0700e6875700100020004f047800fb
:10959c0000000600881f780000a48000ce0d070094
:1095ac00801f7800811f7800f0ad2a00801f7800a2
:1095bc000800780070e2070008007800c43b070040
:1095cc00e6875700100020004f04780000000600ca
:1095dc00881f780010a48000bf0d0700801f780042
:1095ec00811f7800c0ae2a00801f78000800780028
:1095fc0061e2070008007800b53b0700e6875700da
:10960c00100020004f047800000006001e00fa0035
:10961c00881f7800800078002210240033b42400c6
:10962c00b60d07007c8057009fe20700f8e79f000b
:10963c0000fe2f000f004000a53b070000fe2f008e
:10964c000f004000683c07004f0478000080fa00cf
:10965c00000006001e00fa00881f780080007800c9
:10966c0022e0240013b42400a40d07007c805700d2
:10967c008de20700f8e79f00a50d0700229120005e
:10968c00624078000080fb00801f780090af2a00b9
:10969c00801f78007d80570037e20700c0fd2f0047
:1096ac000f0040008a3b0700c0fd2f000f00400058
:1096bc004d3c0700e48757004f0478000080fa0007
:1096cc0000000600889fbe00950d0700a8902000a2
:1096dc0000004400ed00400032002000d08e20003d
:1096ec0060e20700800078000004e00004003a000b
:1096fc0010c0b300e9e8b70001007800e8e8b70053
:10970c00ae0d07000980b90000004400ed004000d8
:10971c0032002000908c200052e20700800078007c
:10972c000004e00004003a0010c0b300c5e8b70024
:10973c0001007800c4e8b7004f04be00000006002a
:10974c000600fa00060d07006680570021e20700ac
:10975c009c0c070003003600100020000080fa006b
:10976c0000000600e0a48000801f7800821f7800b3
:10977c0001812a00811f7800408a2000fee1070049
:10978c00408a2000523b0700408a2000583c0700ca
:10979c00e6875700100020000080fa000000060049
:1097ac00f0ff37000600fa00881f7800600d0700f4
:1097bc006880570007e207000001780030ed2f00a9
:1097cc00820c070004003600100020004f047800c3
:1097dc000080fa0000000600084890000000fb0022
:1097ec00801f7800484090000000fb00801f78002c
:1097fc00e0a48000801f7800821f7800007a2a0085
:10980c00801f7800408a2000dbe10700408a20009e
:10981c002f3b0700162f07001d2f07006c94a80084
:10982c00ea875700100020004f0478000080fa00ef
:10983c0000000600e8ff37000600fa00889fbe0013
:10984c008a1f7800500d07000045eb008aff9f002f
:10985c006c805700dfe1070080047800c0f92f000e
:10986c000080440031382000810f50000500360084
:10987c00100020004f0578004f04be000080fa0055
:10988c000000060058409000c0f79f006840900010
:10989c00d0f79f0078409000e0f79f00084c9000b4
:1098ac00f8f79f008aff9f006c805700c9e1070002
:1098bc00d9438800801f7800e0a48000801f7800c6
:1098cc00891f780010822a00801f780000882000f1
:1098dc00a9e1070000882000fd3a0700342f07009b
:1098ec003b2f07006cd4a800e8875700100020001d
:1098fc004f0578004f04be000080fa0000000600ff
:10990c00e0ff37000600fa00881f7800080d0700fa
:10991c0068805700afe1070000017800f0e62f00e7
:10992c002a0c070017003e0088499000c8409000a0
:10993c00cf0c070017003200d60c070028003200ad
:10994c000300fb00801f78000100fb00801f7800e3
:10995c00e0a48000801f7800821f7800307b2a00f2
:10996c00801f7800408a200083e10700408a200095
:10997c00d73a0700be2e0700c52e07006d34a8008d
:10998c00ea875700100020004f0478000080fa008e
:10999c00000006007214a8000300fb00801f780072
:1099ac000100fb00801f7800e0a48000801f78007d
:1099bc00821f7800307b2a00801f7800408a2000ac
:1099cc006de10700408a2000c13a0700a82e07006d
:1099dc00af2e07006d34a800ea875700e9ff370067
:1099ec007214a9000300fb00801f78000100fb002b
:1099fc00801f7800e0a48000801f7800821f780010
:109a0c00307b2a00801f7800408a20005ae1070032
:109a1c00408a2000ae3a0700952e07009c2e0700c6
:109a2c006d34a800ea875700d6ff37000600fa000d
:109a3c00881f7800be0c07006880570065e107009e
:109a4c00bf0c070004003600b0e02f0000004100fe
:109a5c00810f500015003e00c8409000d243880092
:109a6c00830c0700150032008a0c0700240032001a
:109a7c000100fb00801f7800e0a48000801f7800ac
:109a8c00821f7800607c2a00801f780000882000ec
:109a9c0039e10700008820008d3a0700c42e07002a
:109aac00cb2e07006cd4a800e887570010002000cc
:109abc004f0478000080fa00000006007234a80001
:109acc000100fb00801f7800e0a48000801f78005c
:109adc00821f7800607c2a00801f7800008820009c
:109aec0025e1070000882000793a0700b02e070016
:109afc00b72e07006cd4a800e8875700ebff37009f
:109b0c007234a9000100fb00801f7800e0a48000e3
:109b1c00801f7800821f7800607c2a00801f7800ec
:109b2c000088200014e1070000882000683a070034
:109b3c009f2e0700a62e07006cd4a800e8875700bc
:109b4c00daff37000600fa00050c070066805700a4
:109b5c0020e107007a0c070018003e000200e0002c
:109b6c0010003200e0a48000801f7800821f780073
:109b7c0091752a00811f7800c0852000fee0070047
:109b8c00c0852000523a07009c2e0700a32e070028
:109b9c006d14a80010002000e68757000080fa0022
:109bac000000060000732a006b3b07001000200029
:109bbc000080fa0000000600faff3700d0782a0077
:109bcc00653b07000000eb000080fa000000060077
:109bdc00f4ff37000600fa00889fbe008a9fbe0083
:109bec008004780010407800a0f79f001940900086
:109bfc00b0f79f0029409000c0f79f0039409000bb
:109c0c00d0f79f000044eb00e8f79f006e805700f0
:109c1c00f0e007000005780059409000a0f79f0085
:109c2c0069409000b0f79f00c8f79f006e80570006
:109c3c00e8e007008005780079409000a0f79f00cd
:109c4c0009489000b0f79f00c8f79f006e8057003e
:109c5c00e0e00700090c070008003e00c940900036
:109c6c00030c0700210032007254a9000a00e00026
:109c7c0007003a0000732a00373b07001000200051
:109c8c004f05be004f04be000080fa000000060025
:109c9c00821f78008b1f78000100fb00801f78006a
:109cac00e0a48000801f78008a1f780020742a00ae
:109cbc00801f7800c0852000afe00700c085200021
:109ccc00033a07004d2e0700542e07006d14a80010
:109cdc00ec875700100020004f05be004f04be005b
:109cec000080fa0000000600e9ff37007254a8005b
:109cfc00deff37000600fa00881f78000c0c070006
:109d0c0068805700b3e007002e0b070004003600f4
:109d1c00100020004f0478000080fa0000000600bc
:109d2c00f24488008200780080012000af220700f6
:109d3c00c840900090c4b30080cf50001600320091
:109d4c00e0a48000f2448000884890008100fb0071
:109d5c00811f7800801f7800821f7800b07e2a0057
:109d6c00801f7800408a200083e00700e8875700b6
:109d7c00408a2000d6390700bd2d0700c42d0700ee
:109d8c006cf4a800100020004f0478000080fa004a
:109d9c0000000600e2ff3700e0a48000f2448000df
:109dac00884890008100fb00811f7800801f78009c
:109dbc00821f7800907d2a00801f7800408a200046
:109dcc006de00700e8875700408a2000c039070083
:109ddc00a72d0700ae2d07006cf4a800e9ff370093
:109dec003200fa00889fbe008a1f780000057800b8
:109dfc0071d4bf000038a30047003a006c54a8008f
:109e0c000000eb00709e88007334a9006c34a9002c
:109e1c00ea40900081cf9f00fa41900093cf9f00c1
:109e2c00a0cf9f0080fc2f000f00400069e00700ce
:109e3c000000e000020032006c34a800709e880024
:109e4c00d0c4b3009a4f1000650032009a409000c5
:109e5c0030c5b30080cf50000500320000c5b30000
:109e6c0080cf500053003200630b070056003200c5
:109e7c006e74a8006c54a80080a48000609e8800ba
:109e8c002a41900061c4b300814f51003900320067
:109e9c0020c4b300804f51003f00320071d4bf008a
:109eac000008a30003003a0070d4bf000068a300b0
:109ebc00020032007a0b070005003a001000200067
:109ecc004f0578004f04be000080fa000000060029
:109edc008099800091998000809fbe00e1af2a009c
:109eec00811f780020fc2f000f00400022e00700ab
:109efc0020fc2f000f004000973a0700e687570020
:109f0c00100020004f0578004f04be000080fa00be
:109f1c0000000600eeff37000bc9bf008080fb007d
:109f2c00600220000089b900c0fd2f0000844700aa
:109f3c002010240031b42400008cbe008044eb00bf
:109f4c0089e79f00409120008000410032002000f2
:109f5c0003fe2f000380470053e00700b9e79f0082
:109f6c00080078005a390700080078001e3a0700ec
:109f7c00a2ff3700f13d21009140780020c4b300ce
:109f8c0080cf5000c5ff3a0071d4a80002007800c1
:109f9c00def3b700c1ff3700dfd3bf00814f5000a5
:109fac00beff3a0071d4a80002007800def3b700bf
:109fbc00baff37006e74a8006c54a80081a480000e
:109fcc00619e8800aeff37006e74a8006c54a80028
:109fdc0083a48000639e880071d4a800a8ff37007a
:109fec0066404000260d07009a40900030c5b30033
:109ffc0080cf50001a00320020c4b30080cf500034
:10a00c001700320000c5b30080cf5000140032009e
:10a01c0020c5b30080cf500014003200c0c4b30080
:10a02c0080cf5000110032002a41900061c4b3006f
:10a03c00814f51001200320020c4b300804f5100f8
:10a04c0096ff3a00dfd3bf00814f500093ff3a00d8
:10a05c0071f4a80002007800def3b7008fff370020
:10a06c007114a80070d4a900efff37007114a90077
:10a07c0070d4a80001007800dcf3b700eaff3700c9
:10a08c00f13d21009140780020c4b30080cf5000f6
:10a09c0082ff3a0071f4a80002007800def3b700ea
:10a0ac007eff37002400fa00889fbe008a9fbe0006
:10a0bc008c1f78008004780010409000a0d79f007f
:10a0cc00a9419000b3d79f0039409000c0d79f00a2
:10a0dc00e48544009b417800d3d79f000046eb00f9
:10a0ec00ecd79f0020fd2f000f004000b9df0700c8
:10a0fc000005780080f32f00000045003106200099
:10a10c00810f50003e003e0071d4bf000038a30008
:10a11c0010003a003a41880031418000400620008e
:10a12c00b22107009b407800da0a070027003200b2
:10a13c0012002000ce0a07003a003200020078001c
:10a14c004f0678004f05be004f04be000080fa0099
:10a15c00000006000bc9bf008080fb0060022000dd
:10a16c000089b90020fd2f000f004000650440005d
:10a17c0000b22a0004000900305c78005800b100dd
:10a18c00409120008000410032002000b3fd2f00e0
:10a19c0003804700c4df0700ecdf9f000800780055
:10a1ac00cb380700080078008f3907003a41880047
:10a1bc0031418000400620008c2107009b40780034
:10a1cc00f0c4b30080cf5000d9ff3a007314a9003b
:10a1dc007034a9005e74a9002c28ef000000eb007d
:10a1ec00e6340700100020004f0678004f05be0033
:10a1fc004f04be000080fa0000000600d5ff3700b7
:10a20c0060b02a00d4390700000020004f06780007
:10a21c004f05be004f04be000080fa00000006008f
:10a22c00ccff370079409000a0d79f00894c90005c
:10a23c00b9d79f00ccd79f0020fd2f000f00400006
:10a24c0064df0700000178008000e9002006200090
:10a25c00808f5000010036003200200062418800df
:10a26c007034a800100020004f0678004f05be0087
:10a27c004f04be000080fa0000000600b5ff370056
:10a28c000f02b000889fbe008a9fbe008c9fbe004c
:10a29c008e1f7800c90a0700680220000880b900e8
:10a2ac0068004000aa9020008a0478000a00400050
:10a2bc000048eb0068d4bf000018a30031003a003e
:10a2cc00bb0a0700000045002048900032c4b300d0
:10a2dc00824f5000390032009c0a070030c5b30091
:10a2ec0080cf5000d7003200980a0700450a0700bb
:10a2fc004b013200950a070010c4b30080cf500008
:10a30c0021023200aa0a07006800400042c0b300d4
:10a31c0002f07c000044eb0068d4bf000028a300ce
:10a32c000c0032007a0a07006800400060407d0093
:10a33c00e44f50004c023200a00a07000280b90022
:10a34c0068004000a290200060407900e34f50006c
:10a35c00e4013200720a070064004000ab90200058
:10a36c0060007d00e10f50006a0032004f0778005a
:10a37c004f06be004f05be004f04be000f02b100d9
:10a38c00000006000bc9bf000080fb000880b9006c
:10a39c0000004500690040006f3907000bc9bf0081
:10a3ac000080fb000880b9000000450020489000a8
:10a3bc0032c4b300824f5000c7ff3a000006eb00d6
:10a3cc00e97021006b0220000d7121000bc9bf0048
:10a3dc000080fb000b80b90000004500eb00400042
:10a3ec000e17ec00220020001edf07000004e00026
:10a3fc00a20132000c06e800e6864600e684440022
:10a40c000bc9bf000080fb000b80b90000004500a9
:10a41c00eb0040001900e8002200200011df0700cb
:10a42c000004e00009003a000bc9bf000080fb00eb
:10a43c000b80b90066004000e0007d0049409000b0
:10a44c000080fb00808f5000670032000c06e80093
:10a45c006684460088067800668744008e0478007f
:10a46c000bc9bf000080fb000b80b9000000450049
:10a47c00eb0040001e00e80022002000f9de07007f
:10a48c000004e00009003a000bc9bf000080fb008b
:10a49c000b80b90066004000e0007d004e4090004b
:10a4ac000080fb00808f50004f003200e606440015
:10a4bc00e68444000bc9bf000080fb000b80b90090
:10a4cc0000004500eb0040001900e80022002000cd
:10a4dc00e4de07000004e0003a0032000c86e800dd
:10a4ec00ec064400ec044700f60f5600c4ff3a009b
:10a4fc000bc9bf000080fb00620220000280b90083
:10a50c006800400042c0b30002707d000044eb00c4
:10a51c0081ff3700e14f54007e0132000bc9bf00b0
:10a52c000080fb000980b9000081450020e0240078
:10a53c0011b42400a0af9f00b1af9f000044eb000a
:10a54c0088df9f00ea0041003200200083fd2f00cd
:10a55c0003804700d4de0700b8df9f000bc9bf00a3
:10a56c000080fb000980b9006800400060c07d00dd
:10a57c000080fb00801f780090af2a00801f7800bd
:10a58c0071fd2f00018047007bde070000fd2f00ce
:10a59c000f004000ce37070000fd2f000f004000d9
:10a5ac0091380700e48757004f0778004f06be002c
:10a5bc004f05be004f04be000f02b10000000600a4
:10a5cc0070ff37000bc9bf000080fb000b80b90087
:10a5dc0066004000e0007d00494090000080fb00d8
:10a5ec00808f5000bdff3a000bc9bf000080fb00fc
:10a5fc000b80b900640040001200200002307d0086
:10a60c000bc9bf000080fb000b80b90000004500a7
:10a61c006d0040009d0078000100010000447800ae
:10a62c000004e0003cff3a000bc9bf000080fb00b7
:10a63c000b80b9006800400032c0b30002707d008e
:10a64c0035ff37008006eb00498621006b022000a5
:10a65c006e8621000bc9bf000080fb000b80b90087
:10a66c0000004500eb0040006418ec0022002000c4
:10a67c007cde07000004e0000d0132008d06e800ce
:10a68c0066074700e68444000bc9bf000080fb004e
:10a69c000b80b90000004500eb0040001900e800f9
:10a6ac00220020006fde07000004e00009003a00e1
:10a6bc000bc9bf000080fb000b80b9006600400096
:10a6cc00e0007d00494090000080fb00808f50002e
:10a6dc003c0032008d06e80066044700080778004d
:10a6ec00668644008c0478000bc9bf000080fb0018
:10a6fc000b80b90000004500eb0040001c00e80096
:10a70c002200200057de07000004e00009003a0098
:10a71c000bc9bf000080fb000b80b9006600400035
:10a72c00e0007d004c4090000080fb00808f5000ca
:10a73c002400320066074400e68444000bc9bf00c5
:10a74c000080fb000b80b90000004500eb004000ce
:10a75c001900e8002200200042de07000004e0009f
:10a76c000f0032008d86e8006c074400ec044600b4
:10a77c0050022000808f5600c3ff3a000bc9bf0067
:10a78c000080fb00620220000280b90068004000db
:10a79c0042c0b30002707d000044eb00defe3700c7
:10a7ac000bc9bf000080fb000b80b90066004000a5
:10a7bc00e0007d00494090000080fb00808f50003d
:10a7cc00e8ff3a000bc9bf000080fb000b80b9000a
:10a7dc00640040001200200002307d000bc9bf0055
:10a7ec000080fb000b80b900000045006d004000ac
:10a7fc009e00780001000100004478000004e00095
:10a80c00c5fe3a000bc9bf000080fb000b80b900ed
:10a81c006800400032c0b30002707d00befe3700fd
:10a82c008006eb002e7921000e0478006c022000cb
:10a83c000bc9bf000080fb000c80b9000000450074
:10a84c00eb0040001800e8002200200005de0700a5
:10a85c000004e00009003a000bc9bf000080fb00b7
:10a86c000c80b90066004000e0007d00484090007c
:10a87c000080fb00808f5000630032008d04e800e4
:10a88c0089067800e60544000b0478000bc9bf006c
:10a89c000080fb000c80b90000004500eb0040007c
:10a8ac001b00e80022002000eedd07000004e000a1
:10a8bc0009003a000bc9bf000080fb000c80b900f6
:10a8cc0066004000e0007d004b4090000080fb00e3
:10a8dc00808f50004c0032008d06e8006604440066
:10a8ec000bc9bf000080fb000c80b90000004500c4
:10a8fc00eb0040001800e80022002000d9dd070022
:10a90c000004e00009003a000bc9bf000080fb0006
:10a91c000c80b90066004000e0007d0048409000cb
:10a92c000080fb00808f5000370032008986e800e1
:10a93c006c8445000bc9bf000080fb000c80b90083
:10a94c0000004500eb0040001800e8002200200049
:10a95c00c4dd07000004e00009003a000bc9bf0089
:10a96c000080fb000c80b90066004000e0007d0018
:10a97c00484090000080fb00808f50002200320085
:10a98c00e3864400728445000bc9bf000080fb00c5
:10a99c000c80b90000004500eb0040001800e800f6
:10a9ac0022002000afdd07000004e0000d003200a3
:10a9bc0078844500e4864400ff8f54009cff3a00e5
:10a9cc000bc9bf000080fb00620220000280b900ae
:10a9dc006800400042c0b30002707d000044eb00f0
:10a9ec004dfe37000bc9bf000080fb000c80b90086
:10a9fc0066004000e0007d00484090000080fb00b5
:10aa0c00808f5000eaff3a004001200090408800ff
:10aa1c000bc9bf000080fb000c80b9006400400033
:10aa2c000001eb0002307d000bc9bf000080fb0071
:10aa3c000c80b900000145006668b9000080e80090
:10aa4c006d014100e0007f00020078000100010070
:10aa5c00802921009e3607008029210062370700db
:10aa6c004f0778004f06be004f05be004f04be00d6
:10aa7c000f02b1000000060042fe37000bc9bf00f8
:10aa8c000080fb000b80b90066004000e0007d00f8
:10aa9c0012d7bf000080fb00808f5000d2fe320026
:10aaac000c06e800e6864600e684440054fe3700b7
:10aabc000bc9bf000080fb000b80b9006600400092
:10aacc00e0007d0068d8bf000080fb00808f500044
:10aadc003cff32008d06e80066074700e684440020
:10aaec00e9fe370000b42a009b3707000bc9bf00f2
:10aafc000080fb00690220000980b900640040005e
:10ab0c00ab90200060007d00e10f500017fe3a0072
:10ab1c0080fe37000bc9bf000080fb000980b90024
:10ab2c00000145002010240031b42400a0af9f0088
:10ab3c00b1af9f000044eb0088df9f00ea004100aa
:10ab4c003200200083fd2f000380470056dd0700f4
:10ab5c00b8df9f0040fd2f000f0040005c3607005f
:10ab6c0040fd2f000f0040001f3707004f077800f3
:10ab7c004f06be004f05be004f04be000f02b100d1
:10ab8c0000000600fffd37000bc9bf000080fb0072
:10ab9c000880b9000080440030489000824f50007b
:10abac0053fe3a000bc9bf000080fb000880b900bf
:10abbc0000804400c0489000b0c4b30080cf500067
:10abcc004bfe3a000bc9bf000080fb000880b900a7
:10abdc00640040000005eb000ab07c000bc9bf000c
:10abec000080fb000880b90000804400ed004000ac
:10abfc0032002000d08e20001add07000004e00097
:10ac0c0004003a0010c0b300e9e8b7000a0078006d
:10ac1c00e8e8b7000bc9bf000080fb000880b90052
:10ac2c0000804400ed00400032002000908c200099
:10ac3c000cdd07000004e000ccfd3a0010c0b300ae
:10ac4c00c5e8b7000a007800c4e8b7004f077800e1
:10ac5c004f06be004f05be004f04be000f02b100f0
:10ac6c0000000600c7fd370050b22a003a37070033
:10ac7c000bc9bf000080fb00690220000980b900ed
:10ac8c0064004000ab90200060007d00e10f50009c
:10ac9c00b6fd3a001ffe37001e00fa00889fbe006a
:10acac008a9fbe00800578006ad4bf000008a3000c
:10acbc001e003a006ad4bf000018a3001b003a0023
:10accc0071d4bf000038a3001c003a00d4c2bf00ee
:10acdc000048a300800032007607070064004000a3
:10acec008001eb0002d82000033079007354e2009d
:10acfc0033003d00220020008b00780090b52a0024
:10ad0c00d8dc07000000e000b9003a00c0c4b30072
:10ad1c00e0f3b700710807000000eb004f05be0020
:10ad2c004f04be000080fa00000006006a34ef00f9
:10ad3c0071d4bf000038a300e4ff32006c74a9008a
:10ad4c000bc9bf000080fb00690220000980b9001c
:10ad5c00aa902000000145002010240031b42400ea
:10ad6c00d0af9f00e1af9f000044eb00e8df9f00f5
:10ad7c00ea00410032002000e3fd2f000380470071
:10ad8c00c9dc070098e79f00a0fd2f000f004000d2
:10ad9c00cf350700a0fd2f000f00400092360700b2
:10adac000bc9bf000080fb000980b90064004000a3
:10adbc000001eb0002307d007354e200cdff350042
:10adcc00220020008b00780080b62a00a5dc07004a
:10addc00800078000000e00049003200cb82a8001f
:10adec00cb62a800ab409000c0c4b30080cf500031
:10adfc008d0032000040e80080cf5000030032008c
:10ae0c006540500080cf50004b013200b3a480004d
:10ae1c00339d8800b0a48000209d88002200200073
:10ae2c008b00780020b62a008edc07000001780029
:10ae3c000000e00005013a007134210091407800d7
:10ae4c0030c5b30080cf50002b013200713421008b
:10ae5c009140780020c4b30080cf5000980032009d
:10ae6c0071342100914078006a40400080cf50003e
:10ae7c00930032007134210091407800664040000c
:10ae8c0080cf50008e00320061c4b3000100780006
:10ae9c00ddf3b700ddd3bf00dff3b700dc02a800a1
:10aeac00dc82a900a0002000109d88000100780021
:10aebc0047f3b7006e74a9006c54a9007094a800f5
:10aecc000000eb004f05be004f04be000080fa00ee
:10aedc000000060095ff37006c74a80081cdbf0000
:10aeec000080fb00620220000280b9006400400078
:10aefc008001eb0002d82000033079007bff370083
:10af0c005c94a8005cb4a9005cd4a9005cf4a90012
:10af1c0073d4bf000048a3003f003a007354e20012
:10af2c007dff350070d4bf000048a3007aff3200cb
:10af3c00509d800012032000820f50003f0034000f
:10af4c00409d8000820f50003c00340070d4bf0044
:10af5c000038a300fdff32007074a900419d8000f1
:10af6c00509d8000f1070700509e8000e10f5000bb
:10af7c0004003400cc13e20006003400cc33ed00a6
:10af8c00f2ff370010002000509e8800cc13e20026
:10af9c00faff3c0080a48000609e8800519d8000d8
:10afac0020032000808f500063013400519d8000ed
:10afbc00509e8000808f50005f013400509d8000b7
:10afcc00519e800001005000509d8800419d8000e2
:10afdc00509e8000808f500057013400409d8000af
:10afec00519e800001005000409d8800d7ff370023
:10affc00220020008b007800c0b52a0019dc070065
:10b00c000000e00043013a0020c5b300e0f3b700b4
:10b01c00b207070040ff370073f4a9007354e20035
:10b02c00c0ff3d003cff3700a3a48000339d880087
:10b03c00a0a48000209d880078ff3700519d8800d7
:10b04c00419d8800419d8000509d8000b7070700fe
:10b05c00aa33ef00a833ef00a633ef00a433ef00c0
:10b06c006000b800b10707007094a9006c74a900c7
:10b07c006c54a90030c5b30047f3b700f13d210073
:10b08c00914078006d40500080cf5000300132006c
:10b09c0020c4b300ddf3b700ddd3bf00dff3b7008e
:10b0ac00dc02a900dc82a8000000eb004f05be000a
:10b0bc004f04be000080fa00000006001bff3700a2
:10b0cc00509d800011032000810f50004d00340072
:10b0dc00409d8000810f50004a00340070d4bf00a6
:10b0ec000038a300fdff32007074a900419d800060
:10b0fc00509d80008d070700509e8000e10f50008e
:10b10c0004003400cc13e20006003400cc33ed0014
:10b11c00f2ff370010002000509e8800cc13e20094
:10b12c00faff3c0080a48000609e8800519d800046
:10b13c0020032000808f500032003400519d80008d
:10b14c00509e8000808f50002e003400509d800057
:10b15c00519e800001005000509d8800419d800050
:10b16c00509e8000808f500026003400409d80004f
:10b17c00519e800001005000409d8800d7ff370091
:10b18c00220020008b007800e0b62a00b5db070017
:10b19c000000e0009b023a00309d8000220020005d
:10b1ac00110009000200d800209d88007134210094
:10b1bc009140780020c4b30080cf50000a003200c8
:10b1cc0071342100914078006a40400080cf5000db
:10b1dc000500320071342100914078006640400037
:10b1ec0080cf500028ff3a00509d800011032000b2
:10b1fc00810f500003003400409d8000810f5000ef
:10b20c006f023c00aa33ef00a833ef00419d800091
:10b21c00509d80004507070061c4b3000100780011
:10b22c00ddf3b700ddd3bf00dff3b700dc02a8000d
:10b23c00dc82a900a0002000109d88008000fd0089
:10b24c0047f3b7008000fd001aff370022002000f2
:10b25c008b00780050b62a0082db070000017800d2
:10b26c000000e000c6003a007134210091407800e3
:10b27c0030c5b30080cf500034003200713421004f
:10b28c009140780060c4b30080cf50003f00320082
:10b29c0071342100914078006640400080cf50000e
:10b2ac003a00320071342100914078006640400031
:10b2bc0080cf50003500320021c4b300010078006b
:10b2cc00ddf3b700ddd3bf00dff3b700dc02a9006c
:10b2dc00dc82a800a0002000109d88008000fd00ea
:10b2ec0047f3b7008000fd006e74a9006c54a900f0
:10b2fc007094a800f2fe3700429d8800439d8000a8
:10b30c00539d880061c4b30001007800ddf3b700e1
:10b31c00ddd3bf00dff3b700dc02a800dc82a9009c
:10b32c00a0002000109d88008000fd0047f3b700ae
:10b33c008000fd00dffe3700c3a48000339d880031
:10b34c00c0a48000209d8800b4fe3700429d880078
:10b35c00439d8000539d880021c4b30001007800f8
:10b36c00ddf3b700ddd3bf00dff3b700dc02a900cb
:10b37c00dc82a800a0002000109d88008000fd0049
:10b38c0047f3b7008000fd00d7ff3700509d8000c9
:10b39c0011032000810f500035003400409d8000c7
:10b3ac00810f50003200340070d4bf000038a3006d
:10b3bc00fdff32007074a900419d8000509d8000fb
:10b3cc00da060700509e8000e10f500004003400a4
:10b3dc00cc13e20038003400cc33ed00f2ff370020
:10b3ec0010002000509e8800f9ff3700220020003a
:10b3fc008b00780040b72a001adb07000000e00041
:10b40c006d023a00309d80002200200011000900de
:10b41c000200d800209d88007134210091407800f2
:10b42c0060c4b30080cf50000a0032007134210098
:10b43c00914078006640400080cf500005003200fb
:10b44c0071342100914078006640400080cf50005c
:10b45c0099ff3a00509d800011032000810f50008d
:10b46c0003003400409d8000810f500044023c00da
:10b47c00aa33ef00a833ef00419d8000509d80005f
:10b48c00aa06070021c4b30001007800ddf3b70061
:10b49c00ddd3bf00dff3b700dc02a900dc82a8001b
:10b4ac00a0002000109d88008000fd0047f3b7002d
:10b4bc008000fd008cff370080a48000609e880017
:10b4cc00519d800020032000808f5000e8ff340045
:10b4dc00519d8000509e8000808f5000e4ff34000e
:10b4ec00509d8000519e800001005000509d8800ae
:10b4fc00419d8000509e8000808f5000dcff340006
:10b50c00409d8000519e800001005000409d8800ad
:10b51c00a5ff3700220020008b007800f0b52a0030
:10b52c00d0da07000000e00081003a007114a80096
:10b53c006a060700f8fd3700aa33ef00a833ef00c6
:10b54c00419d8000509d800078060700c0fe3700aa
:10b55c0001007800ddf3b700ddd3bf00dff3b700e7
:10b56c00dc02a800dc82a9000000eb004f05be0045
:10b57c004f04be000080fa0000000600ebfd37000f
:10b58c00220020008b007800c0b52a00b5da070035
:10b59c000000e00089003a006cd4bf000008a30052
:10b5ac0084003a0020a480007f00b9000000d10084
:10b5bc00309d880020a480007f00b9000000d100dd
:10b5cc00209d88007134210091407800c0c4b300e4
:10b5dc0080cf500017003200713421009140780068
:10b5ec006640500080cf50001200320071342100b0
:10b5fc00914078006440500080cf50000d00320024
:10b60c0021c5b30001007800ddf3b700dc02a8000f
:10b61c00dc82a800a0002000109d880001007800aa
:10b62c0047f3b7006e74a9006c54a9007094a8007d
:10b63c0023fe3700509d800011032000810f500025
:10b64c0014003400409d8000810f50001100340024
:10b65c0070d4bf000038a300fdff32007074a90045
:10b66c00419d8000509d800030060700509e800058
:10b67c00e10f500004003400cc13e200150034003c
:10b68c00cc33ed00f2ff370010002000509e8800f4
:10b69c00f9ff3700aa33ef00a833ef00419d80007b
:10b6ac00509d80002106070021c5b30001007800e1
:10b6bc00ddf3b700dc02a800dc82a800a0002000ab
:10b6cc00109d88008000fd0047f3b7008000fd004e
:10b6dc00d4ff370083a48000639e8800519d8000b6
:10b6ec0020032000808f5000eaff3400519d800021
:10b6fc00509e8000808f5000e6ff3400509d8000eb
:10b70c00519e800001005000509d8800419d80009a
:10b71c00509e8000808f5000deff3400409d8000e2
:10b72c00519e800001005000409d8800c8ff3700ea
:10b73c00220020008b00780020b62a0049da07008e
:10b74c000000e00089003a0033c5b3000300780024
:10b75c00e0f3b700113a210091407800c2c4b30065
:10b76c0082cf50009000320093003c0080c4b300a4
:10b77c0080cf50000a003200c0c4b300a0f3b70061
:10b78c00d605070064fd3700d0c4b30080cf50004d
:10b79c008e0032006640400080cf5000f6ff3a0029
:10b7ac008000fd00a0f3b7008000fd00cb05070072
:10b7bc0059fd37006c14a90082ff370022002000cd
:10b7cc008b00780090b52a0026da07000000e00014
:10b7dc0085003a006cd4bf000008a30080003a003a
:10b7ec0020a480007f00b9000000d100309d8800ab
:10b7fc0020a480007f00b9000000d100209d8800ab
:10b80c00713421009140780020c5b30080cf5000e6
:10b81c001700320071342100914078006c405000c8
:10b82c0080cf50001200320071342100914078001a
:10b83c006440500080cf50000d003200c1c4b300f2
:10b84c0001007800ddf3b700dc02a900dc82a9005e
:10b85c00a0002000109d88000100780047f3b7007d
:10b86c006e74a9006c54a9007094a80094fd370064
:10b87c00509d800011032000810f500014003400f3
:10b88c00409d8000810f50001100340070d4bf0027
:10b89c000038a300fdff32007074a900419d8000a8
:10b8ac00509d8000a1050700509e8000e10f5000c4
:10b8bc0004003400cc13e20015003400cc33ed004e
:10b8cc00f2ff370010002000509e8800f9ff37006f
:10b8dc00aa33ef00a833ef00419d8000509d8000fb
:10b8ec0092050700c1c4b30001007800ddf3b70076
:10b8fc00dc02a900dc82a900a0002000109d8800b9
:10b90c008000fd0047f3b7008000fd00d4ff370036
:10b91c0080a48000609e8800519d80002003200040
:10b92c00808f5000eaff3400519d8000509e8000b3
:10b93c00808f5000e6ff3400509d8000519e8000a7
:10b94c0001005000509d8800419d8000509e800059
:10b95c00808f5000deff3400409d8000519e80009f
:10b96c0001005000409d8800c8ff370022002000d5
:10b97c008b00780050b62a00bad907000000e0000e
:10b98c0062003a00113a210091407800c2c4b30021
:10b99c0082cf5000700032007bff3c0080c4b300ab
:10b9ac0080cf500074ff3a00d0c4b300a0f3b700ae
:10b9bc004a050700d8fc3700d0c4b30080cf500034
:10b9cc006100320083cf50006bff3a000001fd0094
:10b9dc00a0f3b7000001fd0040050700cefc3700c6
:10b9ec006c14a90086ff3700220020008b00780021
:10b9fc00b0b62a009bd907000000e000e0fd3a0039
:10ba0c00209d800022002000110009000200d800b7
:10ba1c00309d8800713421009140780020c4b3001f
:10ba2c0080cf50000a003200713421009140780020
:10ba3c006a40400080cf5000050032007134210074
:10ba4c00914078006640400080cf50000efd3a00d7
:10ba5c00509d800011032000810f5000e9fd34003f
:10ba6c00409d8000810f5000e6fd340070d4bf0073
:10ba7c000038a300fdff32007074a900419d8000c6
:10ba8c00509d800029050700509e8000e10f50005a
:10ba9c0004003400cc13e20005003400cc33ed007c
:10baac00f2ff370010002000509e8800f9ff37008d
:10babc0083a48000639e8800519d80002003200099
:10bacc00808f5000cffd3400519d8000509e80002f
:10badc00808f5000cbfd3400509d8000519e800023
:10baec0001005000509d8800419d8000509e8000b8
:10bafc00808f5000c3fd3400409d8000519e80001b
:10bb0c0001005000409d8800d8ff37002200200023
:10bb1c008b00780080b62a0052d907000000e000a4
:10bb2c007cfc3a0071d4bf000008a3000200320074
:10bb3c0030c5b300a0f3b700a0d3bf005006070078
:10bb4c00e604070074fc370080c4b300a0f3b70010
:10bb5c00e204070070fc370030c5b300a0f3b70057
:10bb6c00de0407006cfc370083a48000639e880011
:10bb7c00519d800020032000808f5000a1fd3400d7
:10bb8c00519d8000509e8000808f50009dfd3400a0
:10bb9c00509d8000519e800001005000509d8800f7
:10bbac00419d8000509e8000808f500095fd340098
:10bbbc00409d8000519e800001005000409d8800f7
:10bbcc0070d4bf000038a300fdff32007074a900d0
:10bbdc00419d8000509d8000d4040700509e800041
:10bbec00e10f500004003400cc13e200deff3400ff
:10bbfc00cc33ed00f2ff370010002000509e88007f
:10bc0c00f9ff3700220020008b00780010b72a00c3
:10bc1c0014d907000000e000f4fd3a00209d8000dc
:10bc2c0022002000110009000200d800309d88007d
:10bc3c00713421009140780060c4b30080cf500073
:10bc4c000a003200713421009140780066404000b7
:10bc5c0080cf5000050032007134210091407800f3
:10bc6c006640400080cf500093fd3a00509d80000c
:10bc7c0011032000810f5000fdfd3400409d800019
:10bc8c00810f5000fafd340070d4bf000038a300bf
:10bc9c00fdff32007074a900419d8000509d800012
:10bcac00a2040700509e8000e10f500004003400f5
:10bcbc00cc13e20005003400cc33ed00f2ff37006a
:10bccc0010002000509e8800f9ff370083a48000ec
:10bcdc00639e8800519d800020032000808f5000bf
:10bcec00e3fd3400519d8000509e8000808f5000f9
:10bcfc00dffd3400509d8000519e800001005000fb
:10bd0c00509d8800419d8000509e8000808f500087
:10bd1c00d7fd3400409d8000519e800001005000f2
:10bd2c00409d8800d8ff370083a48000639e880064
:10bd3c00519d800020032000808f5000ccfd3400ea
:10bd4c00519d8000509e8000808f5000c8fd3400b3
:10bd5c00509d8000519e800001005000509d880035
:10bd6c00419d8000509e8000808f5000c0fd3400ab
:10bd7c00409d8000519e800001005000409d880035
:10bd8c0070d4bf000038a300fdff32007074a9000e
:10bd9c00419d8000509d800064040700509e8000ef
:10bdac00e10f500011003400cc13e200deff340030
:10bdbc00cc33ed00f2ff3700220020008b0078001e
:10bdcc0070b72a00a7d807000000e0000a003a006c
:10bddc006ed4a8000000eb004f05be004f04be005f
:10bdec000080fa0000000600d0fb37001000200095
:10bdfc00509e8800ecff3700220020008b0078005a
:10be0c00a0b72a0097d807000000e000c2fb3a0058
:10be1c006eb4a8000000eb004f05be004f04be003e
:10be2c000080fa0000000600c0fb3700cb030700bf
:10be3c004d003200000307006f03070007003200bb
:10be4c000003070005003200020307000300320064
:10be5c0061c4b300f202070021013700509d80003d
:10be6c0011032000810f500011003400409d800010
:10be7c00810f50000e00340070d4bf000038a300b6
:10be8c00fdff32007074a900419d8000509d800020
:10be9c0026040700509e8000e10f5000170034006c
:10beac00cc13e20019003400cc33ed00f2ff370064
:10bebc00aa33ef00a833ef00419d8000509d800015
:10becc001a04070061c4b30001007800ddf3b70069
:10bedc00ddd3bf00dff3b700dc02a800dc82a900d1
:10beec00a0002000109d88008000fd0047f3b700e3
:10befc008000fd0000000600d8ff37001000200075
:10bf0c00509e8800cc13e200e7ff3c0080a4800028
:10bf1c00609e8800519d800020032000808f50007f
:10bf2c00e3ff3400519d8000509e8000808f5000b4
:10bf3c00dfff3400509d8000519e800001005000b6
:10bf4c00509d8800419d8000509e8000808f500045
:10bf5c00d7ff3400409d8000519e800001005000ae
:10bf6c00409d8800c4ff3700a833ef00409d80003f
:10bf7c00509d880061c4b30001007800ddf3b70068
:10bf8c00ddd3bf00dff3b700dc02a800dc82a90020
:10bf9c00a0002000109d88008000fd0047f3b70032
:10bfac008000fd0000000600acff37006b030700ab
:10bfbc004e003200a00207000c03070008003200fc
:10bfcc00a402070006003200a2020700040032009f
:10bfdc0021c4b300010078008c0207006600370012
:10bfec00509d800011032000810f5000110034007f
:10bffc00409d8000810f50000e00340070d4bf00b3
:10c00c000038a300fdff32007074a900419d800030
:10c01c00509d8000c5030700509e8000e10f50002a
:10c02c0017003400cc13e20019003400cc33ed00bf
:10c03c00f2ff3700aa33ef00a833ef00419d8000d8
:10c04c00509d8000b903070021c4b30001007800a3
:10c05c00ddf3b700ddd3bf00dff3b700dc02a900ce
:10c06c00dc82a800a0002000109d88008000fd004c
:10c07c0047f3b7008000fd0000000600d8ff370032
:10c08c0010002000509e8800cc13e200e7ff3c001b
:10c09c0080a48000609e8800519d800020032000b9
:10c0ac00808f5000e3ff3400519d8000509e800033
:10c0bc00808f5000dfff3400509d8000519e800027
:10c0cc0001005000509d8800419d8000509e8000d2
:10c0dc00808f5000d7ff3400409d8000519e80001f
:10c0ec0001005000409d8800c4ff3700a833ef00ca
:10c0fc00409d8000509d880021c4b3000100780051
:10c10c00ddf3b700ddd3bf00dff3b700dc02a9001d
:10c11c00dc82a800a0002000109d88008000fd009b
:10c12c0047f3b7008000fd0000000600acff3700ad
:10c13c006cd4bf000008a30056003a004902070067
:10c14c003d020700c0c4b30080cf50001000320085
:10c15c00390207006640500080cf50000c003200be
:10c16c00490207000a00320021c5b3000100780023
:10c17c00ddf3b700dc02a800dc82a800a0002000e0
:10c18c00109d88000100780047f3b70000000600fe
:10c19c00509d800011032000810f50002c003400b2
:10c1ac00409d8000810f50002900340070d4bf00e6
:10c1bc000038a300fdff32007074a900419d80007f
:10c1cc00509d800059030700509e8000e10f5000e5
:10c1dc0004003400cc13e20006003400cc33ed0034
:10c1ec00f2ff370010002000509e8800cc13e200b4
:10c1fc00faff3c0080a48000609e8800519d800066
:10c20c0020032000808f500011003400519d8000cd
:10c21c00509e8000808f50000d003400509d800097
:10c22c00519e800001005000509d8800419d80006f
:10c23c00509e8000808f500005003400409d80008f
:10c24c00519e800001005000409d8800d7ff3700b0
:10c25c00aa33ef00a833ef00419d8000509d800071
:10c26c003203070021c5b30001007800ddf3b700ed
:10c27c00dc02a800dc82a800a0002000109d880031
:10c28c008000fd0047f3b7008000fd0000000600b1
:10c29c00bfff37006c14a900a9ff37006cd4bf0096
:10c2ac000008a30051003a00ee010700e20107006c
:10c2bc00540207000c003200df0107006c405000f4
:10c2cc0080cf500008003200ef010700060032005a
:10c2dc00c1c4b30001007800ddf3b700dc02a90093
:10c2ec00dc82a900a5ff3700509d800011032000bf
:10c2fc00810f50002c003400409d8000810f5000b5
:10c30c002900340070d4bf000038a300fdff3200b8
:10c31c007074a900419d8000509d800003030700ac
:10c32c00509e8000e10f500004003400cc13e2005a
:10c33c0006003400cc33ed00f2ff37001000200073
:10c34c00509e8800cc13e200faff3c0080a48000d1
:10c35c00609e8800519d800020032000808f50003b
:10c36c0011003400519d8000509e8000808f500041
:10c37c000d003400509d8000519e80000100500043
:10c38c00509d8800419d8000509e8000808f500001
:10c39c0005003400409d8000519e8000010050003b
:10c3ac00409d8800d7ff3700aa33ef00a833ef0079
:10c3bc00419d8000509d8000dc020700c1c4b30089
:10c3cc0001007800ddf3b700dc02a900dc82a900d3
:10c3dc00a0002000109d88008000fd0047f3b700ee
:10c3ec008000fd0000000600bfff37006c14a900a0
:10c3fc00aeff370079010700ff010700050032008e
:10c40c009001070003003200920107000100320086
:10c41c008ffe3700509d800011032000810f5000cb
:10c42c002c003400409d8000810f50002900340006
:10c43c0070d4bf000038a300fdff32007074a90057
:10c44c00419d8000509d8000b8020700509e8000e6
:10c45c00e10f500004003400cc13e200060034005d
:10c46c00cc33ed00f2ff370010002000509e880006
:10c47c00cc13e200faff3c0080a48000609e880090
:10c48c00519d800020032000808f5000110034004b
:10c49c00519d8000509e8000808f50000d00340014
:10c4ac00509d8000519e800001005000509d8800de
:10c4bc00419d8000509e8000808f5000050034000c
:10c4cc00409d8000519e800001005000409d8800de
:10c4dc00d7ff3700aa33ef00a833ef00419d80004f
:10c4ec00509d80009102070061c4b30001007800e8
:10c4fc00ddf3b700ddd3bf00dff3b700dc02a8002b
:10c50c00dc82a900a0002000109d88008000fd00a6
:10c51c0047f3b7008000fd0000000600bdff3700a8
:10c52c0034010700b4010700050032004501070083
:10c53c0003003200470107000100320044fe3700bf
:10c54c00509d800011032000810f50002c003400fe
:10c55c00409d8000810f50002900340070d4bf0032
:10c56c000038a300fdff32007074a900419d8000cb
:10c57c00509d80006d020700509e8000e10f50001e
:10c58c0004003400cc13e20006003400cc33ed0080
:10c59c00f2ff370010002000509e8800cc13e20000
:10c5ac00faff3c0080a48000609e8800519d8000b2
:10c5bc0020032000808f500011003400519d80001a
:10c5cc00509e8000808f50000d003400509d8000e4
:10c5dc00519e800001005000509d8800419d8000bc
:10c5ec00509e8000808f500005003400409d8000dc
:10c5fc00519e800001005000409d8800d7ff3700fd
:10c60c00aa33ef00a833ef00419d8000509d8000bd
:10c61c004602070061c4b30001007800ddf3b700e7
:10c62c00ddd3bf00dff3b700dc02a800dc82a90079
:10c63c00a0002000109d88008000fd0047f3b7008b
:10c64c008000fd0000000600bdff3700e30007007e
:10c65c006601070005003200fe00070003003200ef
:10c66c00fc0007000100320059fe3700509d80008d
:10c67c0011032000810f50002c003400409d8000dd
:10c68c00810f50002900340070d4bf000038a30083
:10c69c00fdff32007074a900419d8000509d800008
:10c6ac0022020700509e8000e10f5000040034006d
:10c6bc00cc13e20006003400cc33ed00f2ff37005f
:10c6cc0010002000509e8800cc13e200faff3c00c2
:10c6dc0080a48000609e8800519d80002003200073
:10c6ec00808f500011003400519d8000509e8000be
:10c6fc00808f50000d003400509d8000519e8000b2
:10c70c0001005000509d8800419d8000509e80008b
:10c71c00808f500005003400409d8000519e8000a9
:10c72c0001005000409d8800d7ff3700aa33ef006e
:10c73c00a833ef00419d8000509d8000fb01070055
:10c74c0021c4b30001007800ddf3b700ddd3bf00d6
:10c75c00dff3b700dc02a900dc82a800a0002000f7
:10c76c00109d88008000fd0047f3b7008000fd009d
:10c77c0000000600bdff37009e0007001b010700ec
:10c78c0005003200b300070003003200b1000700bf
:10c79c00010032000efe3700509d80001103200076
:10c7ac00810f50002c003400409d8000810f500000
:10c7bc002900340070d4bf000038a300fdff320004
:10c7cc007074a900419d8000509d8000d701070026
:10c7dc00509e8000e10f500004003400cc13e200a6
:10c7ec0006003400cc33ed00f2ff370010002000bf
:10c7fc00509e8800cc13e200faff3c0080a480001d
:10c80c00609e8800519d800020032000808f500086
:10c81c0011003400519d8000509e8000808f50008c
:10c82c000d003400509d8000519e8000010050008e
:10c83c00509d8800419d8000509e8000808f50004c
:10c84c0005003400409d8000519e80000100500086
:10c85c00409d8800d7ff3700aa33ef00a833ef00c4
:10c86c00419d8000509d8000b001070021c4b300a1
:10c87c0001007800ddf3b700ddd3bf00dff3b700b4
:10c88c00dc02a900dc82a800a0002000109d88001a
:10c89c008000fd0047f3b7008000fd00000006009b
:10c8ac00bdff37005c94a8005cb4a9005cd4a9005f
:10c8bc005cf4a90073d4bf000048a300010032004f
:10c8cc0073f4a9007354e2002c003500bb00070080
:10c8dc002a003200509d800011032000810f50006f
:10c8ec0011003400409d8000810f50000e00340078
:10c8fc0070d4bf000038a300fdff32007074a90093
:10c90c00419d8000509d800088010700509e800052
:10c91c00e10f50001a003400cc13e2001c0034006c
:10c92c00cc33ed00f2ff3700cc0007007f0107008d
:10c93c00aa33ef00a833ef00a633ef00a433ef00c7
:10c94c006000b800790107007094a9006c74a9000c
:10c95c006c54a90030c5b30047f3b700f13d21007a
:10c96c00914078006d40500080cf50001200320092
:10c97c0020c4b30025000700dc82a80000000600dc
:10c98c0010002000509e8800cc13e200e4ff3c0015
:10c99c009f000700e4ff3400519d8000509e8000f2
:10c9ac00808f5000e0ff34009f000700deff340052
:10c9bc00a5000700ceff370019000700dc82a90094
:10c9cc000000060000017800b0e02f0000004100dc
:10c9dc0021062000810f500000000600209d8000e1
:10c9ec0022002000110009000200d800309d8800b0
:10c9fc0011003700309d800022002000110009003a
:10ca0c000200d800209d88000b003700ddf3b70032
:10ca1c00ddd3bf00dff3b700dc02a9000000060085
:10ca2c0001007800ddf3b700ddd3bf00dff3b70002
:10ca3c00dc02a8000000060071342100914078004f
:10ca4c0000000600fcff07006a40400080cf500049
:10ca5c0000000600f8ff07006640400080cf500041
:10ca6c000000060020a480007f00b9000000d10067
:10ca7c00309d880020a480007f00b9000000d10008
:10ca8c00209d880000000600ebff0700644050006a
:10ca9c0080cf500000000600c848dd000080fb007d
:10caac00008170009840780000c3b30080cf500024
:10cabc000000060081cdbf000080fb006202200058
:10cacc000280b900000006000080fb004400dd007d
:10cadc0080844400384090000000060090407800ac
:10caec0081f79f009040900091f79f00a04090002c
:10cafc00a1f79f0030409000b0f79f000040eb0082
:10cb0c00c0f79f0000000600000478008000eb00d6
:10cb1c00703e2000800f540000000600904078000a
:10cb2c00c1f79f0090409000d1f79f00a04090006b
:10cb3c00e1f79f0030409000f0f79f000040eb00c1
:10cb4c0080ff9f000000060000047800ea005000ff
:10cb5c000001eb00600e2000808f500000000600ea
:10cb6c0090407800e1f79f0090409000f1f79f0013
:10cb7c00a040900081ff9f003040900090ff9f00ec
:10cb8c000040eb00a0ff9f000000060077000700ac
:10cb9c00603e2000808f50000000060073000700ec
:10cbac0030062000808f5000000006007300070044
:10cbbc00f0702200808f50000000060070d4bf007f
:10cbcc000048a300000006006ed4bf000028a3009c
:10cbdc00000006006ed4bf000018a3000000060081
:10cbec006ed4bf000008a3000000060060c4b300b0
:10cbfc0080cf50000000060020c4b30080cf50004e
:10cc0c000000060020c5b30080cf500000000600d5
:10cc1c0080a48000609e8800519d8000200320002d
:10cc2c00808f500000000600509d8000519e8000b7
:10cc3c0001005000509d8800419d8000509e800056
:10cc4c00808f500000000600409d8000519e8000a7
:10cc5c0001005000409d880000000600aa33ef0040
:10cc6c00a833ef00419d8000509d8000000006001d
:10cc7c0090c4b30080cf5000000006000001780083
:10cc8c00b0f92f000000450021062000810f500054
:10cc9c0000000600f0c4b30080cf50000000060076
:10ccac00a0998000b19980008099880091998800a2
:10ccbc0051a480007199880068d4bf000028a3009b
:10cccc000000060088292100f20120001100090053
:10ccdc000200d80000000600e1a480008829210091
:10ccec0000000600e9a48000882921000200200031
:10ccfc00a3472400edcf07002bcf3700e2af9f00f6
:10cd0c00f3af9f000044eb0088e79f003200050062
:10cd1c002a000700620220000280b9000000060011
:10cd2c0026000700690220000980b90000000600f7
:10cd3c00150007000040eb0080ff9f00000006007c
:10cd4c0000017800b0f92f0020ff37001800070011
:10cd5c0000804400a04890000000060036ff070049
:10cd6c0030c5b30080cf50000000060000017800f1
:10cd7c008000e9008001eb000000060080007800d4
:10cd8c000001eb0000000600000478001040780061
:10cd9c0080f79f001840900090f79f00284090006b
:10cdac00a0f79f0038409000b0f79f0000000600ed
:10cdbc00020007000880b900000006000bc9bf0084
:10cdcc000080fb00000006000001e90001003a00b1
:10cddc00000006000200e90067006000000000008f
:10cdec0011002000828f5000f9ff32000000e0009b
:10cdfc001c003200810f500016003200e20f500070
:10ce0c0012003200e30f50000e003200e40f50000d
:10ce1c000a003200e50f500006003200e60f500009
:10ce2c000200320000000000210020000000000081
:10ce3c008100e800000000008100e8000000000014
:10ce4c008100e800000000008100e8000000000004
:10ce5c008100e800000000008100e800828f500093
:10ce6c00dbff3200000000000100e80000000000c1
:10ce7c0000000000000000000000000000000000a6
:10ce8c000000000000000000e7004000828f50000e
:10ce9c00cfff3200000000000100e800000000009d
:10ceac000000000000000000000000000000000076
:10cebc000000000000000000e7004000828f5000de
:10cecc00e8ff3a00c2ff370080007800e833ef003b
:10cedc0021130700feff3900000006002113070094
:10ceec00060032002413070008003200674050008f
:10cefc0080cf50000900320000000600caa2a80032
:10cf0c00cac2a90070b82a00932e3700caa2a80082
:10cf1c00cac2a80000b92a008f2e3700caa2a900e5
:10cf2c00cac2a800e0b72a008b2e37008001780017
:10cf3c000102780010032000808f510001003c009a
:10cf4c008001eb00800f520001003c000002eb005e
:10cf5c00c1d42100818f510001003400810178007f
:10cf6c00810f520001003400010278000300e00040
:10cf7c0002003a000400e0001b003200dc62a80052
:10cf8c00d23d21001241780060c4b300804f5100a3
:10cf9c001b003200804f510008003600c0c4b300a3
:10cfac00804f51000800320066404000804f510015
:10cfbc0005003200d6110700000006006440500046
:10cfcc00804f5100fbff3a00949f8800839f88009c
:10cfdc00909f8000b00e8800809f8000d00e88004b
:10cfec0000000600f5ff3700dc62a900d23d2100ed
:10cffc001241780060c4b300804f5100e5ff3a0045
:10d00c00939f8800849f8800909f8000b00e8800ba
:10d01c00809f8000d00e880000000600e7ff3700dc
:10d02c00d8120700010032006ad4a800d8120700f9
:10d03c00010032006ad4a800e233ec00109f80009b
:10d04c00e10f5000020034005a130700e233ef00e6
:10d05c0074d4bf000068a3006100320074d4bf0018
:10d06c000048a3005700320074d4bf000038a3005e
:10d07c004d0032007454e20044003d0075d4bf00f2
:10d08c000008a3003a0032007554e20031003d0064
:10d09c0075d4bf000038a3002700320075d4bf0040
:10d0ac000048a3001d00320075d4bf000028a30067
:10d0bc001300320075d4bf000018a3000800320022
:10d0cc006ad4bf000068a30001003a00000006000b
:10d0dc00c0122000d939070073f4a9000000060023
:10d0ec006ad4a80000c22a001b2e0700bc1207003d
:10d0fc006ad4bf000068a300f4ff3200f4ff3700cd
:10d10c006ad4a80000c12a00132e0700a31207003e
:10d11c000018a300eaff3a00f1ff37006ad4a80018
:10d12c0000c02a000c2e07009c1207000028a30048
:10d13c00e0ff3a00f2ff37006ad4a80000bf2a00d3
:10d14c00052e0700951207000048a300d6ff3a00f1
:10d15c00f2ff37006ad4a80040be2a00fe2d07005b
:10d16c008e1207000038a300ccff3a00f2ff370004
:10d17c006ad4a80090bd2a00f72d0700981207006a
:10d18c007554e200c2ff3500f2ff37006ad4a800e4
:10d19c0090bc2a00f02d0700801207000008a300a5
:10d1ac00b9ff3a00f2ff37006ad4a80090bb2a00fe
:10d1bc00e92d07008a1207007454e200afff350016
:10d1cc00f2ff37006ad4a80090ba2a00e22d0700bb
:10d1dc00751207000038a300a6ff3a00f2ff3700d3
:10d1ec006ad4a80090b92a00db2d07006e12070044
:10d1fc000048a3009cff3a00f2ff37003c13e2000a
:10d20c00020034003c33ed00000006005e54e200e6
:10d21c00040035005ef4a80010002000e09988009e
:10d22c00000006005ef4a90090002000fbff370010
:10d23c0062d4bf000038a300090032007574a80046
:10d24c005c12070004003a006254e2000200350050
:10d25c007594a900000006007594a8000000060053
:10d26c007574a900f6ff3700e6874700889fbe005b
:10d27c008a9fbe008c9fbe008e1f78006066b8002f
:10d28c000000eb00f0b79f00e9342100390478006e
:10d29c0009077800cc11070041003500ce110700ba
:10d2ac007fb097000000e80080bf9f001904780051
:10d2bc008e84e800c411070049003500cb1107002b
:10d2cc00e4044700c011070052003500c7110700e5
:10d2dc00e6044700bc1107005b003500381207005c
:10d2ec000006be0019047800e8044700b6110700d8
:10d2fc001d003500b81107000006be000fb89700de
:10d30c0064004000f0b79f00fe0f5000dfff3a00b2
:10d31c0002002000031f24000a00be00c3cd07003a
:10d32c00020020006351240002ce070012c9210024
:10d33c0063bf23005dce07000200200043192400c8
:10d34c00fdcd0700020020000312240057ce070079
:10d35c004f0778004f06be004f05be004f04be00bd
:10d36c006f00b100000006000200200003782400ca
:10d37c00f1cd07000001be000c00be00eecd070091
:10d38c000005be000006be000fb897006400400008
:10d39c00f0b79f00fe0f5000bcff3a00dcff3700d7
:10d3ac000200200003782400e3cd07000001be003a
:10d3bc000c00be00e0cd07000005be007fb097005a
:10d3cc000000e80080bf9f00190478008e84e800fc
:10d3dc006140b90069ce07000800e000b7ff3d00ce
:10d3ec000200200003782400d3cd07000001be000a
:10d3fc000a00be00d0cd07000005be00190478005d
:10d40c00e40447006140b9005cce07000800e0006e
:10d41c00aeff3d000200200003782400c6cd0700bb
:10d42c000001be000a00be00c3cd07000005be000f
:10d43c0019047800e60447006140b9004fce07009c
:10d44c000800e000a5ff3d00020020000378240046
:10d45c00b9cd07000001be000a00be00b6cd070022
:10d46c000006be0019047800e80447006140b900ca
:10d47c0042ce07000800e0009eff3d00baff3700d7
:10d48c00881f780000447800c0c4b300804f54005b
:10d49c00370032001c003400d0c4b300804f54005d
:10d4ac005f00320066404000804f5400470032005d
:10d4bc00a0c52a00282d070091a48000719d88002a
:10d4cc0030c5b300a1f3b70030022000b09e880035
:10d4dc0040a2800051a28000c0a08800d1a088008a
:10d4ec0060a2800071a28000e0a08800f1a08800fa
:10d4fc0080a2800091a2800000a1880011a1880068
:10d50c004f0478000000060064405000804f540027
:10d51c00e7ff3a0000c32a000f2d0700c0a48000cb
:10d52c00709d880008007800a1f3b700a0002000cf
:10d53c00b09e880020a1800031a18000c0a088008e
:10d54c00d1a0880040a1800051a18000e0a08800fb
:10d55c00f1a0880060a1800071a1800000a188006a
:10d56c0011a188004f04780000000600e6ff370088
:10d57c00c0c42a00f82c0700a1a48000719d88006b
:10d58c0008007800a1f3b70090012000b09e88003d
:10d59c00e0a18000f1a18000c0a08800d1a088008b
:10d5ac0000a2800011a28000e0a08800f1a08800f9
:10d5bc0020a2800031a2800000a1880011a1880067
:10d5cc004f04780000000600cfff3700a0c52a00ea
:10d5dc00e12c070091a48000719d88000800780060
:10d5ec00a1f3b70030022000b09e880040a280005a
:10d5fc0051a28000c0a08800d1a0880060a2800049
:10d60c0071a28000e0a08800f1a0880080a28000b8
:10d61c0091a2800000a1880011a18800b8ff3700fa
:10d62c00e0c32a00cc2c0700b1a48000719d8800b7
:10d63c0008007800a1f3b70040012000b09e8800dc
:10d64c0080a1800091a18000c0a08800d1a088009a
:10d65c00a0a18000b1a18000e0a08800f1a088000a
:10d66c00c0a18000d1a1800000a1880011a1880078
:10d67c004f04780000000600a3ff3700521007008b
:10d68c0005003200dd100700e01007000700320033
:10d69c006a34ef00100005006d54e200faff35000b
:10d6ac00dd100700682d070000000500df100700e3
:10d6bc00652d0700000005000040eb00fdf2b700ef
:10d6cc000cf3b700eef2b700fef2b7000df3b700a3
:10d6dc00eff2b700fff2b7000ef3b700f0f2b700ad
:10d6ec0000f3b7000ff3b700f1f2b70001f3b70086
:10d6fc0010f3b700f2f2b70002f3b70011f3b70062
:10d70c00f3f2b70003f3b70012f3b700f4f2b7006b
:10d71c0004f3b70013f3b700f5f2b70000000600ee
:10d72c00c51007000f003a00e60f07000e0032008c
:10d73c002011070008003a0062d4bf000048a30083
:10d74c00180032008b0f07001b003200a80f0700d7
:10d75c00170032008a0f0700bd10070001003400cb
:10d76c00be1007000000060062d4bf000008a30032
:10d77c0002003a0010c0b30017e8b700bb10070056
:10d78c0002003a0020c0b30017e8b700ba10070037
:10d79c0002003a0030c0b30017e8b700b910070018
:10d7ac00edff37005a0f0700e8ff3a000200370080
:10d7bc005a0f0700e8ff37005b0f0700e5ff3a0040
:10d7cc00fbff3700889fbe00c00f0700030034002a
:10d7dc00af1007004f04be00000006000801be0099
:10d7ec000800be0031cd070002002000a32f24004a
:10d7fc008ecc07004f04be0000000600f7ff370078
:10d80c003200fa00803e2000d0a48800e0fc2f00fb
:10d81c000f00400051c92a0023000900315878003c
:10d82c004002b100e0fc2f000f004000302c07003c
:10d83c00e0a48000801f780091cb2a00811f780023
:10d84c00a0fc2f000f004000cbd10700a0fc2f0044
:10d85c000f004000262c0700e48757000080fa00d8
:10d86c00000006008001e9000002eb00848f5000ec
:10d87c00350032000300e000300032000300e90004
:10d88c00670060000000000012002000828f510031
:10d89c002a0032000000e0001c003200820f500011
:10d8ac0016003200e20f500012003200e30f50005d
:10d8bc000e003200e40f50000a003200e50f500059
:10d8cc0006003200e60f500002003200000000009b
:10d8dc0022002000000000000201e800000000000f
:10d8ec000201e800000000000201e8000000000056
:10d8fc000201e800000000000201e8000000000046
:10d90c000201e800828f51000c0032000000000080
:10d91c000200e80000000000000000000000000011
:10d92c0000000000000000000000000000000000eb
:10d93c0067014000828f5100f4ff3a000402e800b6
:10d94c00848f5000cbff3a0000000600271107001f
:10d95c00e922a80000000000e922a900000006004e
:10d96c000a00fa0071b4a900c013e20003003400ed
:10d97c00c033ed00c013e2000e013200be13e20012
:10d98c0003003400be33ed00be13e2000701320089
:10d99c004853e200030032004873ed004853e200a4
:10d9ac002b013200ba13e20003003400ba33ed004d
:10d9bc00ba13e200fb003200b813e200030034009b
:10d9cc00b833ed00b813e200f4003200b613e200f5
:10d9dc0003003400b633ed00b613e200ed00320064
:10d9ec00b413e20003003400b433ed00b413e200ce
:10d9fc00e60032001208e200010034001228ed00ab
:10da0c0062d4bf000038a300de0032007574a80099
:10da1c00d4c2bf000018a3008b003a006254e2008d
:10da2c00890035007594a900d5c2bf000028a30059
:10da3c0089003a006dd4a800e0012000009e880007
:10da4c00e6c2bf000038a3008a003a006db4a800fb
:10da5c00e0012000f09d88007354e2008b003d0033
:10da6c003c13e200580134003c33ed0073d4bf008a
:10da7c000048a30003003a0070d4bf000068a30064
:10da8c0047013a00414621009140780000c8b3009c
:10da9c0000c060009a0032006a14e20009013a00ea
:10daac004173ec0041d3bf000080fb004201200019
:10dabc00110009000280d8000104e000db003200f4
:10dacc001134210091407800c0c3b30080cf5000c6
:10dadc0012013200c942e2008c0035004273ec00a6
:10daec0042d3bf000080fb0042012000110009005e
:10dafc000280d8000104e000c50032006ed4bf00e3
:10db0c000038a300bb00320042d3bf00f44f5000da
:10db1c00330132002134210091407800c0c3b3009e
:10db2c0080cf500004013200c233ec00109e800004
:10db3c00e50f50007a003400c233ef00e8c8bf0094
:10db4c00e14f5000d30032006a300700a0c8bf007c
:10db5c00e14f50000b0132006954e2009d0035008a
:10db6c006854e2009e00350069d4bf000008a30091
:10db7c0092003a0069d4bf000018a30093003a0049
:10db8c0070d4bf000008a3002d0032007014a9004f
:10db9c007354e2002700350070d4bf000018a300b6
:10dbac000e003200d5c2bf000028a3000b003a00c3
:10dbbc002c08e20039013a007034a90064d4bf008b
:10dbcc000058a3003a013a006a74a8005c94a900ba
:10dbdc005cb4a9005cd4a8005cf4a8006cd4bf00b1
:10dbec000018a30013003200ce13e200050034002d
:10dbfc00ce33ed00ce13e20002003a007334a800dd
:10dc0c006c34a90069d4bf000068a300090032007d
:10dc1c00709e8000801f780020ce2a00801f780024
:10dc2c006e805700d4d007006e8057004a2b070037
:10dc3c00e48757006dd4bf000038a3009d003a0064
:10dc4c000080fa00000006007594a800d5c2bf0041
:10dc5c000028a30077ff3200c033ed00c013e200b0
:10dc6c0077ff3a006dd4a900e6c2bf000038a300cc
:10dc7c0076ff3200c033ed00c013e20076ff3a00ad
:10dc8c006db4a9007354e20075ff35005ef4a90071
:10dc9c0064d4bf000008a30079003a0064d4bf002c
:10dcac000018a30071003a0064d4bf000068a30000
:10dcbc0069003a0073d4bf000008a30071ff320062
:10dccc0064d4bf000058a3006eff3a005e74a90034
:10dcdc006a74a8005c94a9005cb4a9005cd4a80088
:10dcec005cf4a8000000eb0024260700414621004c
:10dcfc009140780000c8b30000c0600066ff3a0095
:10dd0c0041f3b700c942e20074ff3d004273ef00db
:10dd1c00c233ec00109e8000e50f500086ff3c00e3
:10dd2c00119e8000e18f50008a003200109e80000e
:10dd3c00e20f5000cb003200109e8000e30f500029
:10dd4c00be003200109e8000e40f5000c50032006f
:10dd5c00109e8000e50f50007fff3a0034c8bf00d2
:10dd6c00e14f50007cff3a003548e2007aff3a0060
:10dd7c0036e8b700f01d07006954e20078ff3d005b
:10dd8c00140037007574a90021ff370074f4a90042
:10dd9c0018ff37007474a90011ff37007494a900a0
:10ddac000aff370074d4a90003ff37006db4a90033
:10ddbc00f7fe37006dd4a900f0fe370030360700af
:10ddcc0069d4bf000018a3006dff32004a3607006b
:10dddc006bff3700e63507006854e20062ff3d0038
:10ddec000936070069d4bf000008a30061ff3200a8
:10ddfc00f2ff37006e74a80080a48000609e88003b
:10de0c0042d3bf00f44f500042ff3a007400370079
:10de1c00cae2a80020032000c09e88006ed4bf0078
:10de2c000038a30038ff3a00f2ff3700cae2a8001e
:10de3c0020032000c09e88001134210091407800fe
:10de4c00c0c3b30080cf500022ff3a00330037002c
:10de5c007374a900d3fe37006e94a80073d4bf006e
:10de6c000008a30007ff320095ff37006eb4a8002e
:10de7c0064d4bf000068a3008eff3200f6ff3700a9
:10de8c006ed4a80064d4bf000018a30086ff320033
:10de9c00f6ff3700e948e2002bff3a00eae8b7004a
:10deac005e2a0700a0c8bf00e14f50002aff3a00cd
:10debc00340037005afc07000080fa00000006000e
:10decc0061ff3700cae2a80020032000c09e880032
:10dedc00cb62a800cb82a8007394a9006a34ef002f
:10deec005c94a8005cb4a9005cd4a9005cf4a90003
:10defc005a54a800b03607004173ec0041d3bf0060
:10df0c000080fb0042012000110009000280d800b3
:10df1c000104e000eafe3a00c4ff3700e833ef00ea
:10df2c0031062000409f8000810f5000fdff36001d
:10df3c000000fe00e7fe3700e833ef00310620005a
:10df4c00409f8000810f5000fdff36000000fe0056
:10df5c00f5fe37007cc8bf00e14f5000fefe3a00d2
:10df6c007d48e200fcfe3a008000fd007ee8b70030
:10df7c008000fd00961d07006954e200f8fe3d008c
:10df8c0094ff3700a148e200f3fe3a00a2e8b70084
:10df9c003f1d07006954e200f1fe3d008dff370084
:10dfac002c13e200b7fe34002c33ed002c13e200ee
:10dfbc00b4fe3a006e74a80070d4a900e0cc2a001c
:10dfcc00212b0700affe37005e54e2002f003d000e
:10dfdc005ef4a90090002000e0998800a3fe3700b1
:10dfec00cb62a800cb82a8007394a9006a34ef001e
:10dffc005c94a8005cb4a9005cd4a9005cf4a900f2
:10e00c005a54a8006c36070073d4bf000008a30054
:10e01c00c0fe32007314a9005e74a9000000eb006e
:10e02c00562507002134210091407800c0c3b3006d
:10e03c0080cf5000bcfe3a00bfff370058c8bf006d
:10e04c00e14f5000c4fe3a005948e200c2fe3a00cb
:10e05c005ae8b700711d07006954e200c0fe3d008c
:10e06c005cff3700c4c8bf00e14f5000bafe3a0055
:10e07c00c548e200b8fe3a00c6e8b700002a07001f
:10e08c006954e200b6fe3d0052ff37005ef4a80072
:10e09c0010002000e099880074fe37002c28ed0059
:10e0ac006cd4bf000018a300e2fe3200cefe370095
:10e0bc007314a8005e74a800100020002f25070020
:10e0cc005c94a8005cb4a9005cd4a8005cf4a90022
:10e0dc006cd4bf000018a300d6fe3200c2fe37007d
:10e0ec004f02b000889fbe008a9fbe008c9fbe006e
:10e0fc008e1f78007134a9006066b8000000eb0038
:10e10c00f0b79f00e9342100390478000907780042
:10e11c006140b90019cb07000800e000b7003500da
:10e12c000001be000c00be0083ca07000005be0043
:10e13c007fb097000000e80080bf9f0019047800b2
:10e14c008e84e8006140b9000ccb07000800e000a9
:10e15c00ba0035000001be000a00be0076ca0700f6
:10e16c000005be0019047800e40447006140b900c2
:10e17c0002cb07000800e000bd0035000001be0026
:10e18c000a00be006cca07000005be001904780026
:10e19c00e60447006140b900f8ca07000800e00037
:10e1ac00c00035000001be000a00be0062ca0700b4
:10e1bc000006be0019047800e80447006140b9006d
:10e1cc00eeca07000800e0007e0035000001be002a
:10e1dc000c00be0058ca07000005be000006be00b9
:10e1ec000fb8970064004000f0b79f00fe0f50007e
:10e1fc00c5ff3a0002002000031f24000a00be00e5
:10e20c000aca0700020020006351240049ca070013
:10e21c0012c9210063bf2300a4ca0700020020001a
:10e22c004319240044ca07000200200003122400f2
:10e23c009eca0700509a8800619a8800f0a380005b
:10e24c00589a8000699a8000cf80de00cbca070004
:10e25c000801be00f4ca07000000e000050034000d
:10e26c006af4a8005c94a9005cb4a9005cd4a80072
:10e27c005cf4a90068d4bf000068a30097003a00c2
:10e28c00509a8000619a800002002000a33724007d
:10e29c00e5ca07000000e000aa003d00509a80008b
:10e2ac00619a80000200200053372400deca070068
:10e2bc000000e000b1003d00509a8000619a80009f
:10e2cc000200200003372400d7ca07000000e0003a
:10e2dc00c6003d00509a8000619a80000200200028
:10e2ec0063362400d0ca07000000e000cd003d00da
:10e2fc00509a8000619a800002002000c3352400ef
:10e30c00c9ca07000000e000aa003d00509a800036
:10e31c00619a80000200200023352400c2ca070045
:10e32c000000e000cd003d00509a8000619a800012
:10e33c000200200083342400bbca07000000e00068
:10e34c00e2003d00509a8000619a8000020020009b
:10e35c00e3332400b4ca07000000e000cd003d0008
:10e36c00cae2a800a0002000c09e880000c0eb00fc
:10e37c00990e07004433ec00209a8000fd0f5000ea
:10e38c0006003400cae2a80040062000c09e8800a7
:10e39c0075f4a900e0012000209a8800930e070074
:10e3ac00e922a80000000000e922a9004f0778002c
:10e3bc004f06be004f05be004f04be004f02b10019
:10e3cc00000006000200200003782400dac90700d0
:10e3dc000001be000c00be00d7c907000005be003e
:10e3ec000006be000fb8970064004000f0b79f0015
:10e3fc00fe0f500044ff3a007eff37000200200061
:10e40c0003782400ccc907000001be000c00be003c
:10e41c00c9c907000005be007fb097000000e800e6
:10e42c0080bf9f00190478008e84e8006140b90019
:10e43c0052ca07000800e00046ff3d000200200021
:10e44c0003782400bcc907000001be000a00be000e
:10e45c00b9c907000005be0019047800e4044700a0
:10e46c006140b90045ca07000800e00043ff3d00c9
:10e47c000200200003782400afc907000001be0091
:10e48c000a00be00acc907000005be0019047800e4
:10e49c00e60447006140b90038ca07000800e000f4
:10e4ac0040ff3d000200200003782400a2c90700b1
:10e4bc000001be000a00be009fc907000006be0096
:10e4cc0019047800e80447006140b9002bca070022
:10e4dc000800e0003dff3d00baff370090ce2a0057
:10e4ec0003290700729c8000509a8000619a80007a
:10e4fc00821f780002002000031224004bc9070081
:10e50c00809fbe00f0ce2a00801f780080fc2f0078
:10e51c000f00400098ce070080fc2f000f00400039
:10e52c00f3280700e8875700509a8000619a800012
:10e53c0002002000a33724003bca07000000e000c3
:10e54c0056ff35000040eb00230e07004433ef006c
:10e55c00260e0700e922a80000000000e922a9000d
:10e56c004f0778004f06be004f05be004f04be009b
:10e57c004f02b1000000060092ff370000c8b30044
:10e58c00150e07004433ef00180e0700e922a8000f
:10e59c0000000000e922a9004f0778004f06be00da
:10e5ac004f05be004f04be004f02b1000000060034
:10e5bc0084ff370000cfb300070e07004433ef0091
:10e5cc000a0e0700e922a80000000000e922a900b9
:10e5dc004f0778004f06be004f05be004f04be002b
:10e5ec004f02b1000000060076ff370000ccb300ec
:10e5fc00f90d07004433ef00fc0d0700e922a800d9
:10e60c0000000000e922a9004f0778004f06be0069
:10e61c004f05be004f04be004f02b10000000600c3
:10e62c0068ff370000ceb300eb0d07004433ef005a
:10e63c00ee0d0700e922a80000000000e922a90065
:10e64c004f0778004f06be004f05be004f04be00ba
:10e65c004f02b100000006005aff370080cfb30014
:10e66c00dd0d07004433ef00e00d0700e922a800a0
:10e67c0000000000e922a9004f0778004f06be00f9
:10e68c004f05be004f04be004f02b1000000060053
:10e69c004cff3700e0cfb300cf0d07004433ef0041
:10e6ac00d20d0700e922a80000000000e922a90011
:10e6bc004f0778004f06be004f05be004f04be004a
:10e6cc004f02b100000006003eff3700c0cfb30080
:10e6dc00c10d07004433ef00c40d0700e922a80068
:10e6ec0000000000e922a9004f0778004f06be0089
:10e6fc004f05be004f04be004f02b10000000600e3
:10e70c0030ff3700889fbe007314a9007034a90035
:10e71c002c28ef002e68ef005e74a9000000eb00bf
:10e72c0096230700e633ef00931b07000004eb0071
:10e73c0088047800dc0c07001f003a00dd0c070091
:10e74c0020003a00de0c070021003a00df0c070025
:10e75c0022003a006ad4bf00e140600023003a0076
:10e76c00e20f540021003c002ec8bf000028a3007b
:10e77c00030032000804e800010078002ee8b7001e
:10e78c00319f8000301f2000808f5000e9ff340043
:10e79c00e633ef008904e80080022000808f5400eb
:10e7ac0012003c00f48f540012003200721b070060
:10e7bc00bd0c0700e1ff32005e290700bd0c07000d
:10e7cc00e0ff32000e2b0700bd0c0700dfff32000c
:10e7dc0043fe0700bd0c0700deff320060fc0700a3
:10e7ec006ad4bf00e1406000ddff32004f04be0080
:10e7fc00000006000000eb00602307005e1b070012
:10e80c00ebff37005c94a9005cb4a9005cd4a800b1
:10e81c005cf4a900aa33ef00a833ef00860c0700c4
:10e82c0015003a00a70b07003a003200e10c070074
:10e83c000e003a0062d4bf000048a30002003a0068
:10e84c0010c0b30016e8b7004a0b070002003a00ec
:10e85c0020c0b30016e8b700650b070002003a00b1
:10e86c0030c0b30016e8b700450b0700780c070062
:10e87c0001003400790c07007354e20034003d00b1
:10e88c0073d4bf000038a3003100320073d4bf0032
:10e89c000028a3002e003a00ba0c07002c003a0006
:10e8ac00bb0c07002a003a007f0c070012003a004c
:10e8bc00800c070013003a00870c070009003a008f
:10e8cc00820c07000a003a00c942e20003003d0036
:10e8dc006ed4bf000038a300d0ff320073f4a9003f
:10e8ec00ceff3700053e0700780c0700f6ff32001c
:10e8fc001bfc0700f4ff37000e2907006d0c070006
:10e90c00edff3200be2a0700730c0700ecff32004b
:10e91c00f4ff370062d4bf000008a30002003a00e5
:10e92c0010c0b30017e8b700500c070002003a0003
:10e93c0020c0b30017e8b7004f0c070002003a00e4
:10e94c0030c0b30017e8b7004e0c0700c7ff370004
:10e95c007394a9007354e20001003d009b0c070066
:10e96c000000060073d4bf00644060000900320050
:10e97c00f00a07003600320030003400d0c4b30077
:10e98c0080cf50004c003200560c0700540032006f
:10e99c000000060017e8b70016e8b70018e8b70043
:10e9ac0073d4bf000028a30012003200280c07000b
:10e9bc000e003c00260c07003000320018c8bf00c7
:10e9cc00e14f5000f2ff3c00da0a07002000320051
:10e9dc00690c0700380032006540500080cf5000b1
:10e9ec001800320090a48000170037007394a80020
:10e9fc0000000600330b0700170032006d0c0700f7
:10ea0c0008003a0062d4bf000048a3003100320075
:10ea1c00d80a07002c003200f50a07002800320043
:10ea2c00d70a07000a0c0700e0ff34000b0c0700a4
:10ea3c00070c0700dfff3400ecff37002c0c07003d
:10ea4c00d3ff3a00c0a48000709d8800000006002f
:10ea5c00a0a48000fcff370062d4bf000008a30014
:10ea6c0029003200010c070022003200020c0700c2
:10ea7c001c003200030c0700eaff37005c94a8006e
:10ea8c005cb4a9005cd4a800ad0a070005003200f4
:10ea9c00390c0700210032006540500080cf500037
:10eaac0020003200a0a480002200200011000900e8
:10eabc000200d800e4ff3700b0a48000e2ff37006a
:10eacc00960a0700d7ff3700970a0700d4ff3a00d1
:10eadc00fbff37008e0a0700cfff3a00faff370022
:10eaec00c0ff370030c0b30017e8b700e50b0700d4
:10eafc00ccff370020c0b30017e8b700de0b0700cf
:10eb0c00dcff3a00f7ff370010c0b30017e8b7007e
:10eb1c00d60b0700d5ff3a00f6ff3700b0a48000f3
:10eb2c00e1ff3700c0a48000dfff3700f30b0700c4
:10eb3c0003003a0073d4bf000048a3000800320061
:10eb4c00cc13e20017003400cc33ed00ac13e20020
:10eb5c000100350000000600ac33ef000000060099
:10eb6c0080ff07006d54e200f8ff3d00e70b070043
:10eb7c0032003200619d8000709d8000808f5000bb
:10eb8c002a003500619d8000709d8000808f5000b0
:10eb9c00eeff3400ac33ed00ac13e200edff3d00b2
:10ebac00edff370080a48000609e8800619d80008e
:10ebbc0020032000808f500008003400619d8000ed
:10ebcc00509e8000808f500011003c00ac33ef0051
:10ebdc00ac13e200dfff3d00dfff370073d4bf0052
:10ebec000048a30006003a0073f4a900b0cf2a0035
:10ebfc0059270700ac13e200d6ff3d00d6ff3700c3
:10ec0c0000ff0700ac13e200d2ff3d00d2ff37003b
:10ec1c00609d8000519e800001005000609d880026
:10ec2c00ac13e200cbff3d00cbff3700ac33ec0064
:10ec3c00ac13e200c7ff3d00c7ff3700709d80009a
:10ec4c00619d800023002000811f780011000900c5
:10ec5c000300d800cf007800810f5000f3ff3c0078
:10ec6c00709d8000619d8000811f7800110009005b
:10ec7c000300d800cf007800810f5000c5ff35008d
:10ec8c00ac13e200b3ff3d00b3ff3700881f7800e0
:10ec9c00d00a070036003500580a070001003c0076
:10ecac000001eb00808f510001003c008001eb0063
:10ecbc00d70a07000100340000017800808f510052
:10eccc0001003400800178000200e00002003a00ec
:10ecdc000300e000170032004e0a07001b00320050
:10ecec0080cf500007003600280a070008003200c9
:10ecfc007c0b070006003200850a07004f047800e1
:10ed0c00000006006440500080cf5000faff3a002b
:10ed1c00939f8800829f8800909f8000b00e88008f
:10ed2c00809f8000d00e88004f0478000000060001
:10ed3c00f4ff3700dc62a900d13d2100914078003e
:10ed4c0060c4b30080cf5000e5ff3a00929f88006a
:10ed5c00839f8800909f8000b00e8800809f800069
:10ed6c00d00e88004f04780000000600e5ff370045
:10ed7c0002002000037824006fc70700c6ff37008d
:10ed8c001e00fa00889fbe008a1f7800800478005d
:10ed9c000104780002057800e633ef008001eb00f7
:10edac0010032000808f540001003400890178008a
:10edbc000001eb0010032000800f54000100340010
:10edcc0008017800c0d42100808f5100010034006c
:10eddc0080017800800f51000100340000017800a0
:10edec000300e0006a003a000200e00068003a000c
:10edfc008a0a07006c00320080cf50003e003e00b3
:10ee0c003b0b070042003200410a0700309f800094
:10ee1c008a0f500047003e006d54e2001000350090
:10ee2c007354e20063003d00560b070061003a008a
:10ee3c00570b07005f003a001b0b070029003a0034
:10ee4c001c0b070022003a00200b07001b003a00a5
:10ee5c001b0b0700d1ff3200a1fc0700cfff3700ce
:10ee6c00e09c8000801f7800b0d22a00801f7800c0
:10ee7c0080fd2f000f0040003fcc0700e19c80007c
:10ee8c00e487570040a12000808f5000e4ff3c0035
:10ee9c00e19c8000b0942000808f5000e0ff340093
:10eeac00800c200065320700100020004f05780010
:10eebc004f04be000080fa0000000600a8fa07000c
:10eecc0071d4bf000018a300b4ff3200e2ff37007a
:10eedc004b29070071d4bf000058a300dcff32009f
:10eeec00f6ff37009327070071d4bf000038a3004a
:10eefc00d5ff3200f6ff3700c0c4b30080cf5000fe
:10ef0c00030032006640400080cf5000beff3a0044
:10ef1c00929f8800839f8800909f8000b00e88008d
:10ef2c00809f8000d00e8800309f80008a0f500098
:10ef3c00b9ff3600dc62a900d13d21009140780078
:10ef4c0060c4b30080cf5000260032001f003e008a
:10ef5c006440500080cf500022003200909f80000f
:10ef6c00b00e8800809f8000d00e880073f4a9003a
:10ef7c0020d12a00782607000000eb004f0578000e
:10ef8c004f04be000080fa0000000600cbff3700e3
:10ef9c00dc62a800d13d21009140780060c4b30030
:10efac0080cf500094ff3a00939f8800829f880086
:10efbc0095ff37000000eb004f0578004f04be00b2
:10efcc000080fa0000000600bcff3700c0c4b3008c
:10efdc0080cf5000030032006640400080cf5000cc
:10efec00deff3a00f233ef00f033ef00909f800029
:10effc00b00e8800809f8000d00e880073f4a900aa
:10f00c0020d12a00542607000000eb00dbff37005c
:10f01c00881f7800c20a070070d32a004e2607000a
:10f02c00000a0700050a0700210032001a003e0002
:10f03c0020c4b30080cf50001d003200040a07002a
:10f04c000c003a009b0a07000e003a009f0a0700ca
:10f05c0006003a006d0a0700f2ff3200c90a0700e9
:10f06c00f0ff3a004f047800000006003cfa07005d
:10f07c00f8ff37002f27070071d4bf000038a3001a
:10f08c00f2ff3200de28070071d4bf000058a30045
:10f09c00f0ff3200f5ff3700c0c4b30080cf500042
:10f0ac00030032006640400080cf5000e3ff3a007e
:10f0bc00f233ef00f033ef00909f8000b00e880029
:10f0cc00809f8000d00e880071d4bf000048a30040
:10f0dc00dcff3200e7ff3700881f7800900a07003a
:10f0ec0040d42a001c260700ce090700d3090700cc
:10f0fc00220032001b003e0020c4b30080cf500021
:10f10c001e003200d20907000d003a00690a070000
:10f11c000f003a006d0a070004003a009c0a070031
:10f12c00f2ff3a004f047800000006000cfa0700ca
:10f13c006ad4bf000018a300ecff3a00f9ff3700b7
:10f14c00fc26070071d4bf000038a300f1ff320089
:10f15c00ab28070071d4bf000058a300efff3200aa
:10f16c00f2ff3700c0c4b30080cf50000300320060
:10f17c006640400080cf5000e2ff3a00f233ef00cf
:10f18c00f033ef00909f8000b00e8800809f8000cd
:10f19c00d00e880071d4bf000048a300dbff320002
:10f1ac00e7ff37000c00fa00889fbe008a9fbe0064
:10f1bc008c9fbe001909070041003400340a070077
:10f1cc001809070030003400a4090700a80907003b
:10f1dc001f003400d3090700d709070001003c00c9
:10f1ec000001eb00808f510001003c008001eb001e
:10f1fc00870907000100340000017800808f51005e
:10f20c0001003400800178000200e00002003a00a6
:10f21c000300e00040003200fe080700440032000a
:10f22c0080cf50002d003600d80807002e00320089
:10f23c002c0a07002c003200cc0907004f06be0038
:10f24c004f05be004f04be000080fa00000006000f
:10f25c0060a0800071a08000a2a08000b3a08000fc
:10f26c0003f0a200f2c607000000e000daff3d0048
:10f27c00a0a08000b1a0800001f0a20060a08800d6
:10f28c0071a08800d4ff370020a0800031a080003e
:10f29c00a2a08000b3a0800003f0a200e4c6070087
:10f2ac000000e000c9ff3d00a0a08000b1a08000dc
:10f2bc0001f0a20020a0880031a08800c3ff370015
:10f2cc000801be000800be0078c60700020020003e
:10f2dc00a32f2400d5c50700b9ff370064405000a8
:10f2ec0080cf5000d4ff3a00939f8800829f880003
:10f2fc00919f8000b10e8800849f8000d40e8800fe
:10f30c004f06be004f05be004f04be000080fa0041
:10f31c0000000600ceff3700dc62a900d13d2100c1
:10f32c009140780060c4b30080cf5000bcff3a001d
:10f33c00929f8800839f8800919f8000b10e880067
:10f34c00849f8000d40e88004f06be004f05be007f
:10f35c004f04be000080fa0000000600bcff37001e
:10f36c00e609070003003200cc13e200450034002c
:10f37c00cc33ed008209070023003d00aa33ec00da
:10f38c00830907001a003d00a833ec00820807002f
:10f39c0001003c000001eb00808f510001003c009b
:10f3ac008001eb001a09070001003400000178000d
:10f3bc00808f510001003400800178000200e000d1
:10f3cc0002003a000300e000200032009108070020
:10f3dc002400320080cf5000110036006b0807006b
:10f3ec0012003200bf09070010003200f1f637009e
:10f3fc00419d8000609d8000808f5000e3ff3400b1
:10f40c00a833ed00e1ff3700519d8000609d800026
:10f41c00808f5000daff3400aa33ed00d8ff37009c
:10f42c006440500080cf5000f0ff3a00939f88005a
:10f43c00829f8800909f8000b00e8800809f800083
:10f44c00d00e880000000600e9ff3700dc62a9003e
:10f45c00d13d21009140780060c4b30080cf5000b2
:10f46c00dcff3a00929f8800839f8800909f800069
:10f47c00b00e8800809f8000d00e8800000006002f
:10f48c00dbff370080a48000609e8800619d8000b7
:10f49c0020032000808f500009003400619d800003
:10f4ac00509e8000808f5000b2ff3400609d800021
:10f4bc00519e800001005000609d8800adff370018
:10f4cc0030d52a002425070073f4a900a9ff3700c2
:10f4dc0033090700220032007074a900519d80008e
:10f4ec00309d8000808f500050003d00aa33ec000e
:10f4fc00419d8000209d8000808f500052003d0077
:10f50c00a833ec002408070001003c000001eb00cc
:10f51c00808f510001003c008001eb00bc0807000b
:10f52c000100340000017800808f5100010034008c
:10f53c00800178000200e00038003a000300e0008f
:10f54c0036003a00b50807003600320080cf500074
:10f55c002c003e00660907002e0032006c080700e4
:10f56c006cd4bf000028a3001f003a005409070008
:10f57c0020003a00580907000e003a004a0907001b
:10f58c0015003a004b0907000e003a004f0907001e
:10f59c000f003a007b09070005003a007c090700c0
:10f5ac0003003a0070d4bf000048a300c8ff3a0023
:10f5bc0000000600d13a07003b090700f1ff3200ba
:10f5cc00050037008e27070040090700f1ff3200c5
:10f5dc00e3f80700efff3700d625070035090700d1
:10f5ec00eaff3200f7ff3700aef4070034090700da
:10f5fc00e0ff3200bafa070037090700dfff3200dc
:10f60c00ecff3700e1070700020032003509070064
:10f61c00d2ff3a00e5070700d1ff3700fd070700ce
:10f62c00caff3a00e1080700cdff3700aa13e20039
:10f63c00afff3400aa33ed00419d8000209d800077
:10f64c00808f5000aeff3500a813e200adff3400f0
:10f65c00a833ed00abff3700889fbe008a9fbe0029
:10f66c008004780070f4a90070d4a9002200200056
:10f67c00110009000200d80000047800aa33ef0042
:10f68c00a833ef00c407070001003c000001eb00a9
:10f69c00808f510001003c008001eb005c080700ea
:10f6ac000100340000017800808f5100010034000b
:10f6bc00800178000200e00002003a000300e00044
:10f6cc00c1003200d3070700c100320080cf5000c8
:10f6dc009c003600ad0707009c00320001090700b2
:10f6ec009a003200b40707009c00320020c5b3001a
:10f6fc00ddf3b700dc02a800dc82a800e433ef00e5
:10f70c00e833ef00b112200013090700feff3600aa
:10f71c003ac5b300909e8000ea0f50003a003c00be
:10f72c00209f8000800f540002003d006e74a800e2
:10f73c005ac4b3007354e200f5003d0011090700f0
:10f74c00b2003a0012090700b0003a00d6080700d0
:10f75c0093003a00d70807008a003a00d80807003f
:10f76c008b003a00d908070084003a008c08070087
:10f77c00e8ff3200e108070003003200cc13e2007e
:10f78c00a6003400cc33ed007d0807009b003d0043
:10f79c00aa33ec007e08070094003d00a833ec006f
:10f7ac007d07070001003c000001eb00808f510039
:10f7bc0001003c008001eb0015080700010034003b
:10f7cc0000017800808f5100010034008001780026
:10f7dc000200e00081003a000300e0007f003a00e4
:10f7ec000e0807007f00320080cf500070003e00f2
:10f7fc00bf08070072003200c5070700909e80000a
:10f80c00ea0f5000c6ff340068d4bf000028a300e4
:10f81c00fa003a0068080700319e8000029b200025
:10f82c0001045100309e80008005410050d72a0011
:10f83c0049240700809e8000e20f5000090034002c
:10f84c00e09c8000800f540006003d00e09c80008e
:10f85c00808f550003003400570807006e74a80011
:10f86c00fac4b300209f8000808f540002003d003a
:10f87c006e74a8005ac4b3007354e20076003d00c5
:10f88c00c008070061003a00c10807005f003a0099
:10f89c0085080700a3003a0086080700ac003a0070
:10f8ac0087080700a4003a0088080700a6003a0061
:10f8bc003b080700dfff320090080700030032000e
:10f8cc00cc13e200de003400cc33ed002c08070032
:10f8dc00c4003d00aa33ec002d080700bb003d001e
:10f8ec00a833ec002c07070001003c000001eb00e2
:10f8fc00808f510001003c008001eb00c407070021
:10f90c000100340000017800808f510001003400a8
:10f91c00800178000200e0009f003a000300e00044
:10f92c009d003a00bd070700a100320080cf5000b7
:10f93c008c003e006e080700900032007407070030
:10f94c00bcff37006a08070066ff3a00939f8800e7
:10f95c00829f88001807070064ff3a0001007800b6
:10f96c00ddf3b700dc02a900dc82a900e433ef0070
:10f97c00e833ef00b112200063ff3700f8f70700ff
:10f98c007aff37009e2607004d08070075ff3200ee
:10f99c00d3f907004d08070074ff3200f7ff37005a
:10f9ac00e4240700430807006cff3200f5ff370022
:10f9bc00f6060700020032004a0807008eff3a00e4
:10f9cc00fa0607008dff3700940707003fff3a0047
:10f9dc00929f8800839f880042ff37000d07070025
:10f9ec0081ff3a00f107070084ff3700e8070700a2
:10f9fc006bff3400a833ed0069ff3700e007070008
:10fa0c0064ff3400aa33ed0062ff37000000eb0006
:10fa1c004f05be004f04be000000060080a480000d
:10fa2c00609e8800619d800020032000808f500024
:10fa3c007f003400619d8000509e8000808f5000bc
:10fa4c0051ff3400609d8000519e800001005000e9
:10fa5c00609d88004cff3700aa33ef00a833ef00fd
:10fa6c00439d8000529d800010032000800f5100a8
:10fa7c0001003c000001eb00808f510001003c00b4
:10fa8c008001eb00c0d42100800f51000100340034
:10fa9c0000017800808f5100010034008001780053
:10faac000200e00075003a000300e00073003a0029
:10fabc00dc62a900d13d21009140780060c4b30004
:10facc0080cf50007d0032006e003600c0c4b30001
:10fadc0080cf5000030032006640400080cf5000c1
:10faec0002003a00939f8800829f8800909f8000bc
:10fafc00b00e8800809f8000d00e8800e833ef00a5
:10fb0c00b1122000409f8000810f5000fdff360095
:10fb1c000a80fb004f05be004f04be00000006002b
:10fb2c00beff37008324070071d4bf000038a30048
:10fb3c005bff32000600370069f9070071d4bf0083
:10fb4c000058a3005aff320085f7070058ff370012
:10fb5c002b26070071d4bf000018a30052ff3200ff
:10fb6c00f5ff3700c0c4b30080cf50000300320053
:10fb7c006640400080cf500070ff3a00939f880091
:10fb8c00829f8800909f8000b00e8800809f80002c
:10fb9c00d00e880027ff3700dc62a800d13d210081
:10fbac009140780060c4b30080cf50005fff3a00f2
:10fbbc00929f8800839f8800909f8000b00e8800e1
:10fbcc00809f8000d00e88001aff3700419d800076
:10fbdc00609d8000808f500042ff3400a833ed0000
:10fbec0040ff3700519d8000609d8000808f500049
:10fbfc0039ff3400aa33ed0037ff370090d62a00c6
:10fc0c0055230700cae2a80040062000c09e8800c9
:10fc1c00319e8000029b200001045100309e800028
:10fc2c008005410050d72a004b23070001ff370005
:10fc3c0030d52a004823070073f4a900d2fe370000
:10fc4c0080a48000609e8800619d800020032000bd
:10fc5c00808f500015003400619d8000509e800004
:10fc6c00808f500019ff3400609d8000519e8000f1
:10fc7c0001005000609d880014ff3700dc62a80072
:10fc8c008cff37006440500080cf500095ff32004d
:10fc9c00909f8000b00e8800809f8000d00e88005e
:10fcac00e833ef00b112200096ff370030d52a0060
:10fcbc002923070073f4a90004ff3700929f8800e2
:10fccc00839f8800909f8000b00e8800809f8000ea
:10fcdc00d00e8800e833ef00b112200089ff370006
:10fcec00881f78008f06070019003a000004eb000b
:10fcfc00e833ef00409f8000e90f5000fdff360015
:10fd0c00ea0f540007003400af0607000a00320067
:10fd1c003a0707003d07070010003a0043070700a9
:10fd2c00c92307007f06070009003a000804e80011
:10fd3c00e833ef00efff37006d54e200f5ff3500bc
:10fd4c0035070700c023070076060700f7ff3200cf
:10fd5c000000eb004f047800000006006a34ef004e
:10fd6c0073f4a800100020004f0478000000060077
:10fd7c00faff370050d82a00f722070073d4bf00cf
:10fd8c000058a3000a003a00420607000a003a0095
:10fd9c006d54e20012003d001c0707000900320000
:10fdac00630607006d060700feff36006f060700ae
:10fdbc006e14a900000006001007070013070700c7
:10fdcc00f7ff3a00190707009f230700e833ef00fd
:10fddc0062060700feff36006906070000000600f9
:10fdec000d07070098230700e833ef00f8ff3700f2
:10fdfc007334a9007406070005003200ff060700e3
:10fe0c00020707000b003200620607000000060024
:10fe1c006d54e200faff3500ff0607008a23070045
:10fe2c00600607004c070700feff3600600607005f
:10fe3c00c9223700fd060700832307005906070077
:10fe4c00f8ff3700881f7800cb82a800cb62a8008f
:10fe5c004407070067003200470707006d003200b7
:10fe6c006740500080cf50007d00320073d4bf003b
:10fe7c000008a30034003a00540707007334a900ab
:10fe8c006c34a90073d4a9006e74a9007094a900f5
:10fe9c0073b4a9004f06070052003500d7050700c0
:10feac0001003c000001eb00808f510001003c0080
:10febc008001eb00560607000100340000017800b9
:10fecc00808f510001003400800178000200e000b6
:10fedc0002003a000300e00039003200cd050700b3
:10feec003d00320080cf500011003600a7050700fe
:10fefc0012003200fb060700100032002f0607002c
:10ff0c000008a30002003a00000707004900320075
:10ff1c00e0da2a004c23070020032000609d8800b3
:10ff2c00509d8800409d88004f047800000006001a
:10ff3c006440500080cf5000f0ff3a00939f88003f
:10ff4c00829f8800edff3700eef907005c94a80053
:10ff5c005cb4a9005cd4a9005cf4a9007334a900ba
:10ff6c006c34a90073d4a9006e74a9007094a90014
:10ff7c0073b4a900ac33ef00aa33ef00a833ef0041
:10ff8c000034ef000234ef000834ef000a34ef00c5
:10ff9c00fc33ef00fe33ef000434ef000634ef00c7
:10ffac000c34ef000e34ef0038a480006140b9002f
:10ffbc0072c307000800e000b8ff3d0009003700dd
:10ffcc00dc62a900d13d21009140780060c4b300ef
:10ffdc0080cf5000c3ff3a00929f8800839f880017
:10ffec00c6ff37000200200003782400d2c20700ad
:10fffc00aaff3700caa2a800cac2a90070b82a007a
:020000040001f9
:10000c005522070073d4bf000008a3009aff3200ea
:10001c00cdff3700caa2a800cac2a80000b92a00a6
:10002c004d22070073d4bf000008a30092ff3200da
:10003c00c5ff37006740500011f50700e0da2a00d1
:10004c000123070020032000609d8800509d88003c
:10005c00409d88004f04780000000600b4ff370074
:10006c00caa2a900cac2a800e0b72a003a22070017
:10007c0073d4bf000008a3007fff3200b2ff37002b
:10008c00881f780085050700340035005b050700e4
:10009c0001003c000001eb00808f510001003c008e
:1000ac008001eb00da050700010034000001780044
:1000bc00808f510001003400800178000200e000c4
:1000cc0002003a000300e0001b003200510507005b
:1000dc001f00320080cf5000110036002b050700a6
:1000ec00120032007f06070010003200b305070033
:1000fc000068a300060032006b05070024003200e4
:10010c006b0507001900320071d4a900de73ef00f3
:10011c00c0db2a00cc2207004f0478000000060048
:10012c006440500080cf5000f0ff3a00939f88004d
:10013c00829f8800edff3700dc62a900d13d2100d1
:10014c009140780060c4b30080cf5000e1ff3a00ca
:10015c00929f8800839f8800e4ff370002002000f4
:10016c000378240074c20700c8ff37000100780030
:10017c00ddf3b700ddd3bf00dff3b700dc02a9006d
:10018c00dc82a80071d4a900de73ef00e0ff370019
:10019c0001007800ddf3b700ddd3bf00dff3b7005b
:1001ac00dc02a800dc82a90071d4a900de73ef0088
:1001bc00d7ff3700881f7800d233ef00113e2100a3
:1001cc00e10407003f003200460607004f003200f2
:1001dc00401f2000992d07007e05070060003500a8
:1001ec000605070024003400808f51001d003400e8
:1001fc008705070017003c00808f510011003c0060
:10020c000200e00020003200020507002600320048
:10021c0080cf500048003600dc0407004900320053
:10022c0030060700470032003905070073f4a900b7
:10023c006a94a8003a0607000000eb004f0478000f
:10024c0000000600800178000200e000eeff3a009a
:10025c000d00370000017800808f5100e8ff34005a
:10026c00f8ff37008001eb00c0d42100800f510053
:10027c00e1ff3400f7ff37000001eb00808f5100e5
:10028c00dbff3c00f7ff37000300e000deff3a0025
:10029c00dc62a900d13d21009140780060c4b3001c
:1002ac0080cf5000daff3a00929f8800839f88002d
:1002bc00909f8000b00e8800809f8000d00e880038
:1002cc00daff370020a480007f00b9008000d10045
:1002dc0082bb2000c0122000a9fa07008000780021
:1002ec00100020000100e000d4ff3a0073f4a900d4
:1002fc006a94a8005c94a9005cb4a9005cd4a80022
:10030c005cf4a8000000eb00ccff370020a48000b8
:10031c007f00b9000000d10082bb2000c112200078
:10032c0097fa070080007800100020000100e00020
:10033c00eeff3200c1ff37006440500080cf500008
:10034c00b9ff3a00939f8800829f8800909f80009d
:10035c00b00e8800809f8000d00e8800b3ff37005d
:10036c000200200003782400f3c1070002002000e3
:10037c00832c2400adc1070080a0880091a08800c8
:10038c00439d8000529d800010032000800f51007f
:10039c0095ff3c00b8ff3700881f78000d0507005b
:1003ac00930035009504070001003c000001eb00b0
:1003bc00808f510001003c008001eb001405070008
:1003cc000100340000017800808f510001003400de
:1003dc00800178000200e00002003a000300e00017
:1003ec007a0032008b0407007e00320080cf500070
:1003fc00400036006504070041003200b9050700d3
:10040c003f003200c2040700a70407004700320077
:10041c00a70407007e003200de73ef006b040700b8
:10042c004e003200b0dd2a0007220700800c2000ad
:10043c0089fc070000417800f13d210044040700cd
:10044c005000320063040700dc73ef00f0c4b3000b
:10045c00804f51005500320030c5b300804f510021
:10046c009200320073f4a9006a94a800e0e12a001b
:10047c00f5210700e833ef00b1122000b6050700a4
:10048c00feff3600d30407005d0035005b04070057
:10049c0001003c000001eb00808f510001003c008a
:1004ac008001eb00da040700010034000001780041
:1004bc00808f510001003400800178000200e000c0
:1004cc006a003a000300e00068003a00d304070019
:1004dc006c00320080cf500054003e0084050700b1
:1004ec00580032008a04070073f4a9004f04780006
:1004fc00000006006440500080cf5000c1ff3a005d
:10050c00939f8800829f8800909f8000b00e880087
:10051c00809f8000d00e8800e13d21009140780042
:10052c0060c4b30080cf5000b9ff3a0001007800de
:10053c00ddf3b700ddd3bf00dff3b700dc02a800aa
:10054c00dc82a900de73ef00c13d210091407800f0
:10055c00c0c4b30080cf5000b2ff3a00b0dc2a0018
:10056c00b9210700800c20003bfc070000417800fb
:10057c00f13d21009140780060c4b30080cf500061
:10058c00b0ff3a0001007800ddf3b700ddd3bf0007
:10059c00dff3b700dc02a800dc82a900dc73ef00fb
:1005ac00f0c4b300804f5100abff3a006e74a90049
:1005bc0063405000b2f30700c0de2a00a2210700fe
:1005cc00e833ef00b1122000acff3700dc62a90069
:1005dc00d13d21009140780060c4b30080cf500021
:1005ec0082ff3a00929f8800839f880085ff370026
:1005fc0002002000037824004fc1070069ff370078
:10060c0002002000037824004bc107009fff370035
:10061c0001007800ddf3b700ddd3bf00dff3b700d6
:10062c00dc02a900dc82a8007bff3700c0c4b30049
:10063c0080cf5000030032006640400080cf500055
:10064c00a8ff3a00939f8800829f8800909f8000ab
:10065c00b00e8800809f8000d00e880073f4a90033
:10066c004f04780000000600a2ff3700dc62a800ef
:10067c00d13d21009140780060c4b30080cf500080
:10068c0094ff3a00929f8800839f8800909f80007f
:10069c00b00e8800809f8000d00e880073f4a900f3
:1006ac004f0478000000060092ff370073f4a90095
:1006bc0040e02a0064210700e833ef00b11220006b
:1006cc006eff37000c00fa00889fbe008a9fbe00a8
:1006dc008c9fbe00dbfd0700d0030700b90034007f
:1006ec00eb040700cf030700a80034005b040700ed
:1006fc005f040700970034008a0407008e0407008b
:10070c0001003c000001eb00808f510001003c0017
:10071c008001eb003e04070001003400000178006a
:10072c00808f510001003400800178000200e0004d
:10073c0078003a000300e00076003a003704070026
:10074c007a00320080cf500062003e00e8040700bf
:10075c0066003200850407009104070057003a0038
:10076c00919e8000b09e8000808f500042003d0022
:10077c00cd04070044003a00ce04070046003a00be
:10078c00d504070048003a00cd04070032003a00b7
:10079c00ce04070034003a007054e2002c003500ff
:1007ac00f804070025003a00f904070023003a007a
:1007bc007354e200c8ff3500b8030700ad003500e4
:1007cc008e03070093003400808f51008c0034009e
:1007dc000f04070086003c00808f510080003c0015
:1007ec000200e0008f0032008a03070095003200ff
:1007fc0080cf500096003e00bd0407009a003200e6
:10080c00959f8000b50e8800809f8000d00e8800d8
:10081c0071d4bf000068a30006003200a2030700d9
:10082c00ab003200a2030700a000320071d4a90073
:10083c00de73ef00c0db2a00032107004f06be0069
:10084c004f05be004f04be000080fa0000000600f9
:10085c00d1fe0700d2ff370021f6070071d4bf008c
:10086c000058a300ccff32003df407007054e200a6
:10087c00cbff3d00f6ff37004efe070071d4bf00e2
:10088c000048a300bcff32002a21070071d4bf002e
:10089c000038a300baff3200d922070071d4bf0080
:1008ac000028a300b8ff32001436070071d4bf0033
:1008bc000018a300b6ff3200e7ff37009bf80700d3
:1008cc00919e8000b09e8000808f5000a8ff350064
:1008dc00e9ff3700c0c4b30080cf500003003200e2
:1008ec006640400080cf50009aff3a00939f8800ea
:1008fc00829f8800919f8000b10e8800849f8000a9
:10090c00d40e880070d4bf000038a30094ff3200ce
:10091c00eaff3700dc62a800d13d2100914078004d
:10092c0060c4b30080cf500086ff3a00929f8800cd
:10093c00839f8800919f8000b10e8800849f800067
:10094c00d40e880070d4bf000038a30084ff32009e
:10095c00daff370060a0800071a08000a2a08000a8
:10096c00b3a0800003f0a20031c107000000e0003a
:10097c0062ff3d00a0a08000b1a0800001f0a200a9
:10098c0060a0880071a088005cff370020a0800068
:10099c0031a08000a2a08000b3a0800003f0a200d0
:1009ac0023c107000000e00051ff3d00a0a0800023
:1009bc00b1a0800001f0a20020a0880031a0880026
:1009cc004bff37000801be000800be00b7c007008f
:1009dc0002002000a32f240014c0070041ff3700a1
:1009ec00800178000200e0007fff3a000d00370024
:1009fc0000017800808f510079ff3400f8ff370038
:100a0c008001eb00c0d42100800f510072ff340034
:100a1c00f7ff37000001eb00808f51006cff3c00aa
:100a2c00f7ff37000300e0006fff3a00dc62a9001b
:100a3c00d13d21009140780060c4b30080cf5000bc
:100a4c006bff3a00929f8800839f88006cff3700f1
:100a5c00c0c4b30080cf5000030032006640400099
:100a6c0080cf500066ff3a00939f8800829f8800d9
:100a7c0063ff370002002000037824002ec007001b
:100a8c0002002000832c2400e8bf070080a088000f
:100a9c0091a08800439d8000529d8000100320008f
:100aac00800f510048ff3c00daff3700010078004e
:100abc00ddf3b700ddd3bf00dff3b700dc02a90024
:100acc00dc82a80071d4a900de73ef0059ff370057
:100adc0001007800ddf3b700ddd3bf00dff3b70012
:100aec00dc02a800dc82a90071d4a900de73ef003f
:100afc0050ff3700881f780090e32a00961f0700ec
:100b0c0073d4bf000008a30009003a002e030700ad
:100b1c000a003a006d54e2006a003d00bb03070076
:100b2c000c003a00c10307004720070073f4a9002a
:100b3c006e54a9004f04780000000600d233ef0079
:100b4c0040012000b09e8800e0c2bf000068a300f6
:100b5c00f4ff32006a34ef0073f4a8006e74a9003d
:100b6c00c8c4b30008007800dcf3b700800c200088
:100b7c00b9fa07008040780060c4b300ddf3b70019
:100b8c00ddd3bf00dff3b700dc02a800dc82a900d4
:100b9c0073f4a8006e74a900f0c4b30080cf5000a9
:100bac007300320030c5b30080cf500065003200b6
:100bbc0073f4a9006e74a8006a94a800d0e72a0008
:100bcc0021200700e833ef00b1122000409f800085
:100bdc00810f5000fdff3600ac33ef00aa33ef005d
:100bec00a833ef000034ef000234ef000834ef00bc
:100bfc000a34ef00fc33ef00fe33ef000434ef0057
:100c0c000634ef000c34ef000e34ef0038a48000f3
:100c1c006140b90059c007000800e00050003500e1
:100c2c0002002000832c240080bf070080a08800d5
:100c3c0091a08800439d8000529d800010032000ed
:100c4c00800f510001003c000001eb00808f51002f
:100c5c0001003c008001eb00c0d42100800f51004a
:100c6c000100340000017800808f51000100340035
:100c7c00800178000200e00029003a000300e00047
:100c8c0027003a00dc62a900d13d21009140780098
:100c9c0060c4b30080cf50002300320013003e002c
:100cac006440500080cf500016003200909f8000ae
:100cbc00b00e8800809f8000d00e880073f4a900cd
:100ccc009bff370073f4a9006ab4a8005c94a900d8
:100cdc005cb4a9005cd4a8005cf4a80080c62a000f
:100cec00d91f070073f4a90091ff3700c0c4b300eb
:100cfc0080cf5000030032006640400080cf50008f
:100d0c00eaff3a00939f8800829f8800909f8000a2
:100d1c00b00e8800809f8000d00e8800e7ff37005f
:100d2c00dc62a800d8ff3700929f8800839f880060
:100d3c00909f8000b00e8800809f8000d00e8800ad
:100d4c00deff370073f4a9006e74a80030e62a00a9
:100d5c00bd1f0700e833ef00b11220009bff3700e6
:100d6c00020020000378240073bf0700acff37009b
:100d7c006e74a90008407800c1f10700b0e42a00a5
:100d8c00b11f0700e833ef00b11220008fff3700ce
:100d9c00881f780080e92a00ef1e070073d4bf007b
:100dac000008a300030032006e54a9004f04780021
:100dbc000000060066d4bf000008a3004a003a00f9
:100dcc006d54e200d5003d00e0c2bf000068a300f6
:100ddc004b003a006a14a800f0c72a009a1f0700bb
:100dec0073f4a9006e34a900ac33ef00aa33ef0002
:100dfc00a833ef000034ef000234ef000834ef00aa
:100e0c000a34ef00fc33ef00fe33ef000434ef0044
:100e1c000634ef000c34ef000e34ef0038a48000e1
:100e2c006140b900d5bf07000800e000b7003500ed
:100e3c0002002000832c2400fcbe070080a0880048
:100e4c0091a08800439d8000529d800010032000db
:100e5c00800f510001003c000001eb00808f51001d
:100e6c0001003c008001eb00c0d42100800f510038
:100e7c000100340000017800808f51000100340023
:100e8c00800178000200e00002003a000300e0005c
:100e9c0091003200dc62a800d13d21009140780025
:100eac0060c4b30080cf50009100320080cf50005e
:100ebc007f003600c0c4b30080cf50007f003200ea
:100ecc006640400080cf50007c003200909f800034
:100edc00b00e8800809f8000d00e88004f047800f0
:100eec0000000600b3ff3700d233ef0040012000b2
:100efc00b09e8800e0c2bf000068a300b5ff3200be
:100f0c006a34ef0073f4a8006e74a90020c5b30016
:100f1c00dcf3b700800c2000cff90700804078008c
:100f2c0060c4b300ddf3b700ddd3bf00dff3b7005f
:100f3c00dc02a800dc82a900f0c4b30080cf500012
:100f4c00b400320030c5b30080cf5000a600320090
:100f5c0073f4a9006e74a8006a94a800f0ed2a003e
:100f6c00391f0700e833ef00b1122000409f8000ca
:100f7c00810f5000fdff3600ac33ef00aa33ef00b9
:100f8c00a833ef000034ef000234ef000834ef0018
:100f9c000a34ef00fc33ef00fe33ef000434ef00b3
:100fac000634ef000c34ef000e34ef0038a4800050
:100fbc006140b90071bf07000800e00091003500e6
:100fcc0002002000832c240098be070080a088001b
:100fdc0091a08800439d8000529d8000100320004a
:100fec00800f510001003c000001eb00808f51008c
:100ffc0001003c008001eb00c0d42100800f5100a7
:10100c000100340000017800808f51000100340091
:10101c00800178000200e0006a003a000300e00062
:10102c0068003a00dc62a900d13d210091407800b3
:10103c0060c4b30080cf50006400320054003e0006
:10104c006440500080cf500057003200909f8000c9
:10105c00b00e8800809f8000d00e880073f4a90029
:10106c006e34a900ac33ef00aa33ef00a833ef00c5
:10107c000034ef000234ef000834ef000a34ef00c4
:10108c00fc33ef00fe33ef000434ef000634ef00c6
:10109c000c34ef000e34ef0038a480006140b9002e
:1010ac0036bf07000800e00061ff3d001700370065
:1010bc006440500080cf500084ff3a00939f88001a
:1010cc00829f8800909f8000b00e8800809f8000d7
:1010dc00d00e880081ff3700dc62a900d13d2100d1
:1010ec009140780060c4b30080cf50006fff3a008d
:1010fc00929f8800839f8800909f8000b00e88008c
:10110c00809f8000d00e880074ff37000200200002
:10111c000378240088be070045ff370073f4a9004c
:10112c006ab4a8005c94a9005cb4a9005cd4a800c3
:10113c005cf4a80080c62a00c31e070073f4a90043
:10114c006e34a900ac33ef00aa33ef00a833ef00e4
:10115c000034ef000234ef000834ef000a34ef00e3
:10116c00fc33ef00fe33ef000434ef000634ef00e5
:10117c000c34ef000e34ef0038a480006140b9004d
:10118c00febe07000800e00029ff3d00dfff37002e
:10119c00c0c4b30080cf5000030032006640400052
:1011ac0080cf5000a9ff3a00939f8800829f88004f
:1011bc00909f8000b00e8800809f8000d00e880029
:1011cc00a6ff3700dc62a80097ff3700929f8800cb
:1011dc00839f8800909f8000b00e8800809f8000c5
:1011ec00d00e88009dff370073f4a9006e74a80020
:1011fc0040ec2a00941e0700e833ef00b1122000e7
:10120c005aff370002002000037824004abe070072
:10121c006bff37006e74a9006340500098f0070014
:10122c00b0ea2a00881e0700e833ef00b112200054
:10123c004eff3700889fbe00780107001c0032006b
:10124c0017003e002a02070019003200c4000700f4
:10125c001b003a000004eb00e833ef00409f8000d5
:10126c00e90f5000fdff3600ea0f54000700340070
:10127c005501070041003200e0010700e3010700bf
:10128c008d003a00e90107006f1e070025010700d9
:10129c000b003a000804e800e833ef00efff3700da
:1012ac00ba000700020032000e020700e7ff3a0006
:1012bc00f233ef00f033ef00a9000700e5ff320036
:1012cc007354e2005400350070d4bf000048a300f2
:1012dc0055003a002b02070056003a002c0207007a
:1012ec0057003a00f001070058003a00f1010700de
:1012fc0059003a00f501070035003a00f0010700eb
:10130c0040003a006ed4bf000028a30034003a001d
:10131c006ed4bf000018a30035003a006ed4bf0095
:10132c000008a3001a003a0073d4bf000018a300f1
:10133c00070032007334a90023010700510032006a
:10134c00ae010700b1010700600032001101070077
:10135c006ed4bf000068a30045003a006ed4bf00f5
:10136c000058a30040003a006ed4bf000048a30010
:10137c00b1ff3200f5290700afff37006d54e200d2
:10138c00beff3500a40107002f1e0700bfff37006a
:10139c0050d82a00701d070073d4bf000058a3005a
:1013ac0009003a00bb0007004c0032009301070013
:1013bc009601070052003200dd000700e70007002d
:1013cc00feff3600e90007006e14a900d6ff3700b7
:1013dc0063f10700ba010700caff320009003700a9
:1013ec00c4fd07006ed4bf000018a300cbff320071
:1013fc0067fe07006ed4bf000008a300caff3200ce
:10140c00e3ff370036f307006ed4bf000028a300bb
:10141c00bfff3200f2ff3700aafc070070d4bf00f8
:10142c000048a300abff320029f80700d5010700e4
:10143c00aaff3200f6f60700d5010700a9ff32001b
:10144c0025f7070098010700a8ff3200391e070096
:10145c0098010700a7ff3200e91f07009b01070056
:10146c00a6ff3200daff3700ea2a0700beff37007a
:10147c00db2907006ed4bf000058a300baff32006e
:10148c00f9ff37006d54e200aeff35006201070032
:10149c00ed1d0700c3000700af010700feff36007b
:1014ac00c30007002c1d07006ed4bf000068a3000a
:1014bc00aaff3200eeff37006a34ef0073f4a80085
:1014cc007354e20080ff3d00d3ff37005701070043
:1014dc00dd1d0700b3000700efff37006d54e2007d
:1014ec00b3ff35004c010700d71d0700e833ef00b0
:1014fc009a000700feff3600a10007008aff3700a4
:10150c004a010700d01d0700e833ef00f8ff370051
:10151c0010c0b30016e8b7001600370030c0b30097
:10152c0016e8b7001600370020c0b30016e8b70065
:10153c002f0037005c94a8005cb4a9005cd4a9000f
:10154c005cf4a900113a2100914078000f0037009b
:10155c009140780060c4b30080cf500000000600ba
:10156c00909f8000b00e8800819f8000d10e880073
:10157c006c00370062d4bf000058a30000000600c6
:10158c0016c8bf0018e8b70000000600c0c4b300be
:10159c0080cf500000000600439d8000529d8000cb
:1015ac0010032000800f510000000600939f88005c
:1015bc00829f8800560037005500070020a4800049
:1015cc007f00b9000000d100609d8800c13d210062
:1015dc00ddff370020c4b300ddf3b700ddd3bf005f
:1015ec00dff3b700dc02a900dc82a80000000600d3
:1015fc0062d4bf000068a3000000060002002000b7
:10160c00832c240009bd070080a0880091a08800cd
:10161c00e1ff3700dc62a8002a003700e09c800064
:10162c002a003700e09f8800f19f880020a08000ee
:10163c0031a08000e29f8000f39f80003ebd070038
:10164c0020a0880031a08800e09f8000f19f8000de
:10165c0002a0800013a0800036bd070040a08800c7
:10166c0051a08800e09f8000f19f800000a08800be
:10167c0011a088002f01070020a0800031a080005d
:10168c00a2a08000b3a08000e7bd07000000e0002e
:10169c0000000600cfff07004b0037004b0107008e
:1016ac0073d4a8004b003700e13d2100a8ff3700a0
:1016bc00e13d21009140780020c4b30080cf500060
:1016cc0000000600d13d2100a1ff3700e09c800006
:1016dc00cf80de00a9bd07000001be000000200085
:1016ec00b151240013bd07000004be00e09c800033
:1016fc00cf80de00d0bd07006022b80006002600b7
:10170c00370a2400cfbd07000000e00000000600ef
:10171c00909f8000b00e8800809f8000d00e8800c3
:10172c0000000600c9c2bf000058a300000006005c
:10173c006a34ef0041a4800061998800a099800070
:10174c00b1998000809988009199880051a48000fb
:10175c0071998800e833ef0000000600419f80007b
:10176c00700c2000808f50000000060073f4a8005d
:10177c0070d4a80060c4b300def3b700000006000c
:10178c0073f4a90070f4a90070d4a9006e14a90018
:10179c00000006006a34ef008700070073f4a8000d
:1017ac000000060084000700e833ef00710c050010
:1017bc008100070070d92a0000000600d4ff070042
:1017cc0071d4bf000000060066d4bf000008a3005f
:1017dc0000000600ac33ef00aa33ef00a833ef0093
:1017ec000034ef000234ef000834ef000a34ef004d
:1017fc00fc33ef00fe33ef000434ef000634ef004f
:10180c000c34ef000e34ef0038a480006e0037006b
:10181c00c0d42100800f510000000600dc62a9003a
:10182c00a8ff370073f4a9007094a9007394a90061
:10183c006e74a80068c4b30000000600dc62a90046
:10184c00d13d21009140780088cf50000000060067
:10185c00daff07000048a30000000600a4a08000e7
:10186c00b5a0800024a0880035a0880000000600e8
:10187c00caa08000dba08000e89f8000f99f800058
:10188c00e0a08000f1a08000c0b79f00d1b79f00fe
:10189c002ca080003da0800000a1800011a1800040
:1018ac0042a0800053a0800084a0800095a08000fe
:1018bc00a4b79f00b5b79f00fcbc0700e0b79f0022
:1018cc00f1b79f000801be000a00be00f7bc07007c
:1018dc000004be000c01be004fb09700dfb09700b3
:1018ec00f2bc07000001be000800be0092bc07005d
:1018fc000001be006fb09700ffb097008ebc0700d0
:10190c002fb19700bfb19700e8bc070060a088001a
:10191c0071a088008700070060a0800071a0800083
:10192c0057ff3700a0a08000b1a0800060a0880005
:10193c0071a0880000000600689d800060a08000f7
:10194c0071a0800018bc070000045400589d88004a
:10195c0060a0800071a08000689d800012bc070010
:10196c0000044400489d88000bff3700919f8000c5
:10197c00b10e8800849f8000d40e88000000060001
:10198c00519d8000609d8000808f500000000600fb
:10199c00419d8000609d8000808f500000000600fb
:1019ac0070d4bf000038a30000000600929f88008e
:1019bc00839f880056ff3700cae2a800400620002b
:1019cc00c09e8800000006006140b900ebbc070017
:1019dc000800e000000006000001be000c00be0084
:1019ec0055bc07000005be0000000600740007008f
:1019fc000005be001904780000000600d233ef0089
:101a0c0040012000b09e880000000600e0c2bf002c
:101a1c000068a3000000060073f4a9006ab4a800d3
:101a2c003f00070080c62a00000006006a14a800c8
:101a3c00f0c72a00000006001768ef001668ef00d8
:101a4c001868ef0073d4bf000028a3000000060044
:101a5c0018c8bf00e24f5000000006007374a800c5
:101a6c0040c1b30048f3b7000000060062d4bf00c9
:101a7c000018a3000000060062d4bf000028a300d9
:101a8c000000060017c8bf0018e8b70000000600e9
:101a9c000801be000800be0084bc07000200200044
:101aac00a32f2c00e1bb370071d4bf000048a3006a
:101abc000000060071d4bf000038a300000006002f
:101acc0071d4bf000018a3000000060071d4bf0041
:101adc000058a3000000060071d4bf000028a3002a
:101aec00000006006640400080cf50000000060059
:101afc006440500080cf5000000006007074a900b4
:101b0c006ed4bf000038a30000000600113a21007b
:101b1c009140780030c5b30080cf50000000060023
:101b2c005c94a9005cb4a9005cd4a8005cf4a80087
:101b3c0000000600609d8000cf80de008fbc070097
:101b4c0002002000030a240058bc0700a0a0880053
:101b5c00b1a0880000000600409f8000810f50005b
:101b6c0000000600013e21009140780020c5b30022
:101b7c0080cf5000000006000040e80080cf5000ed
